:100000000C94D9230C940A240C940A240C940A24EA
:100010000C940A240C940A240C940A240C940A24A8
:100020000C940A240C940A240C940A240C940A2498
:100030000C940A240D94ED530C940A240C940A2475
:100040000C940A240C9497EF0C940A240C940A2420
:100050000C940A240C940A240C945EEC0D94A35383
:100060000C940A240C943B5F0C94315F0C940A248A
:100070000C940A240C940A240C940A240C940A2448
:100080000C94FA420C940A240C940A240C940A242A
:100090000C940A240C940A240C940A240C940A2428
:1000A0000C940A240C940A240C94CC420C940A2438
:1000B0000C940A240C940A240C940A240C940A2408
:1000C0000C940A240C940A240C940A240C940A24F8
:1000D0000C940A240C940A240C940A240C940A24E8
:1000E0000C940A24084AD73B3BCE016E84BCBFFD6A
:1000F000C12F3D6C74319ABD56833DDA3D00C77FF8
:1001000011BED9E4BB4C3E916BAAAABE0000008090
:100110003F05A84CCDB2D44EB93836A9020C50B91F
:10012000918688083CA6AAAA2ABE000000803F004B
:100130000C94899C0D94074E0C948C9C0C94E15F5C
:100140000C94CBDB0C946B920C947AB20C94D1E0AF
:100150000C9465AD0D94FD4D0C94759C0C94309AE7
:100160000C94D5D40C94E0930C94B79A0C9490BF53
:100170000C94F4D40C941ECB0C94959C0C94D0A9A4
:100180000C9475920C9493A70C94C2290C94B6DD30
:100190000C940CCB0C9418CB0C947B420C946C9A62
:1001A0000C94B9940C9436CB0D94114E0C94D193BD
:1001B0000C94BFB80C94BE3B0C94E6260C94389A71
:1001C0000C948D910C9454920C94929C0C94569295
:1001D0000C94B5B80C94999B0C94D15F0C941C9121
:1001E0000C94CADB0C946E960C949DB10C94D5CBF8
:1001F0000C9466920C946E900C94DADF0D94C64DBC
:100200000D941B4E0C9494D40C9460990C944690CD
:100210000C940F240D94DA4D0D94D04D0D944A4D4D
:100220000C945C990C94DB9A0C942A920C945F9138
:100230000C94809C0C946C940C94FB9C0C94CE2697
:100240000C9430CB0C94C4960C9437900C940F9A69
:100250000C942F910C94D6920C940DA80C94CAC6B1
:100260000C94B5900C9434970C94A85F0D942E4D7B
:100270000D94984D0D94444D0D94244D0C94689913
:100280000C949A9C0C948F9C0C947C990C949E9A40
:100290000C9452DE0C9448910C945F900C94D09A7C
:1002A0000C94F89C0C94FA900C9415C10C9448DBB7
:1002B0000C9400CB0C9407E00D94F72E0C94958DC4
:1002C0000D941E4D0D941B4D0D94174D0C94AD9235
:1002D0000C94EECA0C941E900C94C8DF0C9446C289
:1002E0000D94485E0C94A2900C942FDF0C9435DE94
:1002F0000C94E1900C94AB940C94F75F0C94FACAB4
:100300000C94B3940C94D9920C94CADE0D94934D32
:100310000C94EFAE0C9452920C94EBDE0C94709211
:100320000C941EDD0C9458990C94A08D0C9424CB45
:100330000D94A24D0C94C7920C94A4910C94A8BD5A
:100340000C9489900C94FF5F0C9421940D94002ED2
:100350000C9406CB0C94E55F0C94839C0C9475D4A0
:100360000D948B4D0C94795F0C94D55F0C94C096D2
:100370000D94A12D0C94EB290C940C240C9499A4AD
:100380000C9403D40C9429950C9422D40C940991C8
:100390000C94859A0D94F84C0D94FD4C0C9433926A
:1003A0000D944E4D0D94BE4D0C9470990C947D9B04
:1003B0000C9405900C9462960C94FA920C946192B1
:1003C0000C945D940D94E44D0C9412CB0D94B64DA9
:1003D0000C94B7940D94F34D0C94C65F0C94AF45F8
:1003E0000C9489240C94DC920C9465B00C94AF941A
:1003F0000C9460420C942ACB0C94C8900C94B19449
:100400000C94F79E0C9496420C94B5940C947499A9
:100410000C9425CF0C94EC5F0C9489A70C94869CCB
:100420000C9478990C94CFAF0C9498A70C94A29C40
:100430000C948F930C94779B0D94254E0C943F92C3
:100440000C94CAA00C941ED50C94A9BA0C944ADF43
:100450000C948E9B0C94AD940D949A5E0D94CE2DBD
:100460000C949F9C0D94134D0C9464990C94B75F5D
:100470000C9404B10C94BC960C949BCB0D94364D0B
:100480000C946C990C94728D0C94169D0D940F4DD8
:100490000C948EA70C9476910D94324D0C94D7B891
:1004A0000C94CD5F0C94E0B50C9423C90C949C9CE7
:1004B0000C94F4CA0C94F88D0D94AC4D0C94DF920E
:1004C0000D94B85E0D94404D0C94D5A10D943C4D07
:1004D0000C9440AC0C94859B0C94DD5F0C94DF8DE8
:1004E0000D94284D0C94B1420C94EBB30C94D95F4D
:1004F0000C944D2A0C9414B74E414E494E49545910
:10050000494E46CDCCCC3D0AD7233C17B7D13877DE
:10051000CC2B329595E6241FB14F0A0000204100F4
:1005200000C84200401C4620BCBE4CCA1B0E5AAE3E
:10053000C59D7400407A10F35A00A0724E1809004D
:1005400010A5D4E80000E87648170000E40B540238
:100550000000CA9A3B000000E1F505000080969873
:1005600000000040420F000000A0860100000010C3
:100570002700000000E80300000000640000000005
:10058000000A00000000000100000000002C76D8E6
:1005900088DC674F0823DFC1DFAE59E1B1B796E5CC
:1005A000E3E453C63AE651997696E8E6C28426EB30
:1005B000898C9B62ED407C6FFCEFBC9C9F40F2BA43
:1005C000A56FA5F490055A2AF75C936B6CF9676DDB
:1005D000C11BFCE0E40D47FEF520E6B500D0ED9030
:1005E0002E0300943577050080841E080000204EFD
:1005F0000A000000C80C333333330F986E12831196
:1006000041EF8D2114893BE65516CFFEE6DB18D16C
:10061000844B381BF77C1D901DA4BBE4242032843E
:10062000725E228100C9F124ECA1E53D27434F4DC4
:100630004D554E49434154494F4E0044525952552D
:100640004E004552524F525300494E464F004543CB
:10065000484F004572726F722077726974696E67D5
:1006600020746F20454550524F4D210A0053544F7E
:10067000505045442E20005072696E74657220738C
:10068000746F707065642064756520746F20657286
:10069000726F72732E2046697820746865206572C7
:1006A000726F7220616E6420757365204D3939391F
:1006B00020746F20726573746172742E20285465E3
:1006C0006D706572617475726520697320726573EF
:1006D00065742E2053657420697420616674657298
:1006E0002072657374617274696E67290A004E6FB7
:1006F00020436865636B73756D2077697468206C3F
:10070000696E65206E756D6265722C204C61737424
:10071000204C696E653A20004E6F20436865636B1C
:1007200073756D2077697468206C696E65206E75CD
:100730006D6265722C204C617374204C696E653A51
:100740002000636865636B73756D206D69736D61FF
:100750007463682C204C617374204C696E653A2078
:10076000004C696E65204E756D626572206973205C
:100770006E6F74204C617374204C696E65204E75E9
:100780006D6265722B312C204C617374204C696E44
:10079000653A20004D3131300053657269616C203B
:1007A000737461747573206D69736D617463680A25
:1007B00000776169740A00534420726561642065A2
:1007C00072726F720A00486F74656E642049646CBF
:1007D000652054696D656F757400486F74656E644B
:1007E0002049646C652054696D656F75740A002139
:1007F00021204B494C4C20636175736564206279FC
:10080000204B494C4C20627574746F6E2F70696E6A
:100810000A002121204B494C4C20636175736564AB
:1008200020627920746F6F206D75636820696E6136
:1008300063746976652074696D65202D2063757217
:1008400072656E7420636F6D6D616E643A20007026
:1008500061757365004D363030002066696C616DDE
:10086000656E745F72756E6F7574200066696C6179
:100870006D656E745F72756E6F7574205400466995
:100880006C616D656E7452756E6F75742054004D99
:10089000656469612052656D6F766564004D6564BD
:1008A000696120496E736572746564004D31303042
:1008B000305300627573793A2070617573656420F6
:1008C000666F7220696E7075740A00627573793A8A
:1008D0002070617573656420666F72207573657230
:1008E0000A00627573793A2070726F636573736979
:1008F0006E670A00506C656173652052657365749C
:10090000005052494E5445522048414C54454400F1
:1009100025533A20255300706F7765726F66660025
:100920004B494C4C45442E20005072696E746572E0
:100930002068616C7465642E206B696C6C282920BA
:1009400063616C6C6564210A0053544F50504544F8
:100950002E20005072696E7465722073746F70700F
:1009600065642064756520746F206572726F7273A0
:100970002E2046697820746865206572726F722037
:10098000616E6420757365204D39393920746F208C
:10099000726573746172742E202854656D7065726F
:1009A00061747572652069732072657365742E2099
:1009B0005365742069742061667465722072657372
:1009C00074617274696E67290A006563686F3A0022
:1009D0004572726F723A0042696C696E656172208D
:1009E0004C6576656C696E6720477269643A0A00E7
:1009F00021212053544F502063616C6C6564206248
:100A0000656361757365206F6620424C546F756332
:100A100068206572726F72202D2072657374617226
:100A2000742077697468204D3939390A00212120F2
:100A300053544F502063616C6C6564206265636140
:100A4000757365206F6620424C546F75636820652E
:100A500072726F72202D20726573746172742077C8
:100A6000697468204D3939390A005072696E7469A9
:100A70006E67204F626A6563740025532025690004
:100A80002F2F616374696F6E3A0073746172740022
:100A900070726F6D70745F00656E6400486F74658E
:100AA0006E6420746F6F20636F6C640A0053656E10
:100AB00064204D31303820746F20726573756D6518
:100AC0000A00496E736572742066696C616D656EAB
:100AD0007420616E642073656E64204D3130380A75
:100AE0000052656865617420446F6E6500526568E8
:100AF000656174696E672E2E2E005265686561749B
:100B0000004865617465722054696D656F75740085
:100B100053656E64204D31303820746F20686561F4
:100B200074206E6F7A7A6C650A004E6F7A7A6C6503
:100B3000205061726B65640070617573656400506C
:100B40006175736500726573756D656400526573D8
:100B5000756D696E67004732362043616E63656C60
:100B60006564004732362048656174696E67204EBF
:100B70006F7A7A6C65004732362048656174696E19
:100B800067204265640057616974696E6720666F0B
:100B900072206865617475702E0A00466978656414
:100BA000204C656E677468205072696D6500446FF3
:100BB0006E65205072696D696E67004D616E75617A
:100BC0006C207072696D696E672E2E2E004C656107
:100BD00076696E6720473236003F537065636966F9
:100BE00069656420582C5920636F6F7264696E6167
:100BF0007465206F7574206F6620626F756E647304
:100C00002E0A003F28522965706561742076616C58
:100C10007565206E6F7420706C61757369626C65A8
:100C20003B206D757374206265206174206C656172
:100C3000737420312E0A003F5370656369666965DD
:100C400064206E6F7A7A6C652074656D7065726170
:100C500074757265206E6F7420706C617573696253
:100C60006C652E0A003F5370656369666965642090
:100C700066696C616D656E742073697A65206E6F4C
:100C80007420706C61757369626C652E0A003F5345
:100C90007065636966696564207072696D65206C52
:100CA000656E677468206E6F7420706C617573690F
:100CB000626C652E0A003F537065636966696564FE
:100CC000206E6F7A7A6C652073697A65206E6F7416
:100CD00020706C61757369626C652E0A003F526505
:100CE0007472616374696F6E204D756C7469706C99
:100CF000696572206D757374206265207370656319
:100D000069666965642E0A003F53706563696669A8
:100D100065642052657472616374696F6E204D75ED
:100D20006C7469706C696572206E6F7420706C6190
:100D3000757369626C652E0A003F5370656369665E
:100D4000696564206C61796572206865696768749B
:100D5000206E6F7420706C61757369626C652E0A09
:100D60000043292E0A003F53706563696669656414
:100D7000206265642074656D70657261747572655A
:100D8000206E6F7420706C61757369626C652028C9
:100D900034302D00473236207374617274696E6787
:100DA0002E2E2E0A004F46460A00466164652048F2
:100DB00065696768742000426564204C6576656CDF
:100DC000696E6720004661696C656420746F2065F8
:100DD0006E61626C6520426564204C6576656C6965
:100DE0006E670A00496E76616C6964206D65736890
:100DF0002E0A0050726F62696E6720506F696E74C0
:100E00000025532025692F2569002E0A002F005048
:100E1000726F62696E67206D65736820706F696EAE
:100E2000742000202844525952554E290047323927
:100E3000204175746F20426564204C6576656C694D
:100E40006E67003F20284C2C522C462C4229206FE4
:100E50007574206F6620626F756E64732E0A003F92
:100E60002856296572626F7365206C6576656C2003
:100E7000696D706C61757369626C652028302D3402
:100E8000292E0A00426164205A2076616C75650A39
:100E9000004E6F2062696C696E65617220677269CD
:100EA000640A00446576696174696F6E0025533A7F
:100EB0002025730046696E6973686564210A003AEB
:100EC000207A3A2000206F662000476F696E672005
:100ED000746F3A20580043570A00206469723A0040
:100EE00020616E676C653A005374617274207261A0
:100EF000646975733A004D343820506F696E740020
:100F000025533A2025642F256400506F7369746956
:100F10006F6E696E67207468652070726F62652EEF
:100F20002E2E0A003F4C656773206F66206D6F762A
:100F3000656D656E7420696D706C61757369626C46
:100F4000652028302D3135292E0A003F2028582CC5
:100F50005929206F7574206F6620626F756E6473F7
:100F60002E0A0050726F6265206F7574206F6620C4
:100F7000626F756E6473003F53616D706C652073B2
:100F8000697A65206E6F7420706C61757369626C2C
:100F9000652028342D3530292E0A004D3438205A4A
:100FA0002D50726F6265205265706561746162696F
:100FB0006C69747920546573740A003F285629655A
:100FC00072626F7365206C6576656C20696D706CFC
:100FD00061757369626C652028302D34292E0A00F2
:100FE0005374616E646172642044657669617469EA
:100FF0006F6E3A20002052616E67653A2000204DE6
:1010000061783A2000204D696E3A200020536967CC
:101010006D613A20004D65616E3A2000205200411A
:101020006363656C65726174696F6E3A2050005736
:1010300041524E494E4721204C6F77205A204A6535
:10104000726B206D6179206C65616420746F20750E
:101050006E77616E746564207061757365732E0AB6
:10106000004F4646004F4E0020204D61783A200048
:10107000200020204D696E3A2000536F6674206571
:101080006E6473746F70733A20004D3234205325B0
:101090006C642054256C64004739322E3920452574
:1010A0007300473120462564004739322E39205AD3
:1010B0002573004731205A30204632303000473106
:1010C0002058257320592573204633303030004D89
:1010D00034323020532569205A2573004D31303683
:1010E0002050256920532569004D32303020442599
:1010F000730047323852305859004739322E392060
:101100004530205A300A47315A2573004D31303965
:1011100020532569004D31393020532569004D3465
:101120003230205330205A300020496E76616C698D
:1011300064206578747275646572200047322F47A9
:10114000332062616420706172616D6574657273D1
:101150000A00536C6565702E2E2E005A2050726F57
:1011600062652050617374204265640A005A205001
:10117000726F62652050617374204265640047326B
:10118000384C30004D3131372050726F6265206627
:1011900061696C65642E0A4732380A0070726F62AA
:1011A000655F7265776970650047323920526574F2
:1011B0007279696E670050726F62696E672046616E
:1011C000696C6564004D31313720426564206C657F
:1011D00076656C696E67206661696C65642E0A4786
:1011E00030205A31300A4D333030205032352053C0
:1011F0003838300A4D333030205035302053300AE3
:101200004D3330302050323520533838300A4D338A
:101210003030205035302053300A4D33303020509C
:10122000323520533838300A4D3330302050353085
:101230002053300A47342053310070726F62655F6B
:101240006661696C6564004D313137204265642008
:101250006C6576656C696E6720646F6E652E002024
:101260005A3A200020593A200042656420583A201A
:10127000004D65736820706F696E74206F757420FF
:101280006F662072616E67650A004D302053746F7F
:1012900070004D312053746F7000436C69636B2094
:1012A000746F20526573756D652E2E2E004E6F2063
:1012B0004D6F76652E00456E642066696C65206C06
:1012C0006973740A00426567696E2066696C6520FF
:1012D0006C6973740A004E6F206D656469610A0061
:1012E000526573756D696E6720534400286E6F20D8
:1012F00066696C65290043757272656E7420666953
:101300006C653A20005072696E742074696D653A9C
:1013100020000A53746174733A2046696C616D65EC
:101320006E7420757365643A20002C204C6F6E67D4
:10133000657374206A6F623A2000546F74616C2088
:1013400074696D653A200053746174733A20002CFF
:10135000204661696C65643A20002C2046696E69FC
:10136000736865643A20005072696E74733A2000A5
:1013700053746174733A2000436F6F6C696E672E0B
:101380002E2E0048656174696E672E2E2E00452052
:101390002553006F6B006F6666004E0649064206D5
:1013A0003B062D0644454255473A004D3131332026
:1013B000530042656420436F6F6C696E672E2E2E5A
:1013C000004265642048656174696E672E2E2E00A8
:1013D000544D334420435231305632204F46462E2E
:1013E000002F2F004D31343520533C696E646578F1
:1013F0003E206F7574206F662072616E67652028CD
:10140000302D31290A004D32303620580046523AEC
:101410000020466C6F773A20003A20002053657216
:10142000766F2000206F7574206F662072616E6782
:10143000650A00536572766F200020643A002069C7
:101440003A0020703A00496E76616C6964206578D4
:101450007472756465720A0020643A0020693A006B
:1014600020703A0064697300656E0043290A0061C8
:10147000626C656420286D696E2074656D70200053
:10148000436F6C6420657874727564657320617253
:1014900065200046696C616D656E742072756E6FB3
:1014A00075742064697374616E636520286D6D299D
:1014B0003A200046696C616D656E742072756E6FBE
:1014C000757420004D34323120696E636F7272651D
:1014D000637420706172616D6574657220757361EB
:1014E00067650A004D65736820706F696E74206FC0
:1014F0007574206F662072616E67650A004F6666BC
:1015000073657473204170706C6965640045727214
:101510003A20546F6F206661722100546F6F20660D
:1015200061722066726F6D207265666572656E63AA
:101530006520706F696E740A00454550524F4D200A
:101540004F4B0A00506F7765722D6C6F737320726A
:1015500065636F7665727920004D383400446F6E94
:1015600065207072696E74696E672066696C650AC1
:10157000004D3737004D3331004361703A004D451F
:1015800041545041434B00434F4F4C45525F5445EB
:101590004D5045524154555245004348414D4245F6
:1015A000525F54454D5045524154555245004241B9
:1015B00042595354455050494E47004152435300FD
:1015C0004D4F54494F4E5F4D4F444553005448458D
:1015D000524D414C5F50524F54454354494F4E0079
:1015E0004C4F4E475F46494C454E414D4500415595
:1015F000544F5245504F52545F53445F53544154DB
:1016000055530053445F5752495445005245504585
:101610004154005344434152440050524F4D5054A2
:101620005F535550504F525400454D455247454E1B
:1016300043595F50415253455200434153455F4C1B
:10164000494748545F4252494748544E4553530016
:10165000544F47474C455F4C494748545300534FFC
:101660004654574152455F504F57455200425549E5
:101670004C445F50455243454E54004C4556454CF2
:10168000494E475F44415441005A5F50524F4245D2
:101690000052554E4F5554004155544F4C455645F8
:1016A0004C005052494E545F4A4F420050524F47EF
:1016B00052455353004155544F5245504F52545F79
:1016C00054454D5000564F4C554D455452494300DA
:1016D000454550524F4D0042494E4152595F46498F
:1016E0004C455F5452414E53464552005345524972
:1016F000414C5F584F4E5F584F4646004649524D49
:10170000574152455F4E414D453A4D61726C696E8D
:1017100020322E302E375F4457372E3320544D332E
:10172000442053534D4442422028417072203234A9
:1017300020323032312032323A32313A30312920BF
:10174000534F555243455F434F44455F55524C3AC2
:1017500068747470733A2F2F6769746875622E63AA
:101760006F6D2F496E73616E6974794175746F6D19
:101770006174696F6E2F4D61726C696E2F74726542
:10178000652F437265616C6974794477696E5F3265
:101790002E302050524F544F434F4C5F56455253BA
:1017A000494F4E3A312E30204D414348494E455F16
:1017B000545950453A544D334420435231305632F7
:1017C0002045585452554445525F434F554E543A64
:1017D0003120555549443A63656465326132662D5E
:1017E000343161322D343734382D396231322D6342
:1017F00035356336326633363766660A0050726FA7
:101800006265204F6666736574205A0050726F627D
:1018100065204F6666736574205A00290A0020749B
:101820006F20003F5A206F7574206F662072616EC2
:101830006765202800290A0020746F20003F592086
:101840006F7574206F662072616E676520282D00A9
:10185000290A0020746F20003F58206F7574206F94
:10186000662072616E676520282D0050726F626578
:10187000204F666673657420580043616E6E6F7406
:10188000206F70656E20737562646972200025692F
:10189000730025696D202569730025696820256915
:1018A0006D202569730025696420256968202569F4
:1018B0006D202569730025697920256964202569D3
:1018C000682025696D202569730023646566696E4B
:1018D000652044454641554C545F00626564004BA9
:1018E0006420004B6920004B702000504944204187
:1018F00075746F74756E652066696E69736865646A
:10190000212050757420746865206C617374204BBD
:10191000702C204B6920616E64204B6420636F6ED5
:101920007374616E74732066726F6D2062656C6F84
:101930007720696E746F20436F6E66696775726198
:1019400074696F6E2E680A00504944204175746FA7
:1019500074756E65206661696C6564212074696DBB
:10196000656F75740A00504944204175746F747531
:101970006E65206661696C6564212054656D7065D3
:1019800072617475726520746F6F20686967680A88
:1019900000204B643A2000204B693A2000204B7015
:1019A0003A200020436C61737369632050494420DE
:1019B0000A00204E6F206F76657273686F6F740A2D
:1019C000002054753A2000204B753A2000206D61AC
:1019D000783A2000206D696E3A200020643A200099
:1019E00020626961733A2000504944204175746F48
:1019F00074756E652073746172740A0050494420D6
:101A00004175746F74756E65206661696C656421DB
:101A10002054656D706572617475726520746F6FA6
:101A200020686967680A00504944204175746F74E2
:101A3000756E6500504944204175746F74756E650C
:101A4000206661696C65642120426164206865617B
:101A50007465722069640A004572723A2075746672
:101A60003820666F6E74206E6F7420696E697469B9
:101A7000616C697A65642E004572723A20757466ED
:101A80003820666F6E74206E6F7420696E69746999
:101A9000616C697A65642E004572723A20757466CD
:101AA0003820666F6E74206E6F7420696E69746979
:101AB000616C697A65642E00000C0F00FE07022538
:101AC00003BB017FFE08FE08FE0508080600004073
:101AD000F0C88888987810050808060000C0F888C3
:101AE00088888888F80505050600012030F8302030
:101AF0000508080600002070F820202020E00509D5
:101B0000090600FF2070A8A8B8888870200705057E
:101B1000070001D86C366CD80509090600FFF8A843
:101B20008888888888A8F8050A0A0600FE20505090
:101B3000505088A8A8887003030306000340A04003
:101B4000FFFFFFFFFFFFFFFFFFFFFFFFFFFFFFFFA5
:101B5000FFFFFFFFFFFF0000000605FF010707066C
:101B6000020080808080800080030303060105A0BE
:101B7000A0A005060606000050F85050F8500509D0
:101B8000090600FF2070A8A07028A870200507078C
:101B9000060000C8C81020409898050707060000F6
:101BA00040A0A040A8906801030306020580808041
:101BB0000309090601FF2040408080804040200347
:101BC00009090601FF804040202020404080050791
:101BD0000706000020A8702070A820050505060053
:101BE000012020F820200203030601FFC0408005E9
:101BF0000101060003F8020202060100C0C0050749
:101C00000706000008101020404080050707060066
:101C100000708898A8C8887003070706010040C0B4
:101C200040404040E005070706000070880810208B
:101C300040F8050707060000F8081030088870050E
:101C4000070706000010305090F81010050707062F
:101C50000000F880F00808887005070706000030CB
:101C60004080F0888870050707060000F80810100B
:101C7000202020050707060000708888708888707B
:101C800005070706000070888878081060020505BF
:101C9000060100C0C000C0C00206060601FFC0C0A9
:101CA00000C040800305050601012040804020055A
:101CB0000303060002F800F8030505060101804051
:101CC00020408005070706000070881020200020B3
:101CD0000507070600007088B8A8B88070050707D8
:101CE000060000708888F8888888050707060000C5
:101CF000F04848704848F0050707060000708880E3
:101D000080808870050707060000F048484848486A
:101D1000F0050707060000F88080F08080F80507CE
:101D200007060000F88080F0808080050707060025
:101D300000708880809888700507070600008888F2
:101D400088F8888888030707060100E04040404083
:101D500040E00507070600003810101010906005DD
:101D600007070600008890A0C0A090880507070616
:101D70000000808080808080F805070706000088CA
:101D8000D8A8888888880507070600008888C8A81A
:101D900098888805070706000070888888888870FA
:101DA000050707060000F08888F080808005070797
:101DB00006000070888888A890680507070600005C
:101DC000F08888F0A09088050707060000708880DA
:101DD00070088870050707060000F82020202020E2
:101DE000200507070600008888888888887005070E
:101DF00007060000888888885050200507070600DD
:101E00000088888888A8A8500507070600008888E9
:101E10005020508888050707060000888850202039
:101E20002020050707060000F80810204080F8036E
:101E300009090601FFE080808080808080E005073E
:101E40000706000080404020101008030909060121
:101E5000FFE020202020202020E0050303060005CD
:101E60002050880501010600FEF803030306010562
:101E70008040200505050600007008788878050771
:101E8000070600008080F0888888F00505050600B8
:101E900000708080887005070706000008087888B1
:101EA0008888780505050600007088F080700507B1
:101EB00007060000304840E04040400507070600A4
:101EC000FE70888888780870050707060000808003
:101ED000F0888888880307070601004000C040405A
:101EE00040E00409090601FE1000301010101090A7
:101EF0006005070706000080808890E0908803074F
:101F000007060100C04040404040E00505050600CE
:101F100000D0A8A8A8A8050505060000B0C88888B4
:101F20008805050506000070888888700507070683
:101F300000FEF0888888F080800507070600FE789C
:101F4000888888780808050505060000B0C88080E4
:101F50008005050506000078807008F00507070673
:101F600000002020F8202020180505050600008824
:101F7000888898680505050600008888885020052F
:101F800005050600008888A8A8500505050600007C
:101F900088502050880507070600FE888888502052
:101FA0004080050505060000F8102040F8030909E7
:101FB0000601FF20404040804040402001090906C2
:101FC00002FF808080808080808080030909060174
:101FD000FF8040404020404040800503030600024F
:101FE00048A890FF554E4C4F41442046494C414D26
:101FF000454E54004C4F41442046494C414D454EBE
:10200000540046494C414D454E54204348414E47AB
:10201000450042656400456E636C6F7375726500C0
:102020002568753A25303268750025303268753A72
:10203000253032687500202020202020200020201C
:102040002020001FE0201020102010102010202041
:1020500010201030300840048003001FE03FF03FA4
:10206000F03FF01FE01FE03FF03FF03FF00FC007F0
:102070008003003FFFF038007030FC3020FC10205F
:1020800078102030102C00D02E31D02F7BD02F7B19
:10209000D02E31D02C00D020301020781020FC1011
:1020A00030FC303800703FFFF03FFFF038007031F7
:1020B00086302387102787902F87D02F03D020309A
:1020C000102078102078102030102F03D02F87D0C8
:1020D0002787902387103186303800703FFFF01F2C
:1020E000FFF81FFFF8041040020820020820041027
:1020F000400820801041001041000820800410405A
:102100000000001FFFF81FFFF8FFFFFF8000018E97
:1021100000E19F01F19381399F81F99F81F99FB976
:10212000F98F28F18038018000019FFFF99174999F
:102130009B06A99B54A99B56A99B54999FFFF9FF05
:10214000FFFF6E6F74696669636174696F6E20006A
:1021500063616E63656C005072696E742041626FDA
:1021600072746564004469736D6973730055492026
:1021700041626F72746564004D323520500A4D32F1
:102180003400526573756D65005549205061757353
:10219000650050617573696E672E2E2E007265732F
:1021A000756D65004D32340000FE0003FF8007C7E7
:1021B000C00701E00000E00000F0000070040070C3
:1021C0000E00701F00703F80F00E00E00F01E0076E
:1021D000C7C003FF8000FE0000FE0003FF8007C7AA
:1021E000C00F01E00E00E03F80F01F00700E007095
:1021F0000400700000700000F00000E00701E0073C
:10220000C7C003FF8000FE000E000E000E000E008F
:102210000E000E000E000E007FC03F801F000E005B
:10222000040004000E001F003F807FC00E000E005F
:102230000E000E000E000E000E000E00FFFFFF7FCE
:1022400080FFC0FFC0FFC07F807F80FFC0FFC0FF56
:10225000C03F001E000C0050726F6265205A204F74
:1022600066667365740052756E6F75742044697389
:1022700074206D6D004C6F6164206D6D00556E6C47
:102280006F6164206D6D0046696C2E204469612E7B
:10229000004520696E206D6D5E33004D3330332074
:1022A0005531204525692053256900504944204176
:1022B00075746F74756E65202A005049442D442052
:1022C0002A005049442D49202A005049442D5020CD
:1022D0002A0020082046616374002008204D6178A0
:1022E000002008204D696E004F6666004F6E004169
:1022F00075746F74656D70005654726176204D6907
:102300006E00566D696E00566D6178204500566D01
:102310006178205A00566D6178205900566D6178B9
:10232000205800416D6178204500416D6178205A48
:1023300000416D6178205900416D6178205800415D
:102340002D54726176656C00412D52657472616323
:102350007400416363656C0056652D4A65726B00BD
:10236000565A2D4A65726B0056592D4A65726B009C
:1023700056582D4A65726B0050726F6265205A2064
:102380004F66667365740050726F62652059204F06
:1023900066667365740050726F62652058204F66E0
:1023A0006673657400452073746570732F6D6D00DE
:1023B0005A2053746570732F6D6D005920537465E6
:1023C00070732F6D6D00582053746570732F6D6D91
:1023D00000416476616E6365642053657474696E50
:1023E0006773003F0043616E63656C00496E6974FA
:1023F000004D34323800496E697469616C697A65E0
:1024000020454550524F4D0046696C616D656E74B4
:102410000054656D70657261747572650053746502
:1024200070732F6D6D0050726F6265204F6666731A
:10243000657473004A65726B00416363656C657215
:102440006174696F6E0056656C6F636974790053CF
:10245000657420486F6D65204F6666736574730000
:10246000436F6E66696775726174696F6E003F00D5
:102470004E65787420506F696E7400446F6E65000D
:102480004E65787400486F6D696E672058595A0020
:102490003F0043616E63656C204F626A6563740040
:1024A0004E4F005945530043616E63656C204F6287
:1024B0006A656374203D004D61696E0053746F77E7
:1024C000004465706C6F790053656C662D546573BC
:1024D000740053572D4D6F64650052657365740029
:1024E000426564004E6F7A7A6C650046616E2053D7
:1024F0007065656400436F6E6669677572617469C3
:102500006F6E004C6F61642053657474696E6773FD
:1025100000526573746F72652044656661756C74F2
:10252000730053746F72652053657474696E6773BA
:102530000050726568656174202420436F6E6600E8
:10254000506F776572204F7574616765004F6666DE
:10255000004F6E0052756E6F75742053656E736F09
:102560007200424C546F7563680050726F62652050
:102570005A204F666673657400416476616E6365C8
:10258000642053657474696E6773004D61696E00F1
:102590004D37303220542564004D363030204230E3
:1025A00020542564004D373032203B2564004D37E0
:1025B000303120542564004D373032004D373031F2
:1025C000004D363030204230004D61696E004F665C
:1025D00066004F6E0052756E6F75742053656E7392
:1025E0006F72005075726765206D6F726500436F82
:1025F0006E74696E756500524553554D45204F50B8
:1026000054494F4E533A005052494E542050415570
:102610005345440020204E6F7A7A6C653A20005072
:1026200061726B696E672E2E2E000000576169740F
:1026300020666F720066696C616D656E74206368F8
:10264000616E676500746F20737461727400576106
:10265000697420666F720066696C616D656E7420C6
:10266000756E6C6F616400004E6F7A7A6C652068DD
:10267000656174696E6700506C6561736520776190
:1026800069742E2E2E00005072657373206275746B
:10269000746F6E00746F2068656174206E6F7A7A53
:1026A0006C650000496E736572742066696C616DBB
:1026B000656E7400616E642070726573732062755C
:1026C00074746F6E00746F20636F6E74696E7565DD
:1026D000005761697420666F720066696C616D6590
:1026E0006E74206C6F6164000050726573732042D9
:1026F0007574746F6E00746F20726573756D6520EC
:102700007072696E7400005761697420666F722080
:102710007072696E7400746F20726573756D652ECA
:102720002E2E00005761697420666F720066696C16
:10273000616D656E7420707572676500003E2000E3
:10274000256C642E25696D00457874727564656426
:1027500020546F74616C003E20004C6F6E6765738F
:1027600074204A6F622054696D65003E2000546FEA
:1027700074616C205072696E742054696D650043F9
:102780006F6D706C65746564003A20005072696EFC
:102790007420436F756E74003A2000313530003577
:1027A000004245443A204154432031303447542DAF
:1027B000320052756E617761792057617463683AAF
:1027C000204F4E004D61782054656D7000333135D7
:1027D000004D696E2054656D7000350045313A201A
:1027E0004550434F53203130304B00505355004734
:1027F000656E657269630050726F746F636F6C0011
:10280000312E300042617564003235303030300096
:10281000437265616C69747933442052414D505361
:102820000042696C696E656172204C6576656C6901
:102830006E67004578747275646572730031007458
:10284000696E796D616368696E657333642E636F59
:102850006D00544D334420435231305632003230F3
:1028600032312D30342D313800322E302E375F4446
:1028700057372E33004D61726C696E005072696E6D
:1028800074657220537461747300546865726D6965
:1028900073746F727300426F61726420496E666F69
:1028A000005072696E74657220496E666F004D61EA
:1028B000696E004D313030300053746F70205072AB
:1028C000696E7400526573756D65205072696E741F
:1028D00000506F776572204F7574616765004D31E8
:1028E00039305335350A4732380A4732390A4D34C0
:1028F00030300A4D313034533231350A4732380ADC
:102900004D313039533231350A4D34323053310A7A
:102910004731583130305931303046353030300A57
:1029200047315A300A4D3530300A4D313137205356
:102930006574205A204F6666736574004D313036D9
:10294000533132380A4D3330334338533231354501
:1029500030550A4D3530300A4D3131372050494419
:102960002054756E6520446F6E65004D31393053CB
:1029700035350A4D313034533231350A4732380A51
:102980004732394C310A47312058313030593130D3
:102990003046353030300A47315A30004D3530300E
:1029A0000A4D3131372053657474696E6773205353
:1029B000746F726564005072657020666F72205A81
:1029C0002041646A757374005049442054756E65E3
:1029D0000053746F72652053657474696E67730079
:1029E0005365747570004D61696E003F004261630C
:1029F0006B0053746F70005072696E742066726F52
:102A00006D204D65646961004368616E6765204DA6
:102A100065646961004D32310041626F7574205008
:102A200072696E746572004368616E6765204669FD
:102A30006C616D656E74004C6576656C696E6720BF
:102A4000546F6F6C7300436F6E6669677572617463
:102A5000696F6E0054656D706572617475726500A2
:102A60004D6F74696F6E00486F7374205374617298
:102A70007400526573756D65205072696E74004EF6
:102A80006F204D656469610043616E63656C204F22
:102A9000626A6563740054756E650053746F7020CC
:102AA0005072696E74005061757365205072696E62
:102AB0007400496E666F2053637265656E003F0057
:102AC0005374617274205072696E740043616E6356
:102AD000656C005072696E740043616E6E6F742095
:102AE000656E746572207375626469723A200002C3
:102AF0002E2E004D61696E002100486F74656E6472
:102B000020746F6F20636F6C64004261636B0050D0
:102B1000726F6365656400536F667420456E6473FD
:102B2000746F7073004D6F74696F6E0044697361E8
:102B3000626C65205374657070657273004D383433
:102B4000004D34382050726F6265205465737400F4
:102B50004732384F0A4D343820503130004C6576BA
:102B6000656C20436F726E65727300466164652008
:102B7000486569676874004F6666004F6E0042657D
:102B800064204C6576656C696E67004C6576656C93
:102B900020426564004732394E00486F6D65205A07
:102BA000004732385A00486F6D6520590047323867
:102BB0005900486F6D6520580047323858004175FC
:102BC000746F20486F6D6500473238004D61696E43
:102BD0000050726568656174202420456E64005061
:102BE0007265686561742024204265640054656DD7
:102BF000706572617475726500436F6F6C646F7796
:102C00006E005072656865617420240046616E2014
:102C10005370656564207E00426564004E6F7A7A69
:102C20006C65004D61696E0050726F6265205A20BC
:102C30004F666673657400466C6F770046616E2060
:102C40005370656564207E00426564004E6F7A7A39
:102C50006C65005370656564004D61696E00486F76
:102C60006D696E67204661696C6564006F70656EA2
:102C700000545249474745524544003A200066698E
:102C80006C616D656E74007A5F6D696E00795F6D61
:102C9000696E00785F6D696E005265706F7274695D
:102CA0006E6720656E6473746F70207374617475E1
:102CB000730A0020746F6F206C6F6E6720657874E4
:102CC000727573696F6E2070726576656E74656477
:102CD0000A0020636F6C6420657874727573696F85
:102CE0006E2070726576656E7465640A00486F6D5B
:102CF0006520257325732573204669727374005708
:102D000061726E696E673A20486F6D696E67204226
:102D1000756D702044697669736F72203C20310AAA
:102D2000000202040000000000000000000000009B
:102D300000809D4300009B430000C8430000004109
:102D40000000004100000040FFFFFF000000010004
:102D50000000010000800055555500000040003380
:102D6000333300AAAA2A004992240000002000C799
:102D7000711C0099991900D1451700555515003B54
:102D8000B113002449120011111100000010000FAE
:102D90000F0F00E3380E0043790D00CCCC0C00C3BC
:102DA000300C00E8A20B0064210B00AAAA0A0070F4
:102DB0003D0A009DD80900427B090092240900DCED
:102DC000D30800888808001042080000000800F0BE
:102DD000C107008787070075500700711C07003E78
:102DE000EB0600A1BC06006990060066660600704E
:102DF0003E06006118060017F4050074D105005B5B
:102E0000B00500B2900500627205005555050078C6
:102E1000390500B81E0500050505004EEC040087C5
:102E2000D40400A1BD040090A7040049920400C18D
:102E30007D0400EE690400C7560400444404005CAD
:102E40003204000821040041100400000004003F87
:102E5000F00300F8E0030026D20300C3C30300CC54
:102E6000B503003AA803000A9B0300388E0300C094
:102E70008103009F750300D0690300505E03001DAD
:102E800053030034480300913D030033330300161D
:102E9000290300381F030097150300300C030003BB
:102EA0000303000BFA020049F10200BAE802005CD9
:102EB000E002002DD802002DD0020059C80200B057
:102EC000C0020031B90200DAB10200AAAA0200A0D1
:102ED000A30200BC9C0200FA9502005C8F0200DF96
:102EE00088020082820200457C02002776020027C9
:102EF000700200436A02007C640200D05E02003F60
:102F0000590200C8530200FFFDFCFAF8F6F4F2F093
:102F1000EEECEAE9E7E5E3E1E0DEDCDAD9D7D5D4A7
:102F2000D2D0CFCDCBCAC8C7C5C3C2C0BFBDBCBA43
:102F3000B9B7B6B4B3B2B0AFADACAAA9A8A6A5A4B0
:102F4000A2A1A09E9D9C9A99989795949392908FF8
:102F50008E8D8B8A8988878684838281807F7E7D1F
:102F60007B7A797877767574737271706F6E6D6C29
:102F70006B6A696867666564636261605F5E5D5C19
:102F80005B5A5958585756555453525150504F4EFA
:102F90004D4C4B4A4A4948474646454443424241C4
:102FA000403F3E3E3D3C3B3B3A393838373635357D
:102FB000343332323130302F2E2E2D2C2B2B2A2928
:102FC0002928272726252524232322212120201FC5
:102FD0001E1E1D1C1C1B1B1A191918181716161556
:102FE0001514131312121111100F0F0E0E0D0D0CDC
:102FF0000C0B0A0A09090808070706060505040458
:103000000303020201000000809D4300009B430077
:1030100000C8430000000000000000000000005352
:10302000657474696E67732053746F7265640045CC
:103030004550524F4D20496E697469616C697A65DB
:10304000640A003B20003A0A0020204D363033202D
:103050000020440020204D34313220530046696C5A
:10306000616D656E742072756E6F75742073656E18
:10307000736F723A002055004C0046696C616D65B3
:103080006E74206C6F61642F756E6C6F6164206C60
:10309000656E677468733A0020204D3835312058CA
:1030A000005A2D50726F6265204F6666736574001A
:1030B00020204D343133205300506F7765722D4CF2
:1030C0006F7373205265636F766572793A0020449E
:1030D0000020490020204D3330342050002044008F
:1030E00020490020204D33303120500050494420E9
:1030F00073657474696E67733A0020460020480057
:1031000020204D3134352053004D61746572696162
:103110006C2068656174757020706172616D657492
:103120006572733A00204A00202047323920572028
:10313000490020204D3432302053004175746F20F7
:10314000426564204C6576656C696E673A002020A4
:103150004D323036205800486F6D65206F666673BB
:1031600065743A0020580020530020204D3230353D
:10317000204200416476616E6365643A20423C6D92
:10318000696E5F7365676D656E745F74696D655FA9
:1031900075733E20533C6D696E5F66656564726150
:1031A00074653E20543C6D696E5F74726176656C27
:1031B0005F66656564726174653E20583C6D617838
:1031C0005F785F6A65726B3E20593C6D61785F790C
:1031D0005F6A65726B3E205A3C6D61785F7A5F6A08
:1031E00065726B3E20453C6D61785F655F6A657214
:1031F0006B3E0020540020520020204D32303420FD
:103200005000416363656C65726174696F6E20285C
:10321000756E6974732F7332293A20503C7072694D
:103220006E745F616363656C3E20523C72657472BC
:103230006163745F616363656C3E20543C747261CA
:1032400076656C5F616363656C3E0020204D3230B3
:10325000312058004D6178696D756D20416363655B
:103260006C65726174696F6E2028756E6974732F56
:103270007332293A0020204D3230332058004D61FE
:1032800078696D756D20666565647261746573201B
:1032900028756E6974732F73293A005374657073BF
:1032A0002070657220756E69743A002044002020F9
:1032B0004D3230302053002044697361626C656484
:1032C0000A0046696C616D656E742073657474697B
:1032D0006E67733A0020204D3134392043203B2063
:1032E000556E69747320696E2043656C73697573DC
:1032F0000A0020286D6D290020204732312020202F
:10330000203B20556E69747320696E206D6D00003E
:1033100000FA430000FA43000020410000964200FA
:1033200000A0420000A0420000C8430000BA42DCF6
:10333000050000DC050000640000004B00000024D4
:10334000F4D43050C38E20C2A24017828B70111269
:103350007A910D816CD90AA861E108C758660761A6
:103360005143061E4B5D05C145A7041A41110409CE
:103370003D9803713931034036DB0265339102D445
:10338000305402802E1D02632CEE01752AC501B057
:1033900028A001102781018F2564012B244B01E017
:1033A000223401AC211F018D200D01801FFC0084FF
:1033B0001EED00971DDF00B81CD200E61BC60020E2
:1033C0001BBC00641AB200B219A8000A19A0006A56
:1033D000189900D117910040178B00B51684003161
:1033E000167E00B31579003A157300C7146F0058A4
:1033F000146A00EE1366008813630025135E00C78D
:10340000125B006C12570015125400C1115100706C
:10341000114F0021114B00D61049008D1047004676
:1034200010440002104200C00F4000800F3E0042D6
:103430000F3C00060F3B00CB0E3800930E37005CAC
:103440000E3500270E3400F30D3200C10D3100900F
:103450000D3000600D2E00320D2D00050D2C00D911
:103460000C2B00AE0C2900850C29005C0C270035C4
:103470000C27000E0C2600E80B2400C40B2400A02F
:103480000B23007D0B23005A0B2100390B21001860
:103490000B2000F80A1F00D90A1E00BB0A1E009D5F
:1034A0000A1D00800A1D00630A1C00470A1B002C2D
:1034B0000A1B00110A1A00F7091A00DD091900C4D5
:1034C000091900AB091900920917007B091800635C
:1034D0000917004C09160036091600200916000AC3
:1034E000091500F5081500E0081400CC081400B810
:1034F000081400A4081400900813007D0812006B43
:10350000081300580812004608120034081100235E
:103510000811001208110001081100F0071000E066
:10352000071000D0071000C0071000B0070F00A15F
:1035300007100091070E0083070F0074070F006546
:10354000070E0057070E0049070E003B070D002E1F
:10355000070E0020070D0013070D0006070D00F9E8
:10356000060C00ED060D00E0060C00D4060C00C8A9
:10357000060C00BC060C00B0060C00A4060B00995B
:10358000060C008D060B0082060B0077060B006C04
:10359000060B0061060A0057060B004C060A0042A3
:1035A000060A0038060A002E060A0024060A001A37
:1035B000060A001006090007060A00FD050900F4C6
:1035C000050900EB050900E2050900D9050900D04D
:1035D000050900C7050900BE050900B5050800ADCD
:1035E000050800A50509009C050800940508008C45
:1035F000050800840508007C050800740508006CB7
:10360000050700650508005D050700560508004E22
:103610000507004705070040050800380507003189
:103620000507002A050700230507001C05060016EC
:103630000507000F0507000805060002050700FB47
:10364000040600F5040700EE040600E8040600E2A4
:10365000040700DB040600D5040600CF040600C9F9
:10366000040600C3040600BD040600B7040600B14A
:10367000040500AC040600A6040600A00405009B97
:1036800004060095040500900406008A04050085E0
:10369000040500800406007A040500750405007026
:1036A0000405006B04050066040500610405005C68
:1036B00004050057040500520405004D04050048A8
:1036C000040500430405003E0404003A04050035E7
:1036D000040500300404002C040500270404002322
:1036E0000405001E0404001A040400160405001159
:1036F0000404000D0404000904050004040400008F
:10370000040400FC030400F8030400F4030400F0C4
:10371000030400EC030400E8030400E4030400E0F5
:10372000030400DC030400D8030400D4030400D025
:10373000030400CC030400C8030300C503030024F2
:10374000F404D9201BC40C5C0E9804C4095F026504
:10375000077101F405F900FB04B30048048700C1B8
:103760000369005803550003034500BE023A008474
:1037700002310053022A002902250004022000E43D
:10378000011C00C8011900AF011700980114008442
:10379000011300710110006101100051010E00437E
:1037A000010D0036010B002B010B0020010B001551
:1037B0000109000C01090003010800FB000800F3E7
:1037C000000800EB000700E4000600DE000600D859
:1037D000000600D2000600CC000500C7000500C2AC
:1037E000000500BD000400B9000400B5000400B1EC
:1037F000000400AD000400A9000400A5000300A21D
:103800000003009F0004009B000300980003009544
:1038100000020093000300900003008D0002008B63
:10382000000300880002008600020084000300817B
:103830000002007F0002007D0002007B0002007990
:10384000000200770001007600020074000200729E
:10385000000100710002006F0002006D0001006CA9
:103860000002006A000100690002006700010066B2
:1038700000010065000100640002006200010061B7
:10388000000100600001005F0002005D0001005CBB
:103890000001005B0001005A0001005900010058BE
:1038A00000010057000100560001005500010054BE
:1038B00000010053000000530001005200010051BC
:1038C000000100500001004F0001004E0000004EBA
:1038D0000001004D0001004C0001004B0000004BB6
:1038E0000001004A000100490001004800000048B2
:1038F00000010047000100460000004600010045AD
:1039000000000045000100440001004300000043A6
:10391000000100420000004200010041000000419F
:10392000000100400001003F0000003F0001003E98
:103930000000003E0001003D0000003D0001003C91
:103940000000003C0000003C0001003B0000003B88
:103950000001003A0000003A00010039000000397F
:103960000001003800000038000000380001003776
:10397000000000370001003600000036000000366D
:103980000001003500000035000000350001003462
:103990000000003400000034000100330000003358
:1039A000000000330001003200000032000000324D
:1039B0000001003100000031000000310001003042
:1039C00000000030000000300001002F0000002F38
:1039D0000000002F0000002F0001002E0000002E2C
:1039E0000000002E0001002D0000002D0000002D21
:1039F0000000002D0001002C0000002C0000002C15
:103A00000000002C0001002B0000002B0000002B08
:103A10000000002B0001002A0000002A0000002AFC
:103A20000000002A000100290000002900000029F0
:103A300000000029000000290001002800000028E3
:103A400000000028000000280000002800010027D6
:103A500000000027000000270000002700000027CA
:103A600000010026000000260000002600000026BD
:103A700000000026000100250000002500000025B0
:103A800000000025000000250000002500010024A2
:103A90000000002400000024000000240000002496
:103AA0000001002300000023000000230000002389
:103AB000000000230000002300000023000100227A
:103AC000000000220000002200000022000000226E
:103AD0000000002200010021000000210000002160
:103AE0000000002100000021000000210000002152
:103AF0000001002000000020000000200000002045
:103B00000000002000000020000000200000002035
:103B10000001001F0000001F0000001F0000001F28
:103B20000000001F0000001F0000001F0001001E19
:103B30000000001E0000001E0000001E00000039F2
:103B40003000003325000087190000B00F0000DBB3
:103B5000080000BD040000740200003F01000020C6
:103B6000436F756E7420583A004265640045310019
:103B7000626564002C2073797374656D2073746FB3
:103B80007070656421204865617465725F49443ACC
:103B9000200048656174696E67204661696C6564E0
:103BA0000048656174696E67206661696C656400D0
:103BB0004D3131322053687574646F776E00100098
:103BC000C90210012C014001220170011801B0014D
:103BD0000E01F00104015002FA00B002F0003003BF
:103BE000E600D003DC009004D2007005C800A006F7
:103BF000BE000008B400B009AA00D00BA000600EFF
:103C0000960060118C000015820020197800C01DFC
:103C10006E00A0226400B0275A00902C50000031A2
:103C20004600E0343C0010383200903A2800603CF6
:103C30001E00A03D1400803E0A00203F00005448B2
:103C400045524D414C2052554E4157415900546800
:103C500065726D616C2052756E6177617900457295
:103C6000723A204D415854454D50004D41585445ED
:103C70004D502074726967676572656400457272A1
:103C80003A204D494E54454D50004D494E54454DF6
:103C9000502074726967676572656400202F002088
:103CA00042403A0020403A0020573A0020573A005C
:103CB000496E76616C6964206578747275646572AA
:103CC0000A007C3C3E5E2B3D3F2F5B5D3B2C2A2255
:103CD0005C0043616E6E6F74206F70656E2073754B
:103CE000626469722000534420496E697420466101
:103CF000696C0053442063617264206F6B0A006F2B
:103D000070656E526F6F74206661696C65640A003D
:103D1000766F6C756D652E696E6974206661696C6D
:103D200065640A004E6F20534420636172640A0088
:103D30000A4D3234004D3233202573004142530086
:103D4000504C41002E0A006F70656E206661696CF0
:103D500065642C2046696C653A200046696C6520D4
:103D600073656C65637465640A002053697A653A0B
:103D7000200046696C65206F70656E65643A2000AE
:103D8000454E4420535542524F5554494E450A0022
:103D90002220706F73002220706172656E743A2267
:103DA00000535542524F5554494E452043414C4CC7
:103DB000207461726765743A220053756263616CA6
:103DC0006C204F766572666C6F7700457863656529
:103DD000646564206D617820535542524F555449B3
:103DE0004E452064657074683A002E0A0044656C84
:103DF0006574696F6E206661696C65642C20466924
:103E00006C653A200046696C652064656C65746574
:103E1000643A005344207072696E74696E67206260
:103E200079746520004E6F74205344207072696E5F
:103E300074696E670A002F6175746F25632E6700C1
:103E400057726974696E6720746F2066696C653A91
:103E50002000667265736800646F696E6700206693
:103E6000696C653A20004E6F77200002FD5555556C
:103E700055555FFFFFFFFFFFFFFFFFFFFE00000044
:103E800000003FFFFFFFFFFFFFFFFFFFFD000007F8
:103E9000FFFFFFFFFFFFFFFFFFFFFFFFFE07C00564
:103EA00055555555555FFFFFFFFFFFFFFC0A2006E4
:103EB00000000000003FFFFFFFFFFFFFFE141005A2
:103EC000000007FFFFFFFFFFFFFFFFFFFC280806C2
:103ED00007C00555555555555FFFFFFFFE540404B7
:103EE0000A200600000000003FFFFFFFFC60040600
:103EF000141005000007FFFFFFFFFFFFFE50040442
:103F000028080607C00555555555555FFC60040641
:103F10005404040A200600000000003FFE54041C64
:103F200060040614100500000000001FFC28082E85
:103F300050040428080607C00001F03FFE14105486
:103F40006004065404040A200002081FFC0A2066CC
:103F500054041C60040614100005043FFE07C054FE
:103F600028082E5004042808000A021FFC00002E16
:103F700014105460040654040015013FFE00001C98
:103F80000A206654041C60040018011FFC0000068F
:103F900007C05428082E50040014013FFE000004FE
:103FA00000002E14105460040018011FFCFFFFFED7
:103FB00000001C0A206654041C15013FFED5555410
:103FC00000000607C05428082A0A021FFC84104675
:103FD00000000400002E14105105043FFEC41044DC
:103FE000FFFFFE00001C0A206102881FFC841046AF
:103FF000D5555400000607C05101F03FFE8410441F
:1040000084104600000400002A00001FFCC4104673
:10401000C41044FFFFFE00001C00003FFE8410445B
:10402000841046D5555400000000001FFCD555569D
:1040300084104484104600000000003FFCFFFFFC99
:10404000C41046C41044FFFFFFFFFF9FFE000006A0
:10405000841044841046D555555555BFFD555554CB
:10406000D5555684104484104104109FFFFFFFFC77
:10407000FFFFFCC41046C410410411BFFFFFFFFE48
:1040800000000684104484104104109FFFFFFFFDD0
:10409000555554D5555684104104109FFFFFFFFF1E
:1040A000FFFFFCFFFFFCC410410411BFFFFFFFFF37
:1040B000FFFFFE00000684104104109FFFFFFFFF7A
:1040C000FFFFFD555554D555555555BFFFFFFFFF13
:1040D000FFFFFFFFFFFCFFFFFFFFFF9FFFFFFFFF53
:1040E000FFFFFFFFFFFE00000000003FFFFFFFFF9C
:1040F000FFFFFFFFFFFD55555555555FFFFFFFFFC4
:10410000FFFFFFFFFFFFFFFFFFFFFFFFFFFFFFFFBF
:10411000FFFFFFFFFFFFFFFFFFFFFFFFFFFFFFFFAF
:10412000FFFFFFFFFFFFFFFFFFFFFFFFFFFFFFFF9F
:10413000FFFFFFFFFFFFFFFFFFFFFFFFE02EFB7D05
:10414000FBFBCFC1DFBB3EC0E1FE3C1FFDEE7B3978
:10415000F9F3CF9EDFBB3EDFDEFCDDE7FDEE3BBBD0
:10416000F9EBD7BF5FBB5EDFDEFDEDF7FDEEBBD346
:10417000FAEBB73FDFBB4EDFDFFFCDF3FDEEDBC772
:10418000FAEBBB7FC03B6EC0E3FF1DF3FDEECBEF50
:10419000FADBBB7FDFBB66DFF8FFCDF3FDEEEBEFB5
:1041A000FB5B033F5FBB76DFFE7FEDF3FDEEF3EFDE
:1041B000FB5B79BEDFBB7ADFDE7DEDF7FDEEF3EF73
:1041C000FBBAFD9EDFBB7CDFDEFDCDE7FDEEFBEF46
:1041D000FBBAFDC1DFBB7EC0E0FE1C1F6D61726CCF
:1041E000696E66772E6F726700322E302E375F440D
:1041F00057372E33001FFFFFFFFFFFFF6000000057
:104200000001FF400000000000FF800000000000EF
:104210007F83CF00000C303F87FF80000C301F866B
:104220007980000C000F8C30C7838C30E78C30CF46
:10423000C7CC31F38C30DCECEC33B98C30D86C6CFF
:1042400033198C30D06C0C33198C30D86C0C33197A
:104250008C30DC6C0E3B198C30CF7C079F198C3076
:10426000C77C038F194000000000000260000000BE
:104270000000061FFFFFFFFFFFF870012C019001F7
:104280002701B0012201C0011D01F0011801100237
:10429000130130020E016002090190020401C00204
:1042A000FF000003FA004003F5008003F000D00394
:1042B000EB002004E6007004E100E004DC004005AF
:1042C000D700C005D2004006CD00D006C800800748
:1042D000C3003008BE00F008B900C009B400B00A3D
:1042E000AF00B00BAA00D00CA500000EA000500F2C
:1042F0009B00C01096005012910000148C00C01555
:104300008700B0178200B0197D00D01B7800001E16
:10431000730040206E0090226900F0246400402762
:104320005F0090295A00E02B5500102E50002030DD
:104330004B0010324600E033410090353C0010370E
:10434000370070383200A0392D00B03A2800A03B69
:104350002300603C1E00103D1900903D1400103EEB
:104360000F00703E0A00C03E0500003F0000403FC5
:10437000FBFF803FF6FFC03FF1FF2020506C616ED5
:104380006E657242756666657242797465733A202D
:10439000002046726565204D656D6F72793A200088
:1043A000436F6D70696C65643A20417072203234DD
:1043B00020323032310A00204C6173742055706411
:1043C000617465643A20323032312D30342D313809
:1043D000207C20417574686F723A2054696E794D63
:1043E000616368696E657333440A00322E302E377C
:1043F0005F4457372E330A004D61726C696E00209E
:10440000536F6674776172652052657365740A0034
:10441000205761746368646F672052657365740A1E
:10442000002042726F776E206F757420526573653D
:10443000740A002045787465726E616C2052657351
:1044400065740A00506F77657255700A0073746165
:1044500072740A004732385859004D3130303100FB
:104460006572726F722077726974696E6720746FFB
:104470002066696C650A00446F6E65207361766919
:104480006E672066696C652E0A004D323900456EF4
:104490006473746F70730025532025632025632097
:1044A000256320256300205A3A0020593A002058FD
:1044B0003A00656E6473746F7073206869743A2093
:1044C0000000000A0B02090C0D0E0807030401008E
:1044D00000000000000000000000000000000000DC
:1044E0000000000000000000000000000012111099
:1044F00000000000000000000000000000000000BC
:1045000000000000000000004D6F76652025736DEF
:104510006D004D6F766520302E316D6D004D6F76DC
:104520006520316D6D004D6F76652031306D6D0009
:104530004D6F7665204178697300457874727564B3
:104540006572004D6F7665205A004D6F7665205973
:10455000004D6F7665205800403D3C3D4368616EDC
:1045600067652046696C616D656E7400556E6C6F91
:1045700061642046696C616D656E74004C6F6164A6
:104580002046696C616D656E740050726568656186
:104590007420437573746F6D005072656865617443
:1045A0002024004261636B0050726F62696E672065
:1045B0004661696C656400205A3A200020593A200F
:1045C0000042656420583A200073686F7700627576
:1045D00074746F6E00626567696E0044697361622E
:1045E0006C6552756E6F75740050757267654D6FAE
:1045F00072650050617573656400436F6E74696E17
:104600007565004C6F61642046696C616D656E7400
:10461000205400496E736572742066696C616D6523
:104620006E7420616E642073656E64204D31303885
:104630000A00220A00556E6B6E6F776E20636F6DF5
:104640006D616E643A2022002042002050006F6BA2
:1046500000544D334420435231305632205265616C
:1046600064792E005072696E74696E672E2E2E006A
:104670005072696E74205061757365640020450046
:10468000205A00205900204D393220580020453A48
:1046900000205A3A0020593A00583A0020746F6FAF
:1046A000206C6F6E6720657874727573696F6E2009
:1046B00070726576656E7465640A0020636F6C6461
:1046C00020657874727573696F6E20707265766597
:1046D0006E7465640A00526573656E643A20006EFC
:1046E0006F74696669636174696F6E2000000022EF
:1046F00000250028002B002E0031003400020100AC
:1047000000050108010B0100002100240027002AF8
:10471000002D003000330001010000040107010AF0
:104720000105050505070508080808020202020A36
:104730000A08080404040401010101010101010344
:1047400003030303030303040707070C0C0C0C0CFF
:104750000C0C0C0202020206060606060606060BF2
:104760000B0B0B0B0B0B0B01021020200808102069
:1047700040102040800201020108040201010204ED
:1047800008102040808040201008040201800402AC
:104790000180402010080402010804020101020403
:1047A00008102040800102040810204080006002B0
:1047B0002C0211241FBECFEFD1E2DEBFCDBF00E03F
:1047C0000CBF13E0A0E0B2E0E6E7FAEE02E00BBFB8
:1047D00002C007900D92A839B107D9F728E1A8E9DE
:1047E000B3E001C01D92AE3AB207E1F713E2C8EDA3
:1047F000D3E200E006C021970109802FFE010F944B
:104800009171C73DD10780E00807A9F70F94BF5FFA
:104810000D9429750C940000FC0184910895FC010D
:10482000808108951198000000009091020187FD99
:104830009095917090930001119A00000000000083
:1048400000001198000000009091020186FD9095F3
:10485000917090930001119A000000000000000088
:104860001198000000009091020185FD90959170D3
:1048700090930001119A00000000000000001198C0
:10488000000000009091020184FD9095917090933A
:104890000001119A000000000000000011980000C3
:1048A00000009091020183FD90959170909300011A
:1048B000119A0000000000000000119800000000A4
:1048C0009091020182FD9095917090930001119A50
:1048D000000000000000000011980000000090910E
:1048E000020181FD9095917090930001119A000052
:1048F00000000000000011980000000080910201FB
:10490000817080930001119A0000000000000000F7
:10491000089590E080E00895CF93DF93DB01F901E3
:104920009C919130C1F0943080F094509C938830E9
:10493000D1F480819181009771F0019791838083F8
:10494000480F591FEA01188206C08C3539F49C5F64
:104950009C93943041F4DF91CF9108958B3339F7D4
:1049600081E08C93F8CF20813181B9016F5F7F4F57
:1049700071836083420F531FEA0188838081918194
:104980008F3591056CF7E7CF0F931F9381E000916E
:104990009F161091A0162091A1163091A216409159
:1049A0009B1650919C1660919D1670919E1604174F
:1049B00015072607370708F480E01F910F91089527
:1049C00090E080E00895282F9091DA08833021F458
:1049D00095FD0FC094FD0FC0892F90E0B0E0A0E0DE
:1049E00004C0B695A795979587952A95D2F78170BB
:1049F000089581E0089580E00895CF92DF92EF92CC
:104A0000FF92CF93DF93EC01CC80DD80EE80FF80BE
:104A100027E137EB41ED58EBC701B6010F94FA736C
:104A200087FD23C023E030E04BE953E4C701B60122
:104A30000F94A86A1816CCF0C880D980EA80FB8051
:104A400027E137EB41ED58EBC701B6010F94FA733C
:104A500087FD0BC0C1E023E030E84DE953E4C70116
:104A6000B6010F94A86A18160CF4C0E08C2FDF91E1
:104A7000CF91FF90EF90DF90CF9008952F923F92CB
:104A80004F925F926F927F928F929F92AF92BF925E
:104A9000CF92DF92EF92FF920F931F93CF93DF930A
:104AA000CDB7DEB72E970FB6F894DEBF0FBECDBFE1
:104AB000E82ED62E042F122F282F30E03C872B878C
:104AC000462F50E05A87498765E0F62EF29EC001D6
:104AD000F39E900D11249E878D87FA01E80FF91F30
:104AE000EE0FFF1FEE0FFF1FE65EF94F6081718131
:104AF000828193819B01AC010F948C74882309F40B
:104B000034C1E00E612F6D0DFE9CF0011124A985CA
:104B1000BA85AE0FBF1FAA0FBB1FAA0FBB1FA65E91
:104B2000B94FAC901196BC9011971296CC901297F9
:104B30001396DC90E00EFE9CA0011124A985BA8595
:104B4000A40FB51FAA0FBB1FAA0FBB1FA65EB94FAC
:104B5000EC901196FC90119712960C911297139667
:104B60009C90862F90E0AD85BE85A80FB91FAA0F37
:104B7000BB1FAA0FBB1FA65EB94F8C9011967C90ED
:104B8000119712966C90129713965C90610F70E0DB
:104B9000AD85BE85A60FB71FAA0FBB1FAA0FBB1FEF
:104BA000A65EB94F4C9011963C90119712961C91AD
:104BB000129713962C90E80FF91FEE0FFF1FEE0FC0
:104BC000FF1FE65EF94FB081B98321812A833281CC
:104BD0003B8383818C83FA01E60FF71FEE0FFF1FE3
:104BE000EE0FFF1FE65EF94F90819D83A181AE839A
:104BF000B281BF83238128879701402F592DB701A8
:104C0000802F992D0F948C74882321F0E12CF12CA6
:104C100000E0912C9501A601B501C6010F948C749A
:104C2000882319F05701C02ED92C242D332D412F64
:104C3000522D642D732D812F922D0F948C74882307
:104C400021F0412C312C10E0212C282D372D462D20
:104C5000552D682D772D862D952D0F948C748823D6
:104C600021F0842C732C612E522C2D813E814F819A
:104C700058856D817E818F8198850F948C748823EF
:104C800021F01D821E821F82188629813A814B8164
:104C90005C8169817A818B819C810F948C748823DB
:104CA00041F03D8139834E814A835F815B838885F2
:104CB0008C8385E0EB85FC858E9FD0018F9FB00DA6
:104CC000112429853A85A20FB31FAA0FBB1FAA0F73
:104CD000BB1FA65EB94FBA87A9879501A601B5018A
:104CE000C6010F949A719701402F592D0F94997115
:104CF0006B017C01282D372D462D552D682D772DE4
:104D0000862D952D0F949A71242D332D412F522DE0
:104D10000F9499719B01AC01C701B6010F949A7170
:104D20006B017C0129813A814B815C8169817A81A7
:104D30008B819C810F949A712D813E814F81588582
:104D40000F9499719B01AC01C701B6010F949A7140
:104D500020E030E040E450E40F949472A985BA85D5
:104D60006D937D938D939C9313972E960FB6F89425
:104D7000DEBF0FBECDBFDF91CF911F910F91FF908E
:104D8000EF90DF90CF90BF90AF909F908F907F90EB
:104D90006F905F904F903F902F9008951092BD08B4
:104DA0008091590290915A02A0915B02B0915C02ED
:104DB0008093930690939406A0939506B0939606DD
:104DC0000895129A0895269A2E9A0895AF92BF9246
:104DD000CF92DF92EF92FF920F931F93CF93DF93C7
:104DE0006B01E9014A3009F4C1C0453109F073C0D3
:104DF000DB011296ED91FC91F280C681D781809102
:104E00000201809582708093000188E28A950000FB
:104E1000E9F7BF2CB29420EFB22230E1A32EAF0C01
:104E200048E2E42E88EF0E9412248E2D8A9500001D
:104E3000E9F7BFE1BF1508F485C08F2D8077806842
:104E40000E9412248B2D0E9412248E2D8A95000020
:104E5000E9F780E80E94122480E00E9412248E2D3F
:104E60008A950000E9F78AEF0E9412248E2D8A9518
:104E70000000E9F78E01005F1F4F8881807F0E944C
:104E8000122489918295807F0E941224C017D10735
:104E9000A1F78E2D8A950000E9F7F394E0E1BE0EAC
:104EA000FA10C0CF80910201827080930001D60178
:104EB0001296CD91DC91CE010F948C54811147C292
:104EC000DF91CF911F910F91FF90EF90DF90CF90E6
:104ED000BF90AF900895FB0102811381423309F422
:104EE000F1C108F4F5C1463409F4E2C1473409F4CC
:104EF000E5C14B3329F589812B81D80112966C913C
:104F0000129713964C91213009F438C2233009F0DE
:104F100002C238EF380F582F91E0431708F490E0A1
:104F200041E0531708F040E031E0561708F430E054
:104F3000592F542B352309F016C2942309F013C2BC
:104F400081E0BECF80EE8F0D8068807F0E941224AA
:104F50008F2D8295807F0E9412248E2D8A950000CD
:104F6000E9F780E80E94122480E877CF8091010160
:104F70008260809301018091020182708093000120
:104F80008091010181608093010180910201817013
:104F900080930001099A119A809102018095827094
:104FA0008093000188E28A950000E9F788E790E0A5
:104FB000CEE9DFE0FE013197F1F70197D9F788EFED
:104FC0000E94122418E2812F8A950000E9F780E2FE
:104FD0000E94122480E00E941224812F8A950000F2
:104FE000E9F780E00E94122480E80E941224812FB9
:104FF0008A950000E9F780E00E94122480E10E9477
:105000001224812F8A950000E9F7CE010197F1F76C
:10501000CE010197F1F7CE010197F1F7CE0101978B
:10502000F1F7CE010197F1F7CE010197F1F7CE012B
:105030000197F1F7CE010197F1F7CE010197F1F752
:10504000CE010197F1F7CE010197F1F7CE0101975B
:10505000F1F7CE010197F1F7CE010197F1F7219712
:10506000F1F780E20E94122480E40E941224812F32
:105070008A950000E9F780E20E94122480E60E94EF
:1050800012241A950000E9F710E0D0E0C8E28D2F55
:10509000807780680E941224812F0E9412248C2F16
:1050A0008A950000E9F780E80E94122480E00E94BF
:1050B00012248C2F8A950000E9F78AEF0E941224AF
:1050C0008C2F8A950000E9F790E21198000000000B
:1050D00080910201817080930001119A000000000C
:1050E0000000000011980000000080910201817012
:1050F00080930001119A0000000000000000119848
:105100000000000080910201817080930001119ADB
:1051100000000000000000001198000000008091D5
:105120000201817080930001119A000000000000CC
:1051300000001198000000008091020181708093AE
:105140000001119A0000000000000000119800000A
:10515000000080910201817080930001119A00008B
:105160000000000000001198000000008091020182
:10517000817080930001119A00000000000000007F
:10518000119800000000809102018170809300015D
:10519000119A0000000000000000119800000000BB
:1051A00080910201817080930001119A000000003B
:1051B0000000000011980000000080910201817041
:1051C00080930001119A0000000000000000119877
:1051D0000000000080910201817080930001119A0B
:1051E0000000000000000000119800000000809105
:1051F0000201817080930001119A000000000000FC
:1052000000001198000000008091020181708093DD
:105210000001119A00000000000000001198000039
:10522000000080910201817080930001119A0000BA
:1052300000000000000011980000000080910201B1
:10524000817080930001119A0000000000000000AE
:10525000119800000000809102018170809300018C
:10526000119A00000000000000008C2F8A950000B9
:10527000E9F7915009F029CF88EF0E9412248C2F72
:105280008A950000E9F7DF5F105FD03209F0FFCEAA
:1052900080E00E94122480EC0E941224CA95000033
:1052A000E9F78091020182708093000181E008CECD
:1052B000D80115968C91888381E002CEF801818116
:1052C0008883FACFB901C8010F94A95481E0F8CDC1
:1052D000443171F0473109F033CE1882F8018281F0
:1052E0008983858181508A8383818B8381E0E8CDA6
:1052F000D80115964C91159750E0440F551F70E05A
:1053000060E016968D919C910F94CA74C8010F9419
:10531000A25481E0D5CD481708F412CE861708F4C0
:105320000FCEFA80E12CD12C243070F41DC0BE01C8
:10533000C8010F94A954898198819D0D98838E0D81
:105340008983FF0C09F4FCCDF7FEF6CFF0CF4D8139
:1053500050E0440F551F70E060E08E819F810F94F4
:10536000CA7481E0ADCDFA8030E0F901E554FD4F1B
:10537000D08029543D4FF901E080E6CF58E0580F26
:10538000382FCACDEF92FF920F931F93CF93DF93E5
:10539000EC018B017A018A859B858617970731F08E
:1053A000888199810F9482561B870A87B70188816B
:1053B00099810F94D6472E813F81820F932F911DA3
:1053C0009F838E8390E080E0DF91CF911F910F91BA
:1053D000FF90EF9008959F92AF92BF92CF92DF928D
:1053E000EF92FF920F931F93CF93DF93EC018B010A
:1053F000942EA52E8A859B858617970731F0888184
:1054000099810F9482561B870A8788859985019612
:1054100049F5BC800A818E81080FC880D980D601E9
:105420005596ED91FC91C6011995B80EE92CFA2C10
:1054300010E0F70121917F01211127C08E819F810A
:10544000810F911D9F838E8390E080E0DF91CF914B
:105450001F910F91FF90EF90DF90CF90BF90AF9092
:105460009F9008950E811F81692D7A2D88819981E1
:105470000F94D647800F912F911D288539852817C5
:10548000390738F681E090E0E1CF4B2D602FC6015F
:105490000F94DA56080F180FCCCFDF92EF92FF92DD
:1054A0000F931F93CF93DF93EC01D62E1CAD0BAD62
:1054B0007C0184E0E80EF11CE98DFA8DC701199595
:1054C000412F480F2D2D602FC7010F94DA569BAD49
:1054D000890F8BAF81E090E0DF91CF911F910F9109
:1054E000FF90EF90DF900895AB01BC0140939F16B1
:1054F0005093A0166093A1167093A21688E098E1CD
:105500000C941FE680932F028032B8F590916005CD
:10551000891724F091E0980F9093600540915C0505
:1055200050915D0560915E0570915F05082E04C085
:1055300076956795579547950A94D2F741704093B1
:10554000231087FD1DC0282F082E000C330B3F931E
:105550008F938AE69AE09F938F938AE79AE09F93CE
:105560008F931F920E943CCB8DB79EB707960FB6C4
:10557000F8949EBF0FBE8DBF089510922310E1CF07
:105580000D94A0430F931F93CF93DF9300D01F92EE
:10559000CDB7DEB79C0104EA18E090E1E0EDF9E058
:1055A000D80101900D929A95E1F7F901208131819E
:1055B00042815381F80160857185828593850F94BE
:1055C0009A71F801608771878287938780E090E005
:1055D000A0EAB0E489839A83AB83BC83CE010196B1
:1055E0000F9456100F900F900F900F90DF91CF9166
:1055F0001F910F9108952F923F924F925F926F9259
:105600007F928F929F92AF92BF92CF92DF92EF9252
:10561000FF921F93CF93DF93CDB7DEB72C970FB6D2
:10562000F894DEBF0FBECDBF7A011901DC012D91C8
:105630003D914D915C912D833E834F835887FB01B3
:1056400040805180628073808090D0099090D10911
:10565000A090D209B090D309A50194016D817E81FB
:105660008F8198850F94A86A81110EC011E0A30163
:1056700092016091D4097091D5098091D6099091D9
:10568000D7090F94A86A811110E0D1012D913D91A5
:105690004D915C9129873A874B875C87F701C080E1
:1056A000D180E280F3802091130230911402409166
:1056B000150250911602C701B6010F94A86A8823FB
:1056C00009F44EC0C0921302D0921402E092150267
:1056D000F09216028091DC099091DD09A091DE091B
:1056E000B091DF094091D4095091D5096091D60954
:1056F0007091D7098092A4089092A508A092A6085C
:10570000B092A7084093A8085093A9086093AA08EC
:105710007093AB08C092AC08D092AD08E092AE088E
:10572000F092AF088093B0089093B108A093B208AC
:10573000B093B30820E030E040E05FE360915110A7
:105740007091521080915310909154100F940E6BE1
:1057500069837A838B839C83CE0101960F945610C4
:105760002D813E814F8158852093A4083093A50850
:105770004093A6085093A7084092A8085092A90801
:105780006092AA087092AB08D1012D913D914D9184
:105790005C916091B0087091B1088091B2089091CD
:1057A000B3080F949A716093B0087093B108809316
:1057B000B2089093B30811112FC020E030E0A90186
:1057C00069857A858B859C850F94A86A811133C081
:1057D00060E070E088EC92E469837A838B839C8339
:1057E000CE0101960F9456102C960FB6F894DEBF9A
:1057F0000FBECDBFDF91CF911F91FF90EF90DF9053
:10580000CF90BF90AF909F908F907F906F905F9060
:105810004F903F902F9008952AEF3EE74AE25FE3D2
:1058200060915510709156108091571090915810BA
:105830000F940E6BD1CF60E070E080EA91E4CCCFA2
:10584000CF93DF9300D01F92CDB7DEB780E090E01A
:10585000A0EAB0E489839A83AB83BC8361E0CE0184
:1058600001960F9459080F900F900F900F90DF91B1
:10587000CF91089580911E0590911F05009731F0FA
:105880004AE050E070E060E00D94C36860E070E0D2
:10589000CB0108958091E40982FF0BC063E686E5A1
:1058A0009BE00E9457CB0F94964E0E9457D281E006
:1058B000089580E0089580911E0590911F0500973E
:1058C00031F04AE050E070E060E00D94956760E0F0
:1058D00070E0CB0108950E945B2C97FD0CC00E94E4
:1058E0005B2C6F3F71058105910509F034F40E942E
:1058F0005B2C862F089580E008958FEF08958091A6
:105900001E0590911F05892B41F00E946B2C91E0A0
:10591000811101C090E0892F089591E0FCCFCF92D2
:10592000DF92EF92FF920F931F93CF93DF936B0160
:105930007A01EC01C655DB4F28813CE0389F80019D
:10594000399F100D112427FF24C0FB011182108202
:1059500088818F5F888388819801280F311D87FD9A
:105960003A95C90120911C16F6012817190629F04D
:1059700024F088818C300CF43CC0808191810496A5
:1059800080349C4908F475C0F601808191810496A9
:1059900072C088819801280F311D87FD3A95C90191
:1059A00020911C162817190699F294F28881A801F3
:1059B000480F511D87FD5A95FA01EE0FFF1FE40FA6
:1059C000F51FEC52FA4E808187FFC2CF8881F80123
:1059D000E80FF11D87FDFA95CF01EE0FFF1FE80FCD
:1059E000F91FEC52FA4E808160E08F770F94C84C1B
:1059F000AFCF808191812881A801420F511D27FDE1
:105A00005A959A01FA01EE0FFF1FE20FF31FEC52B5
:105A1000FA4E21813281820F931FF7019183808397
:105A200088819801280F311D87FD3A95F901EE0F05
:105A3000FF1FE20FF31FEC52FA4E808187FF20C058
:105A40008881080F111D87FD1A95F801EE0FFF1FC1
:105A5000E00FF11FEC52FA4E808161E08F77DF9109
:105A6000CF911F910F91FF90EF90DF90CF900D9409
:105A7000C84C80E49CE9F701918380838FEF888391
:105A8000DF91CF911F910F91FF90EF90DF90CF901A
:105A90000895AF92BF92CF92DF92EF92FF920F9351
:105AA0001F93CF93DF93EC015B018A01FB011995F2
:105AB00087FD16C0C82ED12CF12CE12C2196F801BF
:105AC000C082D182E282F382CE01DF91CF911F9119
:105AD0000F91FF90EF90DF90CF90BF90AF9008951F
:105AE000982F907E903CA9F48F7190E0B0E0A0E0F8
:105AF0006C017D0156E0CC0CDD1CEE1CFF1C5A95A0
:105B0000D1F7CE010196F50119958F73C82A229617
:105B1000D6CF982F907F903E11F58F7090E0B0E037
:105B2000A0E06C017D0136E0CC0CDD1CEE1CFF1CFE
:105B30003A95D1F7CE010196F50119958F73C82AD0
:105B400046E0CC0CDD1CEE1CFF1C4A95D1F7CE01C3
:105B50000296F50119958F73C82A2396B0CF982F16
:105B6000987F903F79F5877090E0B0E0A0E06C01FD
:105B70007D0186E0CC0CDD1CEE1CFF1C8A95D1F764
:105B8000CE010196F50119958F73C82A96E0CC0CC9
:105B9000DD1CEE1CFF1C9A95D1F7CE010296F50193
:105BA00019958F73C82A26E0CC0CDD1CEE1CFF1C57
:105BB0002A95D1F7CE010396F50119958F73C82A5E
:105BC00024967DCF982F907C903841F4807C80384B
:105BD00069F42196CE01F5011995F8CF8E7F8D3F9E
:105BE00028F02196CE01F5011995F8CFC12CD12CC2
:105BF000760165CF9CE0899F802D112491E0980F5C
:105C0000909361052CE0280F20939E0830E02E5FD2
:105C10003F4F409191164217130619F014F080E09F
:105C20000895209193169217D0F7662341F08E5F66
:105C30000F949C5580919E088E5F0F949C55809187
:105C40009E0890919116891750F320919316909188
:105C50006105291720F3109294168093951681E020
:105C60000895CF9380915405811154C010929416D9
:105C70001092951610929616109262161092611656
:105C800010926416109263161092661681E080934B
:105C9000651682E28093671610926C1610926B164E
:105CA000E0E8F6E12EE836E18FEF81932E173F070B
:105CB000E1F7C1E0C0937D1626EA31E03093731618
:105CC00020937216C0937416109275161092761661
:105CD00090E490937716109278162EE232E030938B
:105CE0008F1620938E1622E232E0309360162093B6
:105CF0005F1697E19093841691E19093851690E159
:105D00009093821680938116809380160F94C354CB
:105D1000C093540581E08093550588EB9AE19093F8
:105D20008615809385151092881510928715CF914E
:105D3000089520915305022E000C330B8217130691
:105D400041F08093530568EB7AE18DE596E10D947F
:105D500082560895CF92DF92EF92FF920F931F9396
:105D6000CF93DF93CDB7DEB72C970FB6F894DEBF95
:105D70000FBECDBF6F3F71058105910509F0D0F4CD
:105D800089E596E10E944D2AE0916116F091621634
:105D90003196849190E02C960FB6F894DEBF0FBE3A
:105DA000CDBFDF91CF911F910F91FF90EF90DF90CA
:105DB000CF900895F0909416E09095162091550597
:105DC00021110FC048E95AE16E2D8F2D0F944657CF
:105DD00090E080E0F80EF0929416E09295169927E4
:105DE000DACFC0906116D09062162DE536E13A8385
:105DF00029832F2D30E03C832B832E2D30E03E83F2
:105E00002D8318861F822FEF3FEF3A8729871C8644
:105E10001B860BEE19E29E012F5F3F4FAB01BC01C9
:105E2000C6010F945B30B6018DE596E10F94825662
:105E30008F819885CFCFCF93DF93FC0125AD2111C2
:105E400004C021E025AF0F94C354C0915F16D091D8
:105E50006016E0918E16F0918F1682E01995E09110
:105E60008E16F0918F1681E0199530E020E044E124
:105E7000BE018DE596E10F94BF5420E936E147E17C
:105E8000BE018DE596E10F94BF54E0918E16F0911E
:105E90008F1680E0DF91CF911994CF92DF92EF922D
:105EA000FF920F931F93CF93DF93CDB7DEB72C975D
:105EB0000FB6F894DEBF0FBECDBFF0909416E09001
:105EC00095162091550521111DC048E75AE16E2D08
:105ED0008F2D0F94465790E080E0F80EF0929416C4
:105EE000E092951699272C960FB6F894DEBF0FBE58
:105EF000CDBFDF91CF911F910F91FF90EF90DF9079
:105F0000CF900895C0906116D09062162DE536E1CD
:105F10003A8329832F2D30E03C832B832E2D30E0D4
:105F20003E832D8318861F827A8769871C861B868D
:105F30000BEE19E29E012F5F3F4F4CE054E2BC0193
:105F4000C6010F941F31B6018DE596E10F9482567C
:105F50008F819885C2CF6FEF7FEF0C944D2FCF923A
:105F6000DF92EF92FF920F931F93CF93DF93CDB702
:105F7000DEB72C970FB6F894DEBF0FBECDBFF09002
:105F80009416E09095162091550521111DC048E505
:105F90005AE16E2D8F2D0F94465790E080E0F80E59
:105FA000F0929416E092951699272C960FB6F894D5
:105FB000DEBF0FBECDBFDF91CF911F910F91FF903C
:105FC000EF90DF90CF900895C0906116D090621648
:105FD0002DE536E13A8329832F2D30E03C832B8356
:105FE0002E2D30E03E832D8318861F827A876987A5
:105FF0001C861B860BEE19E29E012F5F3F4F4FE080
:1060000054E2BC01C6010F941F31B6018DE596E143
:106010000F9482568F819885C2CFBF92CF92DF9224
:10602000EF92FF920F931F93CF93DF938B01F42E88
:10603000E90141FB662760F90E94FA2D882309F4E3
:106040005AC0B12C0115110521F0C8010E9428D3B6
:10605000B82EE12C209721F0CE010E9413D5E82E16
:1060600080E8C82ED12CF0FE1EC085E190E08B198F
:106070009109B7FC93958E199109E7FC939597FDCB
:10608000019695958795F82E30E8C32ED12CFA9479
:10609000F7FC09C060E270E080E090E00E94AA2E68
:1060A000C81AD90AF4CFBB2099F0C60166E070E0A7
:1060B0000F946971262F4091A0085091A10860911A
:1060C0009F08C8010E9468D296E0899F6001112450
:1060D000EE2031F0B601CE010E94AF2FC81AD90AC6
:1060E00087E0C816D10438F060E270E080E090E00C
:1060F0000E94AA2EF3CFDF91CF911F910F91FF90B5
:10610000EF90DF90CF90BF9008956FEF7FEF0C94EA
:10611000AF2FAF92BF92CF92DF92EF92FF920F9389
:106120001F93CF93DF935C016B010E9428D3E82E6D
:10613000C6010E9413D5F12C03E110E0081B1109E0
:10614000C5E20E151F050CF4CFE18C2F90E09C01E9
:106150002E5F3F4F409191164217130609F0CCF580
:10616000099720919316281719069CF14091A008D1
:106170005091A10860919F0810929416C0939516B3
:1061800025E1C5010E9468D2D1E0C114D104B1F06B
:106190006AE370E080E090E00E94AA2E0E151F05D1
:1061A000D4F4C45F80919116C81740F020919316E3
:1061B0004C2F4950550B241715067CF4DF91CF91D5
:1061C0001F910F91FF90EF90DF90CF90BF90AF9015
:1061D0000895D0E0DACFDD2389F3802F880F080FF0
:1061E000000F00939416C093951660E270E080E073
:1061F00090E00E94AA2EC601DF91CF911F910F91CE
:10620000FF90EF90DF90CF90BF90AF900C948530CF
:106210008F929F92AF92BF92CF92DF92EF92FF92B6
:106220000F931F93CF93DF93CDB7DEB72C970FB6A5
:10623000F894DEBF0FBECDBF982F862F5A0179018B
:10624000D02E692F0E94FA2D882309F489C0C70136
:10625000002391F10E9428D3C82E8090611690905F
:10626000621680915505811145C01FEF23E12C195D
:106270004091A0085091A10860919F08C5010E941B
:1062800068D2CC2009F46CC0B6E08B9F5001112479
:106290006AE370E080E090E00E94AA2E57E0A51625
:1062A000B10408F444C060E270E080E090E00E9435
:1062B000AA2EA81AB90AF2CF0E9413D5C82E809030
:1062C00061169090621680915505882371F2FE0147
:1062D00033968AE0DF011D928A95E9F78DE596E114
:1062E0009A83898302EC19E29E012F5F3F4F4FE0B2
:1062F00054E212C0FE0133968AE0DF011D928A95B6
:10630000E9F78DE596E19A83898302EC19E29E0113
:106310002F5F3F4F4CE054E2B701C4010F941F318F
:10632000B4018DE596E10F9482561F819FCF409175
:106330009E08212F30E0A6E0CA9EC00111242E5FE6
:106340003F4F281739070CF49C0180E8821B80938B
:10635000941640939516C701DD20A9F00E94AB2F3B
:106360002C960FB6F894DEBF0FBECDBFDF91CF9154
:106370001F910F91FF90EF90DF90CF90BF90AF9063
:106380009F908F9008950E948530EACFE9E5F6E16D
:1063900083AF64AFCA010C9485302F923F924F9225
:1063A0005F926F927F928F929F92AF92BF92CF92A5
:1063B000DF92EF92FF920F931F93CF93DF93D62F2D
:1063C000C72FFC0180809180A280B380C501B401F9
:1063D00020E831E541E050E00F94EC70C9016DE632
:1063E00071E00F9469716B017C01C501B40120E17A
:1063F0003EE040E050E00F94EC70CA01B90128E1A2
:1064000030E040E050E00F94EC70362E272E062F3F
:10641000172F8CE3482E512C612C712CC501B4012F
:10642000A30192010F94EC70B62EA72ECA01B901F8
:10643000A30192010F94EC70CB01C114D10479F146
:10644000AF92BF927F936F932F923F92FF92EF9202
:10645000DF92CF9286EB98E19F938F93CF93DF9358
:106460000F943F6A8DB79EB70E960FB6F8949EBFF5
:106470000FBE8DBF8D2F9C2FDF91CF911F910F915C
:10648000FF90EF90DF90CF90BF90AF909F908F9054
:106490007F906F905F904F903F902F900895E11400
:1064A000F104C9F0AF92BF927F936F932F923F9206
:1064B000FF92EF9286EA98E19F938F93CF93DF93B9
:1064C0000F943F6AEDB7FEB73C960FB6F894FEBF47
:1064D0000FBEEDBFCFCF012BB9F0AF92BF927F932C
:1064E0006F932F923F928AE998E19F938F93CF9376
:1064F000DF930F943F6A8DB79EB70A960FB6F89454
:106500009EBF0FBE8DBFB6CF892BA9F0AF92BF92B1
:106510007F936F9382E998E19F938F93CF93DF935B
:106520000F943F6AEDB7FEB738960FB6F894FEBFEA
:106530000FBEEDBF9FCFAF92BF928EE898E19F93C1
:106540008F93CF93DF930F943F6A0F900F900F902C
:106550000F900F900F908ECF8F929F92AF92BF921D
:10656000CF92DF92EF92FF920F931F93CF93DF931F
:1065700010925205109251052FE320934C05109272
:106580004B0510924A051092490510924D05109244
:106590004E0510924F05109250059C01F901908113
:1065A0002F5F3F4F9032D1F39E34C9F4818190ED3B
:1065B000980F9A3020F08D3211F08B3281F43296A0
:1065C0009F012F5F3F4F808180538A3008F47BC04A
:1065D0009F012F5F3F4F8081803209F476C0F09396
:1065E000C308E093C2088F010F5F1F4FC0816AE2AA
:1065F00070E0C8010F94EF74009731F0FC013197FF
:1066000080818032E1F31182CD3429F0C43519F054
:10661000C73409F04BC0F80180810F5F1F4F8032F3
:10662000D1F380538A3008F041C0C0934C0530E06C
:1066300020E04AE0DF011196429FC001439F900D88
:1066400011249C01205331098081280F311D87FDC1
:106650003A95818190ED980F9A30C8F130934B05AF
:1066600020934A058E3261F4329690E04AE0DF01D1
:1066700031968C9150ED580F5A3058F1909349054E
:10668000CD01DC0101964C914032D9F3CD3489F52E
:106690002E31310539F018F52731310519F02C313B
:1066A000310539F5B0935205A0935105DF91CF9193
:1066B0001F910F91FF90EF90DF90CF90BF90AF9020
:1066C0009F908F900895F9017BCFF90181CFFD0153
:1066D000B1CF949F800D112490ED980FC8CF25372E
:1066E000310538F027373105E8F2203A83E03807E2
:1066F000C9F2D091C20840E050E0BA0110E000E0D9
:10670000C12CD12C7601C394FD0131968C91882344
:1067100009F47FC08132E1F4CD34D1F42032310567
:10672000B9F440934D0550934E0560934F05709317
:106730005005F0935205E093510563E270E0CF01FC
:106740000F94EF74009709F4B1CFFC011082AECF23
:1067500081548A3108F058C0DF019D91903291F048
:10676000A0EDA90FAA30E8F09E3271F49181905308
:106770009A30B8F00115110519F48F010150110973
:1067800090E013C0FD01E8CF9D3211F09B3291F7EC
:106790009181A0EDA90FAA3020F09E3259F7928185
:1067A000E6CF9E2F9D1B309759F3A82FB0E04601EE
:1067B000570104C0880C991CAA1CBB1C8A95D2F7EF
:1067C000482959296A297B29A15DBA4F9C93808168
:1067D0008154DF018A3108F497CFDF01819188234A
:1067E00009F492CF90ED980F9A30B8F393ED980F8B
:1067F000923098F38B3289F3CD010196EC91E0321F
:1068000009F082CFDC01F8CF0115110501F78D01E8
:10681000DECF109352050093510540934D055093E0
:106820004E0560934F057093500540CFFC01659174
:1068300075918591949108958091B508882319F0F8
:1068400080E00F94CB1380E008954F925F926F9297
:106850007F928F929F92AF92BF92CF92DF92EF92F0
:10686000FF92CF93DF9300D000D01F921F92CDB73D
:10687000DEB75C01DB01CD90DD90ED90FC90E09106
:106880002C16F0912D16FE83ED8384819581A681CF
:10689000B78189839A83AB83BC839C01AD01C70117
:1068A000B6010F9499712B013C01F5018080918014
:1068B000A280B380AD81BE818D919D910D90BC91E0
:1068C000A02D8D839E83AF83B88727E137EB41ED01
:1068D00058EBC301B2010F94FA7387FDD1C023E0D6
:1068E00030E04BE953E4C301B2010F94A86A1816D3
:1068F0000CF4C6C02D813E814F815885C501B4017D
:106900000F9499712B013C0127E137EB41ED58EBD6
:106910000F94FA7387FDB4C023E030E84DE953E4E7
:10692000C301B2010F94A86A18160CF4A9C020E0A4
:1069300030E0A9016D817E818F8198850F949A71D5
:106940002B013C0120E030E040E450E40F94A86AC1
:1069500087FF05C0412C512C30E4632E762C27E1B3
:1069600037EB41ED58E3C301B2010F9499719B01DC
:10697000AC01C501B4010F94FA7387FD81C020E01A
:1069800030E84DE953E46D817E818F8198850F94C5
:106990009A712B013C0120E030E844E953E40F9464
:1069A000FA7318163CF4412C20E8522E24E9622E8A
:1069B00023E4722E27E137EB41ED58E3C301B20126
:1069C0000F949A719B01AC01C501B4010F94A86AA0
:1069D00018160CF455C020E030E0A90169817A81D5
:1069E0008B819C810F949A714B015C0120E030E017
:1069F00040E951E40F94A86A87FF06C0812C912CCE
:106A000090E9A92E91E4B92E27E137EB41ED58E347
:106A1000C501B4010F9499719B01AC01C701B60186
:106A20000F94FA7387FD2CC020E030E04BE953E46B
:106A300069817A818B819C810F949A714B015C01F1
:106A400020E030E04DE853E40F94FA73181634F464
:106A5000812C912C8DE8A82E83E4B82E27E137EB0A
:106A600041ED58E3C501B4010F949A719B01AC014B
:106A7000B1E0B983C701B6010F94A86A18160CF4E7
:106A80001982898128960FB6F894DEBF0FBECDBF5C
:106A9000DF91CF91FF90EF90DF90CF90BF90AF90BC
:106AA0009F908F907F906F905F904F9008958F92FE
:106AB0009F92AF92BF92CF92DF92EF92FF92CF93CD
:106AC000DF93EC018090DB089090DC08A090DD085B
:106AD000B090DE0820E030E0A901C501B4010F94B8
:106AE000A86A882309F452C0C880D980EA80FB8054
:106AF000A7019601C501B4010F94A86A18160CF0FD
:106B00004AC020911A0530911B0540911C055091F7
:106B10001D05C701B6010F94A86A882321F1C09210
:106B20001A05D0921B05E0921C05F0921D052091DC
:106B30001605309117054091180550911905C701A8
:106B4000B6010F940E6B9B01AC0160E070E080E831
:106B50009FE30F94997160931702709318028093CA
:106B6000190290931A026091170270911802809195
:106B7000190290911A02DF91CF91FF90EF90DF9070
:106B8000CF90BF90AF909F908F90089560E070E09D
:106B900080E89FE3F0CF60E070E0CB01ECCF9B0199
:106BA000AC01485F5F4FBC016C5F7F4F0C94FB2AC8
:106BB0000F931F93CF93DF9300D000D01F921F92AB
:106BC000CDB7DEB7FC018B0183A5811112C081E036
:106BD00083A784819581A681B781B05889839A83E0
:106BE000AB83BC83BE016F5F7F4F84EA98E00E9455
:106BF000CF351D821E821F82188620E030E040E0E3
:106C00005FE36091D8097091D9098091DA09909178
:106C1000DB090F949A7169837A838B839C839E012D
:106C20002B5F3F4FAE014F5F5F4F64ED79E080ED2A
:106C300099E00E94FB2A1D821E821F82188620E096
:106C400030E040E05FE3F8016085718582859385DF
:106C50000F949A7169837A838B839C83B8016C5FEC
:106C60007F4F9E012B5F3F4FAE014F5F5F4FC801CB
:106C70000E94FB2A28960FB6F894DEBF0FBECDBF48
:106C8000DF91CF911F910F9108952F923F924F92D4
:106C90005F926F927F928F929F92AF92BF92CF92AC
:106CA000DF92EF92FF920F931F93CF93DF93CDB7B5
:106CB000DEB7A2970FB6F894DEBF0FBECDBF8C0132
:106CC0001B015E834D834090D0095090D1096090A4
:106CD000D2097090D3098090D4099090D509A090E2
:106CE000D609B090D709DB018D919D910D90BC9193
:106CF000A02D8F87988BA98BBA8B9C01AD01C30106
:106D0000B2010F9499716B017C01D10114968D91A0
:106D10009D910D90BC91A02D8B8B9C8BAD8BBE8BD0
:106D20009C01AD01C501B4010F9499716F8B788FEF
:106D3000898F9A8FAD81BE818D919D910D90BC916F
:106D4000A02D8F839887A987BA879C01AD01C301C5
:106D5000B2010F9499716B8F7C8F8D8F9E8FAD8157
:106D6000BE8114968D919D910D90BC91A02D8B8725
:106D70009C87AD87BE879C01AD01C501B4010F940E
:106D800099716F8F78A389A39AA3A7019601C70170
:106D9000B6010F940E6B6B017C012F89388D498DE4
:106DA0005A8DCA01B9010F940E6B9B01AC01C7014A
:106DB000B6010F949A714B015C012F85388949897E
:106DC0005A896F81788589859A850F9499712B01ED
:106DD0003C012B893C894D895E896B857C858D853D
:106DE0009E850F9499716B017C01A3019201C301EF
:106DF000B2010F940E6B2B013C01A7019601C70154
:106E0000B6010F940E6B9B01AC01C301B2010F944C
:106E10009A710F9448746B017C012B8D3C8D4D8DC4
:106E20005E8DCA01B9010F940E6B2B013C012F8DB1
:106E300038A149A15AA1CA01B9010F940E6B9B0157
:106E4000AC01C301B2010F949A719B01AC01C50161
:106E5000B4010F94FA731816B4F520E030E0A901DC
:106E6000C701B6010F94FA7387FF2AC0C701B601A4
:106E7000905820E030E040EA50E40F94FA7318167E
:106E800014F5A1016D817E81C8010E944536A2964C
:106E90000FB6F894DEBF0FBECDBFDF91CF911F912B
:106EA0000F91FF90EF90DF90CF90BF90AF909F90A9
:106EB0008F907F906F905F904F903F902F900895AC
:106EC000C701B601D6CF20E030E040E050E4C50174
:106ED000B4010F94FA73181624F4B101C8010E948A
:106EE000D83519821A821B821C82BE016F5F7F4FC8
:106EF000C1010E94CF352DEC3CEC4CEC5CE3C701AA
:106F0000B6010F940E6B9B01AC01F8016081718199
:106F1000828193810F940E6B69837A838B839C8328
:106F2000C8010F940847BE016F5F7F4F8D819E811E
:106F30000E94CF35ACCF3F924F925F926F927F927B
:106F40008F929F92AF92BF92CF92DF92EF92FF9279
:106F50000F931F93CF93DF93CDB7DEB76C970FB628
:106F6000F894DEBF0FBECDBFDB010C91142F100FC4
:106F7000153008F067C11196DC90C22ECD0CB4E03C
:106F8000BC1508F45FC1ED2DF0E0E35FFA4F80809F
:106F9000912CB12CA12C002E04C0B694A7949794E8
:106FA00087940A94D2F780FE4DC1EC2DF0E0E35FA8
:106FB000FA4F8080912CB12CA12C012E04C0B694E4
:106FC000A794979487940A94D2F780FE3BC1322EFF
:106FD000642F7C0140907E0650907F066090800672
:106FE000709081068091860690918706A091880610
:106FF000B0918906898F9A8FAB8FBC8F660F770B04
:10700000072E000C880B990B0F94AF6A4B015C01A3
:10701000602F000F770B880B990B0F94AF6A298DA7
:107020003A8D4B8D5C8D0F940E6BA30192010F94E2
:107030009A71A50194010F949A716D877E878F874D
:10704000988B612F110F770B880B990B0F94AF6AF8
:10705000298D3A8D4B8D5C8D0F940E6BA30192019F
:107060000F949A71A50194010F94997169837A83A1
:107070008B839C83409082065090830660908406A8
:107080007090850680918A0690918B06A0918C065F
:10709000B0918D06898F9A8FAB8FBC8F632D660F51
:1070A000770B072E000C880B990B0F94AF6A4B01DE
:1070B0005C016D2DDD0C770B880B990B0F94AF6A7B
:1070C000298D3A8D4B8D5C8D0F940E6BA30192012F
:1070D0000F949A71A50194010F949A71698B7A8B20
:1070E0008B8B9C8B6C2DCC0C770B880B990B0F9496
:1070F000AF6A298D3A8D4B8D5C8D0F940E6BA30179
:1071000092010F949A71A50194010F9499716D8366
:107110007E838F839887F70180859185A285B385CB
:1071200089879A87AB87BC878D8B9E8BAF8BB88FF7
:1071300045E351E061E070E0CE0141960E9461EDCF
:1071400045E351E061E070E0CE0105960E9461EDFB
:107150004AE351E061E070E0CE010D960E9461EDDE
:107160004AE351E061E070E0CE0101960E9461EDDA
:1071700089889A88AB88BC8827E137EB41ED58EBCA
:10718000C501B4010F94FA7387FD5CC023E030E0C1
:107190004BE953E4C501B4010F94A86A18160CF426
:1071A00051C08D849E84AF84B88827E137EB41EDD0
:1071B00058EBC501B4010F94FA7387FD43C023E077
:1071C00030E84DE953E4C501B4010F94A86A1816DC
:1071D000CCF18D809E80AF80B88427E137EB41ED04
:1071E00058EBC501B4010F94FA7387FD2BC023E05F
:1071F00030E04BE953E4C501B4010F94A86A1816B6
:107200000CF189809A80AB80BC8027E137EB41ED9F
:1072100058EBC501B4010F94FA7387FD13C023E046
:1072200030E84DE953E4C501B4010F94A86A18167B
:107230004CF0AE014F5F5F4FBE01635F7F4FC701F0
:107240000E9445366C960FB6F894DEBF0FBECDBFD8
:10725000DF91CF911F910F91FF90EF90DF90CF9032
:10726000BF90AF909F908F907F906F905F904F9066
:107270003F9008958C38910514F08CE890E090933D
:10728000E7088093E6080C94B6DD0E945B2CCB01E6
:1072900008950F931F93CF9380911E0590911F0522
:1072A0000097E9F0FC018F01C1912C2F2F7D81F017
:1072B000C53411F0C536B9F7F801108270E060E00E
:1072C0000F943766F801C083CF911F910F910895F5
:1072D00070E060E0CF911F910F910D94376660E0F0
:1072E00070E0CB01F1CF2FEB280F2A3108F047C017
:1072F000E22FF0E080914D0590914E05A0914F0551
:10730000B091500504C0B695A795979587952A9595
:10731000D2F780FD02C081700895E15DFA4FE081EF
:10732000EE2341F18091C2089091C308E80FF92F34
:10733000F11D808190ED980F9A3030F08E3251F42B
:10734000818180538A3098F4F0931F05E0931E05E5
:1073500081E008958D3211F08B3249F4818190EDF6
:10736000980F9A3088F38E3211F48281EACFF0E0E0
:10737000E0E0EACF10921F0510921E05E9CF80E0F1
:1073800008950E947339882341F081E020911E0501
:1073900030911F05232B09F480E00895CF93DF93EC
:1073A000EB010E94C139882319F00E945B2CEB018C
:1073B000CE01DF91CF91089583E50E94C1398823E2
:1073C000E9F00F945D4E6093B6087093B708809310
:1073D000B8089093B9080E94493920E030E04AE7A4
:1073E00054E40F940E6B0F940D7360931B02709313
:1073F0001C0280931D0290931E02089580914D05FA
:1074000084FD0AC080914F0587FD06C0809150051C
:10741000837011F40C9441F40E9430F488E50E94CA
:107420007339882331F05F9A8091B4088E7F8093FE
:10743000B40889E50E947339882331F08A9A8091D3
:10744000B4088D7F8093B4088AE50E94733988233D
:1074500059F0809108018095817080930601809198
:10746000B4088B7F8093B40885E40E94733981113E
:107470000C94E1260895CF93C62F0E94C13988232A
:1074800019F0CF910C946B2C8C2FCF910895CF9243
:10749000DF92EF92FF926A017B010E94C13988233B
:1074A00031F0FF90EF90DF90CF900C944939C701F5
:1074B000B601FF90EF90DF90CF9008954F925F92CA
:1074C0006F927F928F929F92AF92BF92CF92DF92F4
:1074D000EF92FF921F93CF93DF9300D01F92CDB70F
:1074E000DEB719821A821B821C82CE0101964C01E2
:1074F00080EDC82E89E0D82E94EAE92E98E0F92E86
:1075000024ECA22E29E0B22E10E088E5810F0E9423
:10751000C139F40181934F01882341F00E94493918
:107520002B013C0180912310882359F0F6018081C2
:107530009181A281B381F70180839183A283B38378
:1075400014C0812F0E94E324882309F4D0C0F601DF
:107550002081318142815381C301B2010F949A711C
:10756000F70160837183828393831F5FF4E0CF0E02
:10757000D11C84E0E80EF11C94E0A90EB11C13307C
:1075800021F685E40E94C1398C83882309F4B9C0AF
:107590000E9449396B017C0183E00E94E324882327
:1075A00071F02091DC093091DD094091DE095091A4
:1075B000DF09C701B6010F949A716B017C01C0927B
:1075C000B008D092B108E092B208F092B30880916E
:1075D0001906882359F18091A31682FF27C08C8158
:1075E000882321F18981811103C08A818823F1F0E8
:1075F0002DEC3CEC4CE45DE360911B0970911C099F
:1076000080911D0990911E090F949A719B01AC0104
:107610006091D8097091D9098091DA099091DB09BC
:107620000F94FA73181614F40F945B5840E050E06E
:10763000BA0186E40E94473A20E030E0A9010F94A5
:10764000FA73181684F40E94493920E030E040E7CC
:1076500052E40F949472609380027093810280933D
:107660008202909383028091241083FD2CC080912C
:107670002310811128C080911708882321F12091BF
:10768000DC093091DD094091DE095091DF096091FC
:10769000B0087091B1088091B2089091B3080F942E
:1076A0009971209124083091250840912608509125
:1076B00027080F949A71609324087093250880938B
:1076C0002608909327080F900F900F900F90DF914E
:1076D000CF911F91FF90EF90DF90CF90BF90AF9030
:1076E0009F908F907F906F905F904F900895F501DD
:1076F0002081318142815381C301B2010F9499717C
:107700002FCF8091DC099091DD09A091DE09B09125
:10771000DF098093B0089093B108A093B208B093AA
:10772000B30855CFCF93DF93EB010E94C139882373
:1077300021F0DF91CF910C944539CE01DF91CF91AB
:107740000895CF93DF93C82FD62F0E94C139882385
:1077500021F0DF91CF910C947F2C8C2F0E947339F4
:10776000811101C08D2FDF91CF910895E2E1F9E001
:1077700082EBDF011D928A95E9F708958091190641
:10778000811104C00E94B63B0D94205A8091A3162B
:1077900082FD0D945B58089580911209882361F051
:1077A0009091C309891308C08091A31683FF04C078
:1077B00080E599E00D942B5A80E00895FC01238127
:1077C00021110C947BE90895CF92DF92EF92FF9202
:1077D0000F931F93CF9390913002913009F461C0C1
:1077E000662351F01092FC041092F8041092F904F0
:1077F0001092FA041092FB04C82F0F945D4EC090B3
:10780000F804D090F904E090FA04F090FB049B0196
:10781000AC012C193D094E095F0969017A01F7FC99
:1078200040C02091FC04C7FD15C04C2F0C2E000C4D
:10783000550B4C5F5F4FE22F022E000CFF0B4E17D3
:107840005F077CF144EFC42EDD24D394E12CF12CAE
:107850002C1734F438EEC32E33E0D32EE12CF12C68
:10786000C60ED71EE81EF91EC092F804D092F90485
:10787000E092FA04F092FB04022F017010E084E21F
:10788000809FB001819F700D701B112460597C4F47
:1078900082E390E00E947A968091FC048F5F80934F
:1078A000FC04CF911F910F91FF90EF90DF90CF904C
:1078B00008950F931F9301E010E020E030E0082EC0
:1078C00004C0000F111F221F331F0A94D2F74091EA
:1078D0005C0550915D0560915E0570915F05402BE0
:1078E000512B622B732B40935C0550935D05609385
:1078F0005E0570935F0590912F02891303C081E0AC
:10790000809323101F910F9108954F925F926F9271
:107910007F928F929F92AF92BF92CF92DF92EF921F
:10792000FF920F931F93CF93DF93EC0120917E067C
:1079300030917F064091800650918106688179815F
:107940008A819B810F9499716B017C012091820641
:107950003091830640918406509185066C817D812B
:107960008E819F810F9499714B015C01A701960153
:1079700060910B0270910C0280910D0290910E02A9
:107980000F94A86A882309F450C0C0920B02D092C9
:107990000C02E0920D02F0920E022091F004309160
:1079A000F1044091F2045091F304C701B6010F9421
:1079B0000E6B2B013C010F943C736B017C0120E0AA
:1079C00030E0A9010F94A86A87FD70C020E030E084
:1079D00040E450E4C701B6010F94FA7318162CF472
:1079E000C12CD12CC0E4EC2EFE2CA7019601C301C2
:1079F000B2010F9499716093E8047093E904809345
:107A0000EA049093EB04C701B6010F9406736093E8
:107A1000E604062E000C770B6F5F7F4F6430710514
:107A200014F064E070E06093E404D09109021091D6
:107A3000E604A501940160910F02709110028091FB
:107A40001102909112020F94A86A811133C0D113D0
:107A500081C02091CC043091CD044091CE0450914E
:107A6000CF046091E8047091E9048091EA04909158
:107A7000EB040F940E6B2091D0043091D10440910F
:107A8000D2045091D3040F949A71DF91CF911F913A
:107A90000F91FF90EF90DF90CF90BF90AF909F90AD
:107AA0008F907F906F905F904F900895C12CD12C54
:107AB00076019BCF80920F0290921002A092110249
:107AC000B09212022091F4043091F5044091F60432
:107AD0005091F704C501B4010F940E6B4B015C018A
:107AE0000F943C736B017C0120E030E0A9010F94FE
:107AF000A86A87FDF3C020E030E040E450E4C7010D
:107B0000B6010F94FA7318162CF4C12CD12CB0E4E2
:107B1000EB2EFE2CA7019601C501B4010F949971BB
:107B20006093EC047093ED048093EE049093EF0463
:107B3000C701B6010F9406736093E704062E000C8C
:107B4000770B6F5F7F4F6430710514F064E070E075
:107B50006093E504C091E704D11305C080910A0247
:107B60008C1709F470C08091E6049091E70490931B
:107B70000A02809309020C2E000CDD0B25E0120393
:107B8000C0011124FC01EC0FFD1FEE0FFF1FEE0FD3
:107B9000FF1FE65EF94F208131814281538120939E
:107BA000E0043093E1044093E2045093E304009135
:107BB000E504002E000C110BFC01E00FF11FEE0F8D
:107BC000FF1FEE0FFF1FE65EF94F6081718182811A
:107BD00093810F9499716093DC047093DD0480931A
:107BE000DE049093DF042091E40435E02303F001E8
:107BF0001124CE0FDF1FCC0FDD1FCC0FDD1FC65EA3
:107C0000D94F288139814A815B812093D8043093F0
:107C1000D9044093DA045093DB04E00FF11FEE0F18
:107C2000FF1FEE0FFF1FE65EF94F608171818281B9
:107C300093810F9499716093D4047093D5048093C9
:107C4000D6049093D7048090EC049090ED04A0901B
:107C5000EE04B090EF042091DC043091DD044091FB
:107C6000DE045091DF04C501B4010F940E6B209126
:107C7000E0043091E1044091E2045091E3040F9458
:107C80009A716B017C01C092D004D092D104E09231
:107C9000D204F092D3042091D4043091D5044091C1
:107CA000D6045091D704C501B4010F940E6B2091F6
:107CB000D8043091D9044091DA045091DB040F9438
:107CC0009A71A70196010F9499716093CC047093F7
:107CD000CD048093CE049093CF04BBCEC12CD12C85
:107CE000760118CF1F93CF93DF93CDB7DEB72C97D4
:107CF0000FB6F894DEBF0FBECDBF182F882379F0E2
:107D000020E030E0A901609186067091870680919D
:107D10008806909189060F94A86A8823F9F08091CB
:107D2000DF088117D9F00E9430F48CE0EFE8F2E030
:107D3000DE01119601900D928A95E1F7CE01019630
:107D40000E94853C8091DF08882391F080ED99E0C6
:107D50000E9453F41092DF080F9465092C960FB619
:107D6000F894DEBF0FBECDBFDF91CF911F91089574
:107D700081E08093DF0880ED99E00E9480F3ECCFF2
:107D800080E00E94723E109282061092830610924A
:107D900084061092850610927E0610927F0610923D
:107DA00080061092810610928A0610928B0610921D
:107DB0008C0610928D0610928606109287061092FD
:107DC000880610928906EAE1F6E02EE736E080E0C8
:107DD00090E0A0ECBFE780839183A283B383848388
:107DE0009583A683B78380879187A287B38784878B
:107DF0009587A687B787808B918BA28BB38B749660
:107E00002E173F0741F708954F925F926F927F922E
:107E10008F929F92AF92BF92CF92DF92EF92FF929A
:107E20001F93CF93DF93EC01162F2091DB08309145
:107E3000DC084091DD085091DE08688179818A81F3
:107E40009B810F94A86A882309F4AEC0B090DF0824
:107E500080E00E94723EC880D980EA80FB8020E0EA
:107E600030E0A901C701B6010F94FA7318161CF08F
:107E7000C12CD12C7601C092DB08D092DC08E092B4
:107E8000DD08F092DE082DEB37E346E855EBC7013D
:107E9000B6010F94FA7387FD0BC02DEB37E346E86C
:107EA00055E3C701B6010F94A86A18160CF078C004
:107EB000A701960160E070E080E89FE30F94947260
:107EC0006093160570931705809318059093190514
:107ED00080EF9FEFA9E7B4EC80931A0590931B0500
:107EE000A0931C05B0931D05BB2009F45DC0409014
:107EF000D0095090D1096090D2097090D309809038
:107F0000D4099090D509A090D609B090D709C09017
:107F1000D809D090D909E090DA09F090DB0981E026
:107F20000E94723E112309F43FC02091D009309184
:107F3000D1094091D2095091D309C301B2010F94E4
:107F4000A86A81111CC02091D4093091D5094091B3
:107F5000D6095091D709C501B4010F94A86A8111BF
:107F60000EC02091D8093091D9094091DA09509179
:107F7000DB09C701B6010F94A86A8823A9F0DF9135
:107F8000CF911F91FF90EF90DF90CF90BF90AF9077
:107F90009F908F907F906F905F904F900D94E61020
:107FA00060E070E0CB018CCFDF91CF911F91FF900B
:107FB000EF90DF90CF90BF90AF909F908F907F9089
:107FC0006F905F904F9008958F929F92AF92BF9263
:107FD000CF92DF92EF92FF92C0908606D0908706F4
:107FE000E0908806F090890620E030E0A901C70102
:107FF000B6010F94A86A8823E1F1A701960160E019
:1080000070E080E89FE30F9494726B017C01809094
:108010008A0690908B06A0908C06B0908D0620E08A
:1080200030E0A901C501B4010F94A86A882329F1A1
:10803000A501940160E070E080E89FE30F949472E2
:10804000C092F004D092F104E092F204F092F304B2
:108050006093F4047093F5048093F6049093F7040E
:10806000FF90EF90DF90CF90BF90AF909F908F9058
:108070000895C12CD12C7601CACF60E070E0CB010D
:10808000DFCFEFE6F0E08081826080830895809109
:10809000BA089091BB08892B79F48091BA08909125
:1080A000BB08892B49F42091BA083091BB0881E0C4
:1080B000232B19F480E0089581E00895CF92DF9298
:1080C000EF92FF926B017C0183E3C816D104E104B7
:1080D000F10470F082E3C81AD108E108F10862E304
:1080E00070E080E090E00F942A4E0F946709ECCF87
:1080F000C701B6010F942A4EFF90EF90DF90CF900A
:108100000D9467098091A90681110AC08091D90850
:10811000813041F08091A31682FB882780F9089571
:1081200080E0089581E008955F9A8091B4088E7F81
:108130008093B4088A9A8091B4088D7F8093B408A4
:108140008091080180958170809306018091B40828
:108150008B7F8093B4080C94E1269091A31693FB37
:10816000882780F993FF06C081E090910B18911148
:1081700001C080E008958091A906811110C080910E
:10818000D908823061F00E94AD40882349F0809187
:10819000A31682FB882780F991E08927089581E062
:1081A00008950E94BB4081110DC010925C05109291
:1081B0005D0510925E0510925F05109260058FEFCD
:1081C0000E94822A0D94E91781E00D945917EEE080
:1081D000FAE010821182089581E00895DC01EC91AB
:1081E0008E2F90E0FC01EE0FFF1FE80FF91FEC52FD
:1081F000FA4E80818F77808308958F929F92AF92FD
:10820000BF92CF92DF92EF92FF920F93CF93DF93C3
:108210001F92CDB7DEB75C017B0149016B01C40E33
:10822000D51EF501808191810F94C670898300234A
:1082300011F0F7018083BE016F5F7F4FC4010F947F
:108240004530F50180819181019691838083FFEF14
:10825000EF1AFF0AEC14FD0421F780E00F90DF9184
:10826000CF910F91FF90EF90DF90CF90BF90AF90A4
:108270009F908F900895009781F41092900082E073
:10828000809391001092950010929400C19A809171
:1082900071008260809371000895019761F41092DB
:1082A000A00082E08093A1001092A5001092A4008B
:1082B00089BB8093720008957F928F929F92AF92B4
:1082C000BF92CF92DF92EF92FF920F931F93CF93C3
:1082D000DF93EC017B018881883108F0C3C090E016
:1082E000FC01EE0FFF1FE80FF91FEC52FA4E8081E0
:1082F0008F770F94033219821A8288812CE0622FC3
:108300000F944F71829FB001112430E020E0AB0147
:10831000420F531FFA01EE0FFF1FE40FF51FEC523F
:10832000FA4E908197FD08C02F5F3F4F2C303105EA
:1083300071F790E00E943B417880072D10E06801C2
:10834000CC0CDD1CF601E00FF11FEC52FA4E8081DF
:108350008068808377FC86C080E2E81682E0F806B9
:108360000CF03FC08A8128E532E0281B310987FDE7
:108370003395220F331F220F331F032E000C440BA3
:10838000550B898178E8872E912C881A910887FDF2
:108390009394880C991C880C991C092C000CAA0831
:1083A000BB0860E070E0CB01F7FC0AC0B701653B99
:1083B000710514F064EB70E0072E000C880B990B2C
:1083C000281939094A095B090F94DC7024EB30E065
:1083D00040E050E00F940E71820E931EA41EB51E55
:1083E000740187E18715D8F0298188E890E0821B25
:1083F000910927FD9395880F991F880F991FE816FB
:10840000F90604F502972FB7F894E601C00FD11FC3
:10841000CC52DA4E880F991F9A8389832FBF62E36B
:1084200070E080E090E0DF91CF911F910F91FF907D
:10843000EF90DF90CF90BF90AF909F908F907F9004
:108440000C945E402A8188E592E0821B910927FD09
:108450009395880F991F880F991FE816F90694F6CF
:10846000C701D0CFDF91CF911F910F91FF90EF9077
:10847000DF90CF90BF90AF909F908F907F900895A6
:10848000CF93DF93EB01682F70E08DE196E10E94BE
:108490005C41688179818A819B81643F21E0720718
:1084A0008105910520F464EF71E080E090E00E9486
:1084B0005E4089B182FB882780F9DF91CF910895D2
:1084C000CF93DF9300D01F92CDB7DEB78EEE92E050
:1084D000A0E0B0E089839A83AB83BC83BE016F5F69
:1084E0007F4F8AE50E9440420F900F900F900F90AF
:1084F000DF91CF910895CF93DF9300D01F92CDB736
:10850000DEB78EEE92E0A0E0B0E089839A83AB8381
:10851000BC83BE016F5F7F4F8AE00E9440420F9094
:108520000F900F900F90DF91CF910895CF93DF932D
:1085300000D01F92CDB7DEB784EF91E0A0E0B0E0AD
:1085400089839A83AB83BC83BE016F5F7F4F8CE3CB
:108550000E9440420F900F900F900F90DF91CF91AB
:108560000895CF93DF9300D01F92CDB7DEB784EF8D
:1085700091E0A0E0B0E089839A83AB83BC83BE0125
:108580006F5F7F4F80EA0E9440420F900F900F90E4
:108590000F90DF91CF9108951F920F920FB60F9217
:1085A00011240BB60F922F933F934F935F936F93CA
:1085B0007F938F939F93AF93BF93EF93FF9348EA7B
:1085C00050E064EA70E081E090E00E948F2CFF911F
:1085D000EF91BF91AF919F918F917F916F915F913B
:1085E0004F913F912F910F900BBE0F900FBE0F90A8
:1085F0001F9018951F920F920FB60F9211240BB671
:108600000F922F933F934F935F936F937F938F932B
:108610009F93AF93BF93EF93FF9348E950E064E9D2
:1086200070E090E080E00E948F2CFF91EF91BF916D
:10863000AF919F918F917F916F915F914F913F91FA
:108640002F910F900BBE0F900FBE0F901F9018959B
:108650009091C00095FFFCCF8093C6000895CF9302
:10866000DF93EC018991882319F00E942843FACF07
:108670008DE00E9428438AE0DF91CF910C9428433B
:10868000CF92DF92EF92FF92CF936B017C01C42FC8
:108690004A3069F4F7FE0BC0F094E094D094C09493
:1086A000C11CD11CE11CF11C8DE20E9428434C2FFF
:1086B000C701B601CF91FF90EF90DF90CF900D945E
:1086C000BD57CF93DF93EC01FE018491219688235F
:1086D00019F00E942843F8CFDF91CF9108950F93AE
:1086E0001F93CF938C01C62F89E795E10E946143C8
:1086F000C8010E9461438AE30E94284380E38C0FF3
:108700000E9428438AE0CF911F910F910C94284337
:108710008CEF96E10E94614360E08CEE96E10E944E
:108720006F4360E087ED96E10E946F4361E080ED6A
:1087300096E10E946F4361E085EC96E10E946F43F1
:1087400061E085EB96E10E946F4360E08CEA96E180
:108750000E946F4361E082EA96E10E946F4361E00C
:1087600088E996E10E946F4361E081E996E10E9409
:108770006F4361E089E896E10E946F4361E08BE717
:1087800096E10E946F4361E08DE696E10E946F439F
:1087900060E08EE596E10E946F4360E080E596E13F
:1087A0000E946F4360E08AE396E10E946F4361E0BC
:1087B00089E296E10E946F4361E08AE196E10E94BE
:1087C0006F4361E083E196E10E946F4360E08CE0DB
:1087D00096E10E946F4361E083E096E10E946F435F
:1087E00061E08EEE95E10E946F4361E080EE95E1DD
:1087F0000E946F4361E08DEC95E10E946F4360E061
:1088000080EC95E10E946F4361E08BEB95E10E9463
:108810006F4361E08EEA95E10E946F4360E08AE970
:1088200095E10E946F4360E087E895E10E946F4305
:1088300060E087EA96E10E94E024682F61708EE78D
:1088400095E10C946F4380914D05827149F48091BC
:108850004F058C7829F480915005837009F475C018
:1088600082E40E947339882351F00E943A2C60936D
:10887000351070933610809337109093381083E53D
:108880000E947339882351F00E9449396093651022
:1088900070936610809367109093681084E50E942F
:1088A0007339882351F00E9449396093691070939D
:1088B0006A1080936B1090936C1088E50E94733956
:1088C000882351F00E9449396093E6097093E709C3
:1088D0008093E8099093E90989E50E947339882318
:1088E00051F00E9449396093EA097093EB09809333
:1088F000EC099093ED098AE50E9473398823B1F061
:108900000E9449396093EE097093EF098093F00952
:108910009093F1092DEC3CEC4CEC5DE30F94A86ACC
:10892000181624F08FE290E10E94614385E40E94D2
:108930007339882351F00E9449396093F20970938A
:10894000F3098093F4099093F5090895AF92BF92CB
:10895000CF92DF92EF920F931F93CF93DF935B0140
:10896000EA016901882309F463C085E190E10E946E
:108970006143F501608171818281938146E00F94AA
:108980009C21E1100BC08CE090E10E946143688162
:1089900079818A819B8146E00F949C2185E090E15A
:1089A0000E946143F601608171818281938143E07D
:1089B0000F949C218EEF9FE00E946143F80160813B
:1089C00071818281938143E00F949C2185EF9FE028
:1089D0000E946143F6012081318142815381F80177
:1089E00060817181828193810F94997143E00F942A
:1089F0009C21EE20F9F08AE00E94284380EE9FE05F
:108A00000E946143688179818A819B8146E00F944D
:108A10009C218AE00E9428438AE0DF91CF911F9138
:108A20000F91EF90DF90CF90BF90AF900C942843C0
:108A3000E110E4CFDF91CF911F910F91EF90DF9084
:108A4000CF90BF90AF9008950F931F93CF938C0159
:108A5000C62F80E89AE00E946143C8010E946143EA
:108A6000CC2331F08AE0CF911F910F910C942843D1
:108A7000CF911F910F9108950F931F93CF938C0166
:108A8000C62F60E080E99AE00E942445C8010E9458
:108A90006143CC2331F08AE0CF911F910F910C9468
:108AA0002843CF911F910F91089561E088E99AE0E2
:108AB0000C943C45EF92FF920F931F93CF937C0150
:108AC0008B01C42F60E080E99AE00E942445C70131
:108AD0000E94614380E20E942843C8010E946143D2
:108AE000CC2319F08C2F0E9428438AE0CF911F914C
:108AF0000F91FF90EF900C942843DF92EF92FF923A
:108B00000F931F93CF93DF93D82E7B018A01E90146
:108B10000E945545D092BC0840E0B70185ED95E430
:108B20000E945A450115110531F040E0B8018EEC64
:108B300095E40E945A45209731F040E0BE018EEC4A
:108B400095E40E945A4561E089EC95E4DF91CF916C
:108B50001F910F91FF90EF90DF900C943C4561E0E6
:108B60008AE89AE00C942445AF92BF92CF92DF92AC
:108B7000EF92FF920F931F93CF93DF9387ED99E0CE
:108B80000E946143C0E0D7E0D15021F080E20E9412
:108B90002843FACF8C2F0F942458CF5FC53099F714
:108BA0008AE00E9428430AE116E0C0E080E20E94C9
:108BB00028438C2F0F9424585801D5E080E20E945E
:108BC0002843F501C080D180E280F380A70196019F
:108BD000C701B6010F948C74882369F180E20E946A
:108BE00028438DE30E9428438DE30E9428438DE3B0
:108BF0000E9428438DE30E9428438DE30E9428436E
:108C0000D150F4E1AF0EB11CD111D8CF8AE00E944F
:108C10002843CF5F0C5F1F4FC53041F68AE0DF91DC
:108C2000CF911F910F91FF90EF90DF90CF90BF9069
:108C3000AF900C94284320E030E0A901C701B601B1
:108C40000F94FA7387FD03C08BE20E94284343E030
:108C5000C701B6010F949C21D3CF811107C081E6D3
:108C600090E10E9461438AE00C94284385E690E1FC
:108C7000F8CFCF93DF93EB010E946143CE01DF91E8
:108C8000CF910D942B58CF93C62F0E9461438C2F08
:108C9000CF910D942458CF92DF92EF92FF926A0108
:108CA0007B010E94614342E0C701B601FF90EF9053
:108CB000DF90CF900D949C2180914E0587FD2BC0B5
:108CC00080914F058E7039F54091591050915A108E
:108CD00060915B1070915C108FE190E10E944B46B7
:108CE00040915D1050915E1060915F107091601026
:108CF0008CE190E10E944B464091611050916210CE
:108D0000609163107091641083EF91E30E944B4671
:108D10008AE00C94284383E50E94C139882391F0AE
:108D20000E9449396093591070935A1080935B10D8
:108D300090935C1060936110709362108093631045
:108D40009093641080E50E94C139882351F00E94FD
:108D500049396093591070935A1080935B10909327
:108D60005C1082E50E94C139882351F00E94493984
:108D700060935D1070935E1080935F10909360100D
:108D800084E50E94C139882351F00E9449396093DB
:108D90006110709362108093631090936410089533
:108DA000CF92DF92EF92FF926A017B010E946143B2
:108DB0004AE0C701B601FF90EF90DF90CF900C948E
:108DC00040432F923F924F925F926F927F928F9289
:108DD0009F92AF92BF92CF92DF92EF92FF920F934A
:108DE0001F93CF93DF93CDB7DEB7C654D1090FB62B
:108DF000F894DEBF0FBECDBF70E060E085E40E9456
:108E0000923B182F8F3F09F483C08823E9F084E355
:108E10009AE1CA5BDF4F0FB6F894DEBF0FBECDBF3D
:108E2000DF91CF911F910F91FF90EF90DF90CF9046
:108E3000BF90AF909F908F907F906F905F904F907A
:108E40003F902F900C94614324EB30E03A832983C8
:108E500083E50E94C139882321F00E9445399A8315
:108E6000898365E070E083E40E94923B8AA760E01A
:108E700085E50E94A13B25968FAF259760E087E2AC
:108E80009AE10E9457CBA981BA81BD01BB0F880B23
:108E9000990B0F94AF6A6D837E838F8327969FAF64
:108EA00027970F945D4E688B798B8A8B9B8B1F3F26
:108EB00009F045C420E030E04CE053E46D817E8150
:108EC0008F8127969FAD27970F94FA7318160CF091
:108ED000AAC18CEF99E10E946143CA5BDF4F0FB6D4
:108EE000F894DEBF0FBECDBFDF91CF911F910F91E0
:108EF000FF90EF90DF90CF90BF90AF909F908F90BA
:108F00007F906F905F904F903F902F900D94A04373
:108F100046E450E05A8349839BCF1FAEAFC12496ED
:108F2000EEADFFAD2497808383C2FBEE4F2E512C14
:108F3000612C712C04C384E190E0A0E0B0E08C8B44
:108F40009D8BAE8BBF8BE4E14E2E512C612C712C8E
:108F500004C34C8A5D8A6E8A7F8AFFC22496EEAD76
:108F6000FFAD24978083D4C389819A81AB81BC8172
:108F700029A93AA94BA95CA9821B930BA40BB50B99
:108F8000B7FD59C08FAD0F9440228AE00E9428435C
:108F900089819A81AB81BC818053984FAF4FBF4F7D
:108FA00089AB9AABABABBCAB9DA9911177C02EA995
:108FB0003FA948AD59ADB101802F26969FAD2697A8
:108FC0000F94FA7318160CF053C020E030E040E024
:108FD00050E4B101802F26969FAD26970F949A7189
:108FE0006EAB7FAB88AF99AF2CA53DA54EA55FA515
:108FF00089819A81AB81BC81280F391F4A1F5B1F71
:109000002AAF3BAF4CAF5DAF20E030E040EC50E426
:109010006D817E818F8127969FAD27970F949971DF
:109020009101402F26965FAD26970F94A86A881F5E
:109030008827881F8DAB88899989AA89BB89C8161A
:10904000D906EA06FB0610F4D701C60129813A8148
:109050004B815C81281B390B4A0B5B0BDA01C90180
:1090600081389F44A241B105A8F188E499E10EC27C
:1090700089819A81AB81BC812AAD3BAD4CAD5DADA0
:10908000821B930BA40BB50B42E95BE361EA7BE324
:10909000B7FDD1CF812F0E94A3EDCDCF20E030E0EE
:1090A00040EF51E46D817E818F8127969FAD279798
:1090B0000F9499719B01AC01B101802F26969FAD51
:1090C00026970F94A86A87FFB6CF4EE35CE36EE461
:1090D0007CE3E0CF4AA55BA5888D998D4817590799
:1090E0000CF09EC003970CF49BC08BEE98E10E949D
:1090F00061431F3F09F076C0ABEDB8E1BA83A983A5
:109100008AEC98E10E94614389819A810E946143BF
:10911000488559856A857B8587EE98E10E944B4694
:109120008AE00E9428438AEC98E10E946143898189
:109130009A810E94614349A15AA16BA17CA183EE4F
:1091400098E10E944B468AE00E9428438AEC98E10D
:109150000E94614389819A810E946143B501A40103
:109160008FED98E10E944B468AE00E9428432596A5
:10917000FFAD2597FF2391F12CEA35EC47E25EE342
:1091800069A17AA18BA19CA10F940E6B6B017C014C
:109190002CEA35EC47E25EE3C501B4010F9494720A
:1091A000288539854A855B851F3F09F52093E908A5
:1091B0003093EA084093EB085093EC08C092ED0816
:1091C000D092EE08E092EF08F092F0086093F10878
:1091D0007093F2088093F3089093F40881E08093F1
:1091E00065027BCEE7E0F5E4FA83E98389CF20933B
:1091F00098153093991540939A1550939B15C092EA
:109200009C15D0929D15E0929E15F0929F1560934B
:10921000A0157093A1158093A2159093A315DECF8E
:109220000E9494CF80C088EE99E10E9461430E9421
:1092300096EC8FE78093E80824EB30E0A8EEB3E0EB
:109240000F9440716CA77DA78EA79FA728893989A5
:109250004A895B89260F371F481F591F2AAF3BAF2A
:109260004CAF5DAF1092650281E08093740232E0F2
:10927000310F3EAF323008F450CE1FAFC888D988C6
:10928000EA88FB88C9AADAAAEBAAFCAA812C912C4D
:10929000540189A29AA2ABA2BCA288869986AA860A
:1092A000BB868FE790E0A0E0B0E08C8B9D8BAE8B0F
:1092B000BF8B1C8690E49A8FACE1AB8FB6E4BC8F79
:1092C0001D8E1E8E1F8E18A23FE7432E512C612C3F
:1092D000712C1DAA8EAA9FAAA8AEB9AE1EA21FA26B
:1092E00018A619A6E1E0EDA3198E188E212C312CB9
:1092F00000E026961FAE2697F5E11F02C00111245B
:109300009C0121573A4E22963FAF2EAF2297285FFD
:109310003F4F24963FAF2EAF24974AA5042E000C52
:10932000550B5BA74AA780917402882309F4B0C04B
:109330000F945D4E69837A838B839C835091A7063B
:1093400058AB552309F48BC00E9449ED6091E408A5
:109350007091E5081F3F39F02296AEADBFAD229760
:1093600014966D917C91072E000C880B990B0F942D
:10937000AF6A1B01082F26969FAF26972D8D3E8D35
:109380004F8D58A126969FAD26970F94FA73181605
:109390003CF42D8E3E8E0F8F2696BFAD2697B8A338
:1093A0002C853A8D4B8D5C8DB101802F26969FAD1B
:1093B00026970F94A86A87FF07C02C863A8E0B8FDA
:1093C0002696EFAD2697EC8FFDA19101402F2696B2
:1093D0005FAD26976D817E818F8127969FAD279700
:1093E000FF2309F45AC00F94A86A87FF38C0498147
:1093F0005A816B817C814C195D096E097F09DB0103
:10940000CA0188589341A109B109B7FD28C08C89C8
:109410009D89AE89BF8984199509A609B709B595B3
:10942000A795979587951F3F09F079CD8093E80818
:109430004EA35FA368A779A7FD81FD8F2E812E8F94
:109440003F813F8F27964FAD279748A389819A8107
:10945000AB81BC81888B998BAA8BBB8B1DA220E032
:1094600030E040EF51E46D817E818F8127969FAD82
:1094700027970F949A719101402F26965FAD2697FA
:109480000F94A86A87FF70CD86E699E10E94614338
:10949000109274020E9496ECA1CE0F94FA731816E3
:1094A000F4F689819A81AB81BC81288939894A89FE
:1094B0005B89821B930BA40BB50BAC01BD01485813
:1094C00053416109710977FDCACF488D598D452BEC
:1094D00009F40DC1CEA0DFA0E8A4F9A4C80ED91EDE
:1094E000EA1EFB1E2EA13FA148A559A5281B390B3A
:1094F0004A0B5B0BC301B2010F94DC70A70196010C
:109500000F940E714C885D886E887F88420E531EC2
:10951000641E751E54E145165104610471040CF477
:109520000ACD8CEE48165104610471040CF0FDCC98
:1095300090E849165104610471040CF40ACD4C8A78
:109540005D8A6E8A7F8A2EEF30E040E050E0241979
:1095500035094609570929013A014C895D896E8907
:109560007F8980EE99E10E94D046B301A2018BED84
:1095700099E10E94D0464C855A8D6B8D7C8D84ED8F
:1095800099E10E944B464D8D5E8D6F8D78A18DECDB
:1095900099E10E944B46A88DB98D13970CF4A7C092
:1095A000C301B2010F94AF6A20E030E040E850E41C
:1095B0000F940E6B4B015C012C853A8D4B8D5C8DAD
:1095C0006D8D7E8D8F8D98A10F9499712BED3FE05D
:1095D00049E450E40F940E6B20E030E040E05FE39C
:1095E0000F940E6B9B01AC01C501B4010F949472F2
:1095F0006C877D878E879F87C701B6010F94AF6AFE
:109600002FE632E143E85AE30F940E6B6B017C01C5
:109610001E3F59F02AE939E949E15FE3812C912C99
:10962000A12C6EE3B62E1F3F59F42DEC3CEC4CE41C
:109630005EE37BEA872E7AEA972EA92C7EE3B72E8B
:109640006C857D858E859F850F940E6B68877987E5
:109650008A879B879B01AC010F949A71A7019601A1
:109660000F94947269A37AA38BA39CA32885398550
:109670004A855B85C701B6010F940E6BA501940165
:109680000F940E6B4B015C014C855D856E857F856B
:1096900087EC99E10E944B46B701A60181EC99E164
:1096A0000E944B468AE00E942843BEAD82EB99E1BE
:1096B000B23010F083EA99E10E94614348855985F0
:1096C0006A857B858DE999E10E944B4649A15AA1A3
:1096D0006BA17CA187E999E10E944B46B501A401E9
:1096E00081E999E10E944B468AE00E9428438C89D7
:1096F0009D89AE89BF89840D951DA61DB71DB595A1
:10970000A795979587951F3F09F028CC8093E80887
:10971000288D398D2F5F3F4F398F288F3D813C87B2
:109720004E814A8F5F815B8F27968FAD27978C8FF5
:10973000C980DA80EB80FC8098A99DA390CEE12EB1
:10974000012E000CFF08F70183E0EE0FFF1F8A9542
:10975000E1F7E459FD4F668177816F507109072E5B
:10976000000C880B990B0F94AF6A9B01AC016D81C3
:109770007E818F8127969FAD27970F94FA731816D5
:109780000CF4A7CB88EE99E10E9461430E9496EC0D
:1097900085E18E9DF0018F9DF00D1124E157FA4E69
:1097A0008FE7808722E330E049CDCF93DF93EB0151
:1097B0000E946143CE01DF91CF910D94FC313F9225
:1097C0004F925F926F927F928F929F92AF92BF92D1
:1097D000CF92DF92EF92FF920F931F93CF93DF937D
:1097E00080914F0587FD38C0809150058370A1F5A9
:1097F000C0912C16D0912D16488159816A817B81A8
:109800008BE698E10E944B464C815D816E817F81A1
:1098100083E896E40E944B46409128165091291601
:1098200060912A1670912B1680E896E40E944B46B0
:109830008AE0DF91CF911F910F91FF90EF90DF9021
:10984000CF90BF90AF909F908F907F906F905F90E0
:109850004F903F900C9428436090201670902116F2
:109860008090221690902316A0902416B090251672
:109870000091261610912716C0902816D090291610
:10988000E0902A16F0902B1688E50E94C139C82F67
:10989000882309F49AC00E944939362E472E582E43
:1098A000D92F20E030E046E953EC0F94FA7387FD9E
:1098B0000DC020E030E046E953E4632D742D852D82
:1098C0009D2F0F94A86A18160CF081C06CE271E00D
:1098D00088E598E10E94D54B6CE271E083E598E160
:1098E0000E94D54B80E598E10E946143C0E089E584
:1098F0000E94C139882361F10E944939362E472ED2
:10990000582ED92F20E030E046E953EC0F94FA733B
:1099100087FD0DC020E030E046E953E4632D742D4F
:10992000852D9D2F0F94A86A18160CF055C06CE277
:1099300071E08DE398E10E94D54B6CE271E088E321
:1099400098E10E94D54B85E398E10E946143C0E015
:109950008AE50E94C139882309F443C00E9449392D
:109960006B017C0120E030E040E151EC0F94FA7390
:1099700087FD0AC020E030E040E151E4C701B601B4
:109980000F94A86A18166CF567EF7FEF83E298E1F1
:109990000E94D54B69E070E08EE198E10E94D54BC2
:1099A0008BE198E1DF91CF911F910F91FF90EF90A4
:1099B000DF90CF90BF90AF909F908F907F906F90EF
:1099C0005F904F903F900C946143C1E090CF632C27
:1099D000742C852C9D2E8BCFA32CB42C052D1D2FE4
:1099E000B7CFCC23E1F0C301D4018093201690932C
:1099F0002116A0932216B0932316C501D801809397
:109A0000241690932516A0932616B0932716C0927D
:109A10002816D0922916E0922A16F0922B16DF9182
:109A2000CF911F910F91FF90EF90DF90CF90BF905B
:109A3000AF909F908F907F906F905F904F903F90EE
:109A400008952F923F924F925F926F927F928F92E2
:109A50009F92AF92BF92CF92DF92EF92FF920F93BD
:109A60001F93CF93DF93CDB7DEB7CB54D1090FB699
:109A7000F894DEBF0FBECDBF2DB73EB739AF28AFCC
:109A800087E00F94252D81110BC061E086E50E94CF
:109A90003B3A8DA3853060F08BEB9FE00E946143E1
:109AA000A8ADB9AD0FB6F894BEBF0FBEADBF40C3F1
:109AB0003DA1332321F08BE99FE00E9461436AE0DE
:109AC00080E50E943B3A182F8CEF810F8F3218F0FF
:109AD00087E79FE0E3CF60E085E40E94A13B882315
:109AE00009F448C081E08FABE0902C16F0902D1661
:109AF000D7012D913D914D915C916091D00970916C
:109B0000D1098091D2099091D3090F949A71AB0138
:109B1000BC0188E50E94473A69877A878B879C87D2
:109B2000F70124813581468157816091D409709174
:109B3000D5098091D6099091D7090F949A71AB01FC
:109B4000BC0189E50E94473A6D877E878F87988B95
:109B5000BE01635F7F4FCE0109960E942534382EE7
:109B600081110BC063E683E69FE00E9457CB8BE434
:109B70009FE094CF92E09FABB7CF8CE40E94733903
:109B8000082F882309F431C10E946B2C8EA38031E9
:109B900018F084E29FE082CFFEA1F13009F427C1E2
:109BA00060E083E50E94A13B8AAF882321F0011188
:109BB00002C037E03EA38DA1833020F08AE09FE011
:109BC0000E9461439091DF089DAF80E00E94723E49
:109BD0000F9422071D8A1E8A1F8A188E198E1A8ECC
:109BE0001B8E1C8E83EF9FE4A3ECB7E48D8F9E8FBA
:109BF000AF8FB8A383EF9FE4A3ECB7EC89A39AA33C
:109C0000ABA3BCA3A12FB0E0BCA7ABA7EDB7FEB739
:109C100024E0129FE019F10911240FB6F894FEBF59
:109C20000FBEEDBF8DB79EB701969CAF8BAF2DA138
:109C30004FA9BE01635F7F4FCE0109960F941B456C
:109C40009B01AC010F948C74811162C20F945D4E24
:109C5000611571058105910511F00F942E66212C77
:109C60001BAA1CAA1DAA1EAAAEA1A150BB0B2C9612
:109C7000BFAFAEAF2C97E22DF0E0F8A7EFA32BA576
:109C80003CA5E217F3070CF074C23196FEA7EDA7CE
:109C90003F932F93FF93EF9386EF9EE09F938F93D5
:109CA00080E09FE09F938F931F920E943CCB8DB7E3
:109CB0009EB709960FB6F8949EBF0FBE8DBF9EA1AA
:109CC000992309F458C10F94DF652AE030E040E0A1
:109CD00050E00F940E710F94AF6A20E030E040EA3C
:109CE00050E40F94FA730FEF1FEF181614F001E011
:109CF00010E00F94DF6528E631E040E050E00F947B
:109D00000E710F94AF6A2B013C010F94DF6520E2C6
:109D100030E040E050E00F940E716B5F7F4F8F4F4B
:109D20009F4F0F94AF6A4B015C01ADA1A430D1F4F9
:109D3000BC01A40188EE9EE00E944B46B301A20143
:109D400080EE9EE00E944B468AED9EE00E946143B9
:109D50000130110519F483E40E94284386ED9EE04A
:109D60000E946143312CC801110FAA0BBB0B2A962C
:109D70008CAF9DAFAEAFBFAF2A972C96AEADBFAD47
:109D80002C973A161B060CF0F6C02A966CAD7DADEA
:109D90008EAD9FAD2A970F94AF6A6B017C01BAAD6F
:109DA000BB2341F1AC019B010F949A7120E030E09C
:109DB00040E952E40F940E6B9B01AC01C301B20168
:109DC0000F949A712B013C0120E030E044EB53E406
:109DD0000F94FA731816FCF420E030E044EB53E4DF
:109DE000C301B2010F949971EDCF1EA2D9CE22E02A
:109DF0002EA3D6CE0F94DF6524E130E040E050E0A2
:109E00000F940E71675E7F4F8F4F9F4F0F94AF6A15
:109E1000A7019601CFCF20E030E0A901C301B20134
:109E20000F94A86A87FF0BC020E030E044EB53E4B6
:109E3000C301B2010F949A712B013C01ECCF009148
:109E40002C1610912D16F8012481358146815781F9
:109E50006D857E858F8598890F94997122966CAF58
:109E60007DAF8EAF9FAF22972BED3FE049E450E4EA
:109E7000C301B2010F940E6B20E030E044E353E4E1
:109E80000F9494726B017C010F948F726FA778AB63
:109E900089AB9AABD8012D913D914D915C9169852B
:109EA0007A858B859C850F94997126966CAF7DAFD2
:109EB0008EAF9FAF2697A50194016FA578A989A9B8
:109EC0009AA90F940E6B9B01AC0126966CAD7DADEB
:109ED0008EAD9FAD26970F949A7169837A838B8399
:109EE0009C83C701B6010F943A74A50194010F94A5
:109EF0000E6B22962CAD3DAD4EAD5FAD22970F940B
:109F00009A716D837E838F8398874BE351E070E075
:109F100060E0CE0101960E9461ED46E351E070E001
:109F200060E0CE0105960E9461EDBDA1B43099F4C8
:109F300049815A816B817C818AEC9EE00E944B466C
:109F40004D815E816F81788583E896E40E944B465F
:109F50008AE00E942843198A1A8A1B8A1C8AAE0149
:109F60004F5E5F4FBE016B5F7F4FCE0101960F9436
:109F70001808339402CF20E04FA9BE01635F7F4FE2
:109F8000CE0109960F941B454B015C01312CAC01AD
:109F90009B010F948C74811102C033243394A5016A
:109FA0009401C501B4010F948C748111E2C0EFA13A
:109FB000F8A5EE0FFF1FEE0FFF1F2BAD3CADE20F1C
:109FC000F31F80829182A282B382A50194016D8DDC
:109FD0007E8D8F8D98A10F94FA73181624F48D8EB0
:109FE0009E8EAF8EB8A2A501940169A17AA18BA122
:109FF0009CA10F94A86A87FF04C089A29AA2ABA271
:10A00000BCA2A50194016BA97CA98DA99EA90F945E
:10A010009A716BAB7CAB8DAB9EABADA5BEA5BD0104
:10A02000BB0F880B990B0F94AF6A6FA378A789A712
:10A030009AA79B01AC016BA97CA98DA99EA90F943D
:10A0400094722B013C014D8A5E8A6F8A788EEBAD4B
:10A05000FCADF8ABEFA710E0C12CD12C7601AFA579
:10A06000B8A96D917D918D919D91B8ABAFA7A301DA
:10A0700092010F9499719B01AC010F940E6B9B019F
:10A08000AC01C701B6010F949A716B017C011F5F8F
:10A09000211628F72FA138A549A55AA50F94947227
:10A0A0000F944874698F7A8F8B8F9C8FBDA1B230CB
:10A0B00068F18DA59EA50F94FC316BA57CA585EC60
:10A0C0009EE00E94D54B8FEB9EE00E94614343E0EF
:10A0D000C501B4010F949C2180E20E94284381E0D5
:10A0E000EDA1E3300CF480E0E12C8E010F5D1F4FF9
:10A0F0009E01235E3F4FAE01475E5F4FBE016B5E28
:10A100007F4F0E94A6448AE00E9428432394B3CD47
:10A110000E941C340F9409078DAD0E94723E0F946B
:10A12000E61088AD99AD0FB6F8949EBF0FBE8DBFF7
:10A13000E8ADF9AD0FB6F894FEBF0FBEEDBFC55B3D
:10A14000DF4F0FB6F894DEBF0FBECDBFDF91CF91CA
:10A150001F910F91FF90EF90DF90CF90BF90AF9045
:10A160009F908F907F906F905F904F903F902F9037
:10A1700008950E941C34332069F284EB9EE00E9413
:10A18000614381E0FDA11F160CF080E0EE24E39412
:10A190008E010F5D1F4F9E01235E3F4FAE01475E54
:10A1A0005F4FBE016B5E7F4F0E94A644698D7A8D22
:10A1B0008B8D9C8D0052110926E042E00F9475654D
:10A1C0009F938F9383EA9EE09F938F938DEA9EE007
:10A1D0009F938F931F920E943CCB2DB73EB7295F70
:10A1E0003F4F0FB6F8943EBF0FBE2DBF93CF2F92B7
:10A1F0003F924F925F926F927F928F929F92AF9217
:10A20000BF92CF92DF92EF92FF920F931F93CF9363
:10A21000DF93CDB7DEB7CC58D1090FB6F894DEBFC7
:10A220000FBECDBF84E99DE00E94614387E00F949B
:10A23000252D81118FC084E50E94C139882329F022
:10A240000E94453981110E944CEC80E090E0A0E82A
:10A25000BFE389839A83AB83BC838D839E83AF8363
:10A26000B8878DEC9CECACE4BEE389879A87AB871A
:10A27000BC8780E090E0A0E2B1E48D879E87AF8745
:10A28000B88B8CE390E09A8B898B8DEC90E09C8B63
:10A290008B8B8DEC9CECACECBEE38D8B9E8BAF8BF3
:10A2A000B88F80E090E0A0EEBFE3898F9A8FAB8FEC
:10A2B000BC8F1BA61CA64AE959E969E97EE38FE435
:10A2C0000E94473A6D8F7E8F8F8F98A360E083E462
:10A2D0000E94A13B89A360E08BE40E94A13B8AA37A
:10A2E00089E40E94C13910E0F12CE12C8823C1F0EF
:10A2F0000E946B2C90E01816190614F481E090E08F
:10A3000011E0180F212F2150330BC90126E0289F9F
:10A31000F001299FF00D1124E059F74FE280F380FE
:10A3200082E40E94C139882319F00E9445397C01DA
:10A33000E114F10459F1C70188978536910520F1A0
:10A340006CE870E086E69DE00E94D54B81E69DE0DA
:10A350000E946143C457DF4F0FB6F894DEBF0FBEB3
:10A36000CDBFDF91CF911F910F91FF90EF90DF90C4
:10A37000CF90BF90AF909F908F907F906F905F90A5
:10A380004F903F902F900895FA8AE98A8CE40E94BA
:10A39000C1398823E1F00E9449396B017C01C986EB
:10A3A000DA86EB86FC8620E030E0A9010F94FA7390
:10A3B00087FD0AC020E030E040E050E4C701B6016C
:10A3C0000F94A86A18161CF489E39DE0C1CF81E5BB
:10A3D0000E947339882331F180911E0590911F05E9
:10A3E000892BE9F00E9449396B017C01CD82DE8224
:10A3F000EF82F8862DEC3CEC4CE45DE30F94FA73AD
:10A4000087FD0AC020E030E040E751E4C701B60113
:10A410000F94A86A181634F488E09DE099CF8DED6A
:10A420009CE096CF83E50E94C1398823E9F00E9421
:10A4300049396B017C01CD8ADE8AEF8AF88E2DECDA
:10A440003CEC4CEC5DE30F94FA7387FD0AC020E00E
:10A4500030E040E050E4C701B6010F94A86A181636
:10A460001CF486EB9CE074CF80E50E94733988234E
:10A4700041F080911E0590911F05892B29F58FEFE2
:10A480008BA786E40E94C139882309F43DC00E944D
:10A4900049396B017C01C98EDA8EEB8EFC8E20E08F
:10A4A00030E040E85FE30F94FA7387FD0AC020E0D4
:10A4B00030E040E850E4C701B6010F94A86A1816CE
:10A4C0001CF585E69CE044CF8BA58F5F8BA70E948F
:10A4D00049396B017C01CD86DE86EF86F88A20E063
:10A4E00030E0A9010F94FA7387FD0BC020E030E043
:10A4F00048EC51E4C701B6010F94A86A18160CF095
:10A50000C0CF8EE89CE024CFC98CDA8CEB8CFC8C1D
:10A510008D889E88AF88B88CA7019601C701B601C7
:10A520000F940E6B9B01AC0160E070E084E490E45A
:10A530000F94947229813A814B815C810F940E6B48
:10A540002B013C01A5019401C501B4010F940E6BD0
:10A55000A70196010F940E6B2CEE31E548EB5DE3FD
:10A560000F9494729B01AC01C301B2010F940E6B66
:10A5700069837A838B839C83112309F1412F415096
:10A58000550B26E0249FF001259FF00D1124E05982
:10A59000F74F0081118188E40E94C139882319F0A6
:10A5A0000E9445398C010115110571F0C801855AC9
:10A5B00091098838910530F087E39CE0C9CE10E01E
:10A5C00000E0E9CF1C8B0B8B85E50E947339882353
:10A5D000C9F00F945D4E611571058105910511F06B
:10A5E0000F942E6680911E0590911F05892BC9F04E
:10A5F0000E944939609312057093130580931405E6
:10A60000909315056AE170E082E50E94923BAD9659
:10A610009FAF8EAFAD971816190644F083E09CE00B
:10A6200097CE60E070E088E492E4E4CF89E50E9490
:10A63000C139882381F10E9449392091C80930919C
:10A64000C9094091CA095091CB090F9499716B01C6
:10A650007C0188E50E94C139882331F10E94493983
:10A660002091C4093091C5094091C6095091C7098C
:10A670000F9499716BA37CA38DA39EA3CFA2D8A6A0
:10A68000E9A6FAA6CE0183960E94FD24811115C089
:10A6900089ED9BE05DCEC090D409D090D509E090C3
:10A6A000D609F090D709D5CF6091D0097091D10922
:10A6B0008091D2099091D309DDCF84E40E9473394F
:10A6C00011E081270E94723E80E090E0A0EAB0E4B1
:10A6D0008DA79EA7AFA7B8AB60E0CE018D960F9473
:10A6E00059085091F908CD57DF4F5883C358D040CF
:10A6F0001092F9080E941EDD86E89BE00E946143EB
:10A7000089899A894A970CF091C063E683E69BE0B9
:10A710000E9457CB0F94964E8B899C890E94B2F36E
:10A7200041E061E080E00F943824882309F491C06F
:10A730000F94A0430F94964E1092DC091092DD09FD
:10A740001092DE091092DF098CED99E00F947304EA
:10A750001BA5112309F4E2C020E030E040E751E4FA
:10A76000609155107091561080915710909158102B
:10A770000F94947221966CAF7DAF8EAF9FAF2197EF
:10A780001F3F09F00DC581E080935A0563E68BEB0E
:10A790009BE00E9457CB68E873E182E090E00E9462
:10A7A0007A9680E1E0EDF9E0A4EAB8E001900D923C
:10A7B0008A95E1F7CE0101960F940847C12CD12C60
:10A7C00076018091E40982FD9EC068E873E182E031
:10A7D00090E00E947A9620E030E040E85EE36091ED
:10A7E000B0087091B1088091B2089091B3080F94AD
:10A7F0009A716093B0087093B1088093B2089093F7
:10A80000B30820E030E040E85EE3C701B6010F94F2
:10A810009A716B017C0120E030E84BE354E40F9423
:10A82000FA7387FD60C010925A0513C063E686E78D
:10A830009BE00E9457CB0F94964E10935A0589893E
:10A840009A890E943A3961E081E00F94B322811124
:10A850005CCF6FEF8DEC9BE00E9457CB8CA58111F4
:10A8600012C081E08CA78D819E81AF81B885B058E0
:10A870008DA79EA7AFA7B8ABBE01635D7F4F84EAEB
:10A8800098E00E94CF3580E090E0A0EAB0E48093A9
:10A89000AC089093AD08A093AE08B093AF081DA686
:10A8A0001EA61FA618AABE01635D7F4F84EA98E02A
:10A8B0000E94CF35CD57DF4F5881C358D0405093B9
:10A8C000F9080E941EDD10925A058AA1811142CD1D
:10A8D0001092E7081092E6080E94B6DD90E080E052
:10A8E0000E94B2F337CDCE01CD960F94561080E181
:10A8F000E0EDF9E0A4EAB8E001900D928A95E1F765
:10A900000E9430F45ECF0E9457D263E68EEA9BE04D
:10A910000E9457CB0F94964E10925A05EDE0F5E049
:10A9200085E0DF011D928A95E9F780E1E0EDF9E02D
:10A93000A4EAB8E001900D928A95E1F789859A859D
:10A94000AB85BC858093AC089093AD08A093AE080E
:10A95000B093AF081DA61EA61FA618AABE01635D70
:10A960007F4F84EA98E00E94CF35BE01635E7F4F3F
:10A9700084EA98E00E94CF3581E080935A0589A14E
:10A98000882309F463C42091D0093091D109409102
:10A99000D2095091D309E5962CAF3DAF4EAF5FAFD2
:10A9A000E5978091D4099091D509A091D609B091ED
:10A9B000D709E1968CAF9DAFAEAFBFAFE197312C19
:10A9C000212C9FEFA4969FAFA497AFEFA896AFAFAF
:10A9D000A897BFEFC158DF4FB883CF57D040EFE4FF
:10A9E000C058DF4FE883C058D040F3ECCF57DF4F5B
:10A9F000F883C158D04027E4CE57DF4F2883C25890
:10AA0000D04081E090E0A0E0B0E0022C04C0880FCC
:10AA1000991FAA1FBB1F0A94D2F7CC57DF4F888318
:10AA20009983AA83BB83C458D040ADE0B5E0E796D4
:10AA3000BFAFAEAFE79710E000E09101032C000C30
:10AA4000440B550BC857DF4F288339834A835B83F8
:10AA5000C858D040C457DF4F2882CC58D040E79622
:10AA6000AEADBFADE7978D91E796BFAFAEAFE797BD
:10AA700090E0B0E0A0E0CC57DF4F288139814A81D7
:10AA80005B81C458D04082239323A423B523892B10
:10AA90008A2B8B2B09F024C1C857DF4F688179813D
:10AAA0008A819B81C858D0400F94AF6A2091860656
:10AAB0003091870640918806509189060F940E6B5D
:10AAC00020917E0630917F0640918006509181064C
:10AAD0000F949A71EB966CAF7DAF8EAF9FAFEB97F3
:10AAE000B801012E000C880B990B0F94AF6A2091CE
:10AAF0008A0630918B0640918C0650918D060F94FA
:10AB00000E6B20918206309183064091840650910D
:10AB100085060F949A716B017C01EB962CAD3DADCF
:10AB20004EAD5FADEB97E5966CAD7DAD8EAD9FAD57
:10AB3000E5970F9499712B013C01A7019601E196CD
:10AB40006CAD7DAD8EAD9FADE1970F9499714B01CA
:10AB50005C01A3019201C301B2010F940E6B2B01A2
:10AB60003C01A5019401C501B4010F940E6B9B013A
:10AB7000AC01C301B2010F949A710F9448744B0158
:10AB80005C01EB962CAD3DAD4EAD5FADEB976BA18F
:10AB90007CA18DA19EA10F9499712B013C01A7016D
:10ABA00096016FA178A589A59AA50F9499716B015B
:10ABB0007C01A3019201C301B2010F940E6B2B0122
:10ABC0003C01A7019601C701B6010F940E6B9B01D2
:10ABD000AC01C301B2010F949A710F94487420E044
:10ABE00030E040E751E40F949472A50194010F9472
:10ABF0009A716B017C018090120590901305A090D2
:10AC00001405B090150520E030E040E85FE3C50191
:10AC1000B4010F94FA731816F4F4C501B4010F943B
:10AC200006734B015C0160E070E0CB01181419045D
:10AC30001A041B0434F40F94DF65A50194010F94EA
:10AC40000E710F94AF6A9B01AC01B601C7010F945E
:10AC50009A716B017C01C158DF4F2881CF57D040DA
:10AC6000C058DF4F3881C058D040CF57DF4F4881A0
:10AC7000C158D040CE57DF4F5881C258D040B6019E
:10AC8000C7010F94A86A87FF2BC0A4960FAFA497A3
:10AC9000C457DF4F3881CC58D040A8963FAFA89713
:10ACA000EC96CFAEEC97ED96DFAEED97EE96EFAE6D
:10ACB000EE97EF96FFAEEF97C158DF4FC882CF57A0
:10ACC000D040C058DF4FD882C058D040CF57DF4F58
:10ACD000E882C158D040CE57DF4FF882C258D040EA
:10ACE0000F5F1F4F0530110509F0B9CE4FEF241A41
:10ACF000340A55E02516310409F083CEA4968FADB1
:10AD0000A497E82FF0E0E35FFA4F208181E090E024
:10AD1000A0E0B0E0A8960FACA89704C0880F991FD8
:10AD2000AA1FBB1F0A94D2F7822B8083A8969FADDF
:10AD3000A8976A969FAF6A97A496AFADA4976B96B3
:10AD4000AFAF6B97EC968FADEC97ED969FADED970F
:10AD5000EE96AFADEE97EF96BFADEF976F968CAFD7
:10AD60009DAFAEAFBFAF6F97A896BFADA897BF3FDF
:10AD700009F4FAC1A496EFADA497EF3F09F4F4C12A
:10AD80006B2FBB0F770B880B990B0F94AF6A209139
:10AD900086063091870640918806509189060F9467
:10ADA0000E6B20917E0630917F0640918006509177
:10ADB00081060F949A71162F072F382E292E862F71
:10ADC000902FA32DB22D65968CAF9DAFAEAFBFAFC8
:10ADD0006597A496FFADA4976F2FFF0F770B880B95
:10ADE000990B0F94AF6A20918A0630918B0640919F
:10ADF0008C0650918D060F940E6B20918206309137
:10AE0000830640918406509185060F949A716B01D8
:10AE10007C016996CCAEDDAEEEAEFFAE6997CE0199
:10AE20008F5A9F4F0E94FD24882309F4A1C120E07E
:10AE300030E040EA50E4612F702F832D922D0F9463
:10AE40009A714B015C01CB01D50121968CAF9DAF6E
:10AE5000AEAFBFAF21972596CCAEDDAEEEAEFFAE66
:10AE60002597A8962FADA89721112AC2A4963FAD89
:10AE7000A4973111FAC120E030E040EA50E4C70164
:10AE8000B6010F949A716B017C01A4964FADA49703
:10AE9000442309F40CC2A4968FADA49784300CF01F
:10AEA00006C222ED422E23E5522E2BE7622E21E42C
:10AEB000722E21968CAC9DACAEACBFAC2197259682
:10AEC0008CAD9DADAEADBFAD2597A7968CAF9DAFB8
:10AED000AEAFBFAFA7979C01AD0169966CAD7DADDC
:10AEE0008EAD9FAD69970F949971AB966CAF7DAFA6
:10AEF0008EAF9FAFAB97A501940165966CAD7DAD0C
:10AF00008EAD9FAD65970F9499712D966CAF7DAF07
:10AF10008EAF9FAF2D97AB962CAD3DAD4EAD5FADD7
:10AF2000AB9761962CAF3DAF4EAF5FAF6197A50178
:10AF300094016091D0097091D1098091D2099091CA
:10AF4000D3090F9499714B015C01A7962CAD3DADCF
:10AF50004EAD5FADA7976091D4097091D5098091EE
:10AF6000D6099091D7090F949971A7966CAF7DAFD0
:10AF70008EAF9FAFA797812F902FA32DB22D8DA7B6
:10AF80009EA7AFA7B8ABC9AADAAAEBAAFCAAC98444
:10AF9000DA84EB84FC84CDAADEAAEFAAF8AE2DEC0D
:10AFA0003CEC4CEC5CE3C301B2010F940E6B2981C5
:10AFB0003A814B815C810F940E6B2091DC093091BA
:10AFC000DD094091DE095091DF090F949A7169AF54
:10AFD0007AAF8BAF9CAFA5019401C501B4010F946A
:10AFE0000E6B4B015C01A7962CAD3DAD4EAD5FAD38
:10AFF000A797CA01B9010F940E6B9B01AC01C50163
:10B00000B4010F949A7120E030E040E050E40F94D6
:10B01000FA731816ACF420E030E040E05FE3C701BB
:10B02000B6010F949A7129966CAF7DAF8EAF9FAF2A
:10B030002997BE01635C7F4FCE0101960E94D835EF
:10B0400089859A85AB85BC8529968CAF9DAFAEAFBF
:10B05000BFAF2997A3961CAE1DAE1EAE1FAEA39721
:10B06000BE01615A7F4FCE01CD960E94CF35CE01F1
:10B0700001960F940847E0904D10F0904E1000910B
:10B080004F1010915010A0904910B0904A10C090ED
:10B090004B10D0904C109501A601B701C8010F9438
:10B0A000FA73181614F4750186018090800290904E
:10B0B0008102A0908202B09083022DEC3CEC4CEC1B
:10B0C0005DE3B701C8010F940E6B6093800270932B
:10B0D0008102809382029093830240E0BE01675B0D
:10B0E0007F4FCE018D960F94574F80E1E0EDF9E050
:10B0F000A4EAB8E001900D928A95E1F7809280026F
:10B1000090928102A0928202B09283020E944A2C05
:10B1100081119FCB20E04FEFBE01675A7F4FCE01D8
:10B1200001960E949B3720E041E0BE01675A7F4FA5
:10B13000CE0101960E949B372FEF40E0BE01675A77
:10B140007F4FCE0101960E949B3721E040E0BE0177
:10B15000675A7F4FCE0101960E949B370E9430F4C0
:10B160000E944A2C811175CB80916D1080936E10D6
:10B17000AD964EAD5FADAD9741505109AD965FAF05
:10B180004EAFAD97452B09F464CB6A968FAD6A97A5
:10B1900087FD5FCB6B968FAD6B9787FFF0CB59CB5D
:10B1A00063E68BE99BE00E9457CB0F94964E80E1BB
:10B1B000E0EDF9E0A4EAB8E001900D928A95E1F79C
:10B1C0002D853E854F8558896091B0087091B108F2
:10B1D0008091B2089091B3080F949A716093B0086F
:10B1E0007093B1088093B2089093B308CE01CD96C6
:10B1F0000F9456102D853E854F8558896091B00873
:10B200007091B1088091B2089091B3080F94997130
:10B210006093B0087093B1088093B2089093B3081C
:10B220008CA581117BCB81E08CA78D819E81AF8124
:10B23000B885B0588DA79EA7AFA7B8ABBE01635D18
:10B240007F4F84EA98E00E94CF3568CB2BA13CA1C8
:10B250004DA15EA1E5962CAF3DAF4EAF5FAFE59738
:10B260008FA198A5A9A5BAA5A4CB812F902FA32D16
:10B27000B22D21968CAF9DAFAEAFBFAF219720E02E
:10B2800030E040EA50E4C701B6010F949971259669
:10B290006CAF7DAF8EAF9FAF2597A4965FADA4979F
:10B2A00054300CF4E8CD182D092D3A2C2B2C92EDAE
:10B2B000492E93E5592E9BEF692E90E4792EF9CD16
:10B2C000A8969FADA89794300CF452C0A496AFAD49
:10B2D000A497A4300CF120E030E040EA50E4612F64
:10B2E000702F832D922D0F94997121966CAF7DAFA5
:10B2F0008EAF9FAF219720E030E040EA50E4C701D5
:10B30000B6010F9499716B017C01A496EFADA497DF
:10B31000E4300CF4C6CDCBCF812F902FA32DB22DCE
:10B3200021968CAF9DAFAEAFBFAF219720E030E04C
:10B3300040EA50E4C701B6010F949A7125966CAFAC
:10B340007DAF8EAF9FAF2597A496BFADA497B111E7
:10B35000D2CF20E030E040EA50E4612F702F832DFF
:10B36000922D0F949971162F072F382E292E9FCFCB
:10B37000A496FFADA497F1110DC020E030E040E2AB
:10B3800051E4B401C5010F949971162F072F382E7F
:10B39000292E87CDA4962FADA49724309CF020E0D1
:10B3A00030E040E251E4B401C5010F949971219657
:10B3B0006CAF7DAF8EAF9FAF2197182D092D3A2C22
:10B3C0002B2C6FCD182D092D3A2C2B2C82ED482ECD
:10B3D00083E5582E8BEF682E81E4782E6ACD80EDC0
:10B3E00099E00C9461438AEC99E00C946143CF920C
:10B3F000DF92EF92FF928AE50E94C139882309F417
:10B400005AC00E94493920E030E040E050EC0F94EF
:10B41000A86AC12CD12CE12C90ECF92E87FD0FC02D
:10B420000E94493920E030E040E050E40F94FA7384
:10B4300018160CF462C00E9449396B017C012091FE
:10B440004110309142104091431050914410C70177
:10B45000B6010F940E6B0F940673CB010F94114F2E
:10B4600080E50E94733981114EC0A7019601609159
:10B4700028167091291680912A1690912B160F94F8
:10B480009A71609328167093291680932A169093C8
:10B490002B160E94F359409128165091291660915D
:10B4A0002A1670912B168CE098E10E944B468AE098
:10B4B0000E94284305C083E50E94C1398111A1CFB4
:10B4C00080914F0587FD24C080915005837001F560
:10B4D0000E94F359409128165091291660912A161E
:10B4E00070912B168DEF97E10E944B468AE0FF90FA
:10B4F000EF90DF90CF900C942843C12CD12CE12CFD
:10B5000080E4F82E9CCF0E947F2C8111AECFD8CF43
:10B5100082E50E9473398111DBCFFF90EF90DF90BD
:10B52000CF900895CF9384E50E94C139C0E088236D
:10B53000D9F00E946B2CC82F1816B4F40E94F3594E
:10B540008DE40E94284380914A0590914B050F9409
:10B550002B586C2FCC0F770B89E291E10E94D54BD1
:10B560008AE00E942843CFEF8C2FCF9108954F920D
:10B570005F926F927F928F929F92AF92BF92CF9283
:10B58000DF92EF92FF92CF93DF93CDB7DEB72C9788
:10B590000FB6F894DEBF0FBECDBF4090C4095090E7
:10B5A000C5096090C6097090C70920914102309189
:10B5B00042024091430250914402C301B2010F94F0
:10B5C0009A7169837A838B839C838090C809909059
:10B5D000C909A090CA09B090CB09209145023091C9
:10B5E00046024091470250914802C501B4010F94B0
:10B5F0009A716D837E838F839887C090CC09D09099
:10B60000CD09E090CE09F090CF0920914902309108
:10B610004A0240914B0250914C02C701B6010F946F
:10B620009A7169877A878B879C8720914D02309128
:10B630004E0240914F0250915002C301B2010F944B
:10B640009A712B013C01209151023091520240919C
:10B65000530250915402C501B4010F949A714B01E9
:10B660005C01209155023091560240915702509151
:10B670005802C701B6010F949A716B017C010E94B8
:10B68000F3598AE790E10E94614383E50E94733990
:10B69000882321F00E947F2C80933F0280913F02FB
:10B6A000811151C081E690E10E94614382E790E1FF
:10B6B0000E94614349815A816B817C8184E691E3D8
:10B6C0000E944B464D815E816F81788583E896E4C8
:10B6D0000E944B4649855A856B857C8580E896E4B7
:10B6E0000E944B4680E790E10E94614388E690E12A
:10B6F0000E946143B301A20184E691E30E944B469C
:10B70000B501A40183E896E40E944B46B701A60167
:10B7100080E896E40E944B468AE02C960FB6F89497
:10B72000DEBF0FBECDBFDF91CF91FF90EF90DF90D6
:10B73000CF90BF90AF909F908F907F906F905F90D1
:10B740004F900C94284385E690E1AECF2F923F9224
:10B750004F925F926F927F928F929F92AF92BF9221
:10B76000CF92DF92EF92FF920F931F93CF93DF93CD
:10B77000CDB7DEB76A970FB6F894DEBF0FBECDBF68
:10B7800083E50E947339182F3090DF08882319F061
:10B790000E947F2C382E4090D0095090D1096090A3
:10B7A000D2097090D3098091D4099091D509A091C4
:10B7B000D609B091D7098B8B9C8BAD8BBE8B8091BA
:10B7C000D8099091D909A091DA09B091DB098F8B42
:10B7D000988FA98FBA8F112329F0311003C080E010
:10B7E0000E94723E86E50E947339888B20E030E02B
:10B7F000A9016091860670918706809188069091D4
:10B8000089060F94A86A882309F4C5C083E40E94BE
:10B810007339882309F498C00E9449396B017C016F
:10B82000AAE1B6E0B987A887BF83AE83F5E0FD83C0
:10B830001D861E8628EC2F8702EC1A86212C88ECA8
:10B840008B8792E49C87AE81BF81BA8BA98B15E070
:10B85000E989FA8981909190A190B190FA8BE98B56
:10B860002A85322D4B855C85C501B4010F94A86AE9
:10B8700087FF04C08A86292CAB86BC862D853E8531
:10B880004F85502FC501B4010F94FA73181624F494
:10B890008D869E86AF860B2D1150D1F6FD81F1501D
:10B8A000FD838E819F8144969F838E83F111CBCF40
:10B8B0002D853E854F85502F6A85722D8B859C8501
:10B8C0000F949A7120E030E040E05FE30F940E6B3C
:10B8D000A70196010F949A716B017C012DEB37E360
:10B8E00046E855EB0F94FA7387FD0AC02DEB37E35A
:10B8F00046E855E3C701B6010F94A86A181624F567
:10B9000080E00E94723E15E0A884B98405E0D5016C
:10B910006D917D918D919D915D014D01B4E08B1AEA
:10B920009108A70196010F949971F40160837183C6
:10B9300082839383015059F71150888599854496E5
:10B94000998788871111E0CFA889AA2381F020E088
:10B9500030E0A90160918606709187068091880683
:10B96000909189060F94A86A81110E94B4458AE5D6
:10B970000E947339882359F00E94493969837A8378
:10B980008B839C8360E0CE0101960E94043F832D4F
:10B990000E94723E0BC0311003C09889992339F37D
:10B9A0000E94F35984EE9DE00E946143332051F0E0
:10B9B0008091DF08811106C00E94EF5985EC9DE05F
:10B9C0000E9461430E94F35987EB9DE00E9461430E
:10B9D0008091DF080E942D460E94F3598AEA9DE07B
:10B9E0000E946143C090DB08D090DC08E090DD0845
:10B9F000F090DE0820E030E0A901C701B6010F9405
:10BA0000FA7318160CF053C042E0C701B6010F9448
:10BA10009C218DE00E9428438AE00E942843A301D4
:10BA200092016091D0097091D1098091D2099091D1
:10BA3000D3090F94A86A81111FC02B893C894D89B5
:10BA40005E896091D4097091D5098091D609909151
:10BA5000D7090F94A86A81110FC02F89388D498D9D
:10BA60005A8D6091D8097091D9098091DA09909125
:10BA7000DB090F94A86A81110F94E6106A960FB63D
:10BA8000F894DEBF0FBECDBFDF91CF911F910F9114
:10BA9000FF90EF90DF90CF90BF90AF909F908F90EE
:10BAA0007F906F905F904F903F902F90089585EA20
:10BAB0009DE00E946143B3CFCF93C82F82E0C111B4
:10BAC00084E040E060E00E94589C0E94F3598DEAB7
:10BAD0009AE0CC2311F082EC9AE0CF910C94614370
:10BAE0000E9496EC0E94E44080E00F94C243809153
:10BAF0006F088130A1F40E94EF5983E599E00E941C
:10BB0000614360E089E499E00E9457CB6EE571E003
:10BB100080E090E00E945E4088E080936F08089586
:10BB2000CF92DF92EF92FF921F93CF93DF9300D0DB
:10BB30001F92CDB7DEB78EEEC82E82E0D82EE12C54
:10BB4000F12CC982DA82EB82FC82BE016F5F7F4FEB
:10BB50008AE50E94404281110EC010E0812F0F90B3
:10BB60000F900F900F90DF91CF911F91FF90EF906A
:10BB7000DF90CF9008950E94B142C982DA82EB82B1
:10BB8000FC82BE016F5F7F4F8AE50E944042182F02
:10BB9000882319F30E94EF598DE29AE00E946143D5
:10BBA0000E94705DDBCFCF92DF92EF92FF921F93E6
:10BBB000CF93DF9300D01F92CDB7DEB78EEEC82EA5
:10BBC00082E0D82EE12CF12CC982DA82EB82FC8251
:10BBD000BE016F5F7F4F8AE00E94404281110EC01C
:10BBE00010E0812F0F900F900F900F90DF91CF9169
:10BBF0001F91FF90EF90DF90CF9008950E94B14287
:10BC00000E9460420E947B420E946042C982DA82A6
:10BC1000EB82FC82BE016F5F7F4F8AE00E94404250
:10BC2000182F8823E9F20E94EF5980EF99E00E94D3
:10BC300061430E94705DD5CFFF920F931F93CF9306
:10BC4000DF93EC018B01F42E0E9496EC0E94EF59D9
:10BC500089E299E00E9461430115110511F407E0A2
:10BC600015E4209711F4C0E2D9E00E9448D21F9356
:10BC70000F93DF93CF9380E199E09F938F9381E0BF
:10BC80008F930E943CCB0E946F9BC0915E16C6951D
:10BC9000C69589E596E10E941B2FDC2FDD0F1D2F35
:10BCA0001C0FEDB7FEB737960FB6F894FEBF0FBE68
:10BCB000EDBF83E00E94992E44E253E16C2F80E0B7
:10BCC0000E94C63110929416D093951681E099E0A7
:10BCD0000E94AB2F109294161093951684EF98E063
:10BCE0000E94AB2F8DE596E10F9450568111E1CF64
:10BCF00061E087E199E00E94244589EE93E030E617
:10BD0000019729F0232F2A950000E9F7F9CFF8943D
:10BD100089EE93E038EE019729F0232F2A95000051
:10BD2000E9F7F9CF0E9496ECFF2041F00E94944081
:10BD30000E94E326909905C0A895FCCF0E94E126B9
:10BD4000F7CF909B02C0A895FCCFF0E0E0E0DF9138
:10BD5000CF911F910F91FF9019945F926F927F92F4
:10BD60008F929F92AF92BF92CF92DF92EF92FF920B
:10BD70000F931F93CF93DF931F92CDB7DEB77C0154
:10BD800039018B015B01A40EB51ED12CC12CA0166C
:10BD9000B10609F450C0F70180809180F8015190FC
:10BDA0008F015982C4010F94C6705816B9F1652DE0
:10BDB000C4010F94CE70FFEFCF1ADF0AC6018F7750
:10BDC0009927892B21F162E070E080E090E00F94E8
:10BDD0002A4EC4010F94C67099818917F9F00E9408
:10BDE000F35983E596E00E94614381E00F90DF9173
:10BDF000CF911F910F91FF90EF90DF90CF90BF9068
:10BE0000AF909F908F907F906F905F90089562E0C9
:10BE100070E080E090E00E945E40DBCFBE016F5F8B
:10BE20007F4FC3010F944530F701808191810196C6
:10BE300091838083ACCF80E0D9CF80916D109091B9
:10BE40006E102FEF3FEF981751F0E92FF0E0E35914
:10BE5000FF4E228130E09F5F9F7790936E10C90163
:10BE600008951F920F920FB60F9211240F900FBEDC
:10BE70000F901F9018951F920F920FB60F921124DA
:10BE80000BB60F920F931F932F933F934F935F9394
:10BE90006F937F938F939F93AF93BF93CF93DF93D2
:10BEA000EF93FF93C091C60000916E10D0916D107A
:10BEB00011E01D0F1F779091A904913108F09FC0E8
:10BEC000E92FF0E08827E859F04A8F4F0D949171DF
:10BED000795FA85FB75FC65FCD5FFF5FD15FFF5F30
:10BEE000D55FD95FFF5FDD5FE15FE55FEC5FFF5F1F
:10BEF000F75FC03229F028F5CA3011F0CD3031F5A6
:10BF0000011731F0ED2FF0E0E359FF4EC283D12F3E
:10BF1000D0936D10FF91EF91DF91CF91BF91AF91D1
:10BF20009F918F917F916F915F914F913F912F9151
:10BF30001F910F910F900BBE0F900FBE0F901F908F
:10BF40001895CD3481F081E0CE3471F080E10CC0E1
:10BF5000CA3338F4C033A0F6C03291F2CD32B1F713
:10BF6000CFCFCD3499F782E08093A904C9CFC133F4
:10BF700059F018F4C03221F2E9CF88E0C433A1F3BC
:10BF80008BE0C83389F3E2CF83E0EECF84E0C033A7
:10BF900059F386E0C13341F3D9CF85E0C833B1F618
:10BFA000E3CF87E0C23391F6DFCF89E0C13371F68A
:10BFB000DBCF8AE0C03351F6D7CF8CE0C73331F600
:10BFC000D3CF8DE0C63311F6CFCFC03209F498CF6E
:10BFD0008EE0C33549F2BACF80ED8C0F8A3008F07D
:10BFE0008FCF9FE09093A9048093A80489CFCA3093
:10BFF00019F0CD3009F084CF1092A90481CFCA3056
:10C0000019F0CD3009F07CCF809197168823A1F3E9
:10C01000973041F138F4953079F71092740210920C
:10C02000BF08EACF9A3011F19F3031F79091A80400
:10C030008091BC081092BC08823089F38430E9F00A
:10C040008130D1F69923B1F09130B1F682E080933E
:10C05000BE088091BD08882379F210925D020E948B
:10C06000CE26CACF81E080939C06C6CF81E0809324
:10C070009B06C2CF8093BE08BFCF84EA91E2909323
:10C080002D0880932C08B8CF8EBD0DB407FEFDCFD0
:10C0900008958FEF8EBD0DB407FEFDCF8EB50895C8
:10C0A000909164009B7F90936400982F906A96957E
:10C0B0009CBD80FD03C091E0863009F490E09DBDF9
:10C0C0000895CF93DF93EB010E946143CE01DF918E
:10C0D000CF910C9413E6AF92BF92CF92DF92EF9282
:10C0E000FF920F931F93CF93DF93CDB7DEB7E69701
:10C0F0000FB6F894DEBF0FBECDBF00915105109171
:10C100005205F80101900020E9F731976F01C01A3C
:10C11000D10AF801CF01801B910B8C159D053CF4D1
:10C1200081918F32B9F7DF0111971C92F3CF8BE128
:10C13000E4ECF6E1DE015C9601900D928A95E1F760
:10C14000F12CE12CEC14FD040CF05DC0F801EE0DB7
:10C15000FF1D8081811103C08FEFE81AF80A580192
:10C16000AE0CBF1CF5018081882309F44CC0FFEFA1
:10C17000EF1AFF0AF801EE0DFF1D7F01E01AF10A28
:10C1800081918111FACFCE014C960E9479EA8BE120
:10C19000FE017C96DE01119601900D928A95E1F7E1
:10C1A000B501CE0101960E9485E2CE0101960E9462
:10C1B000DE3B8FE20E9428438091E11281113BC057
:10C1C00087E893E00E9413E68091A31684FF1BC0CA
:10C1D00019821C8221E0A501BE01645E7F4FCE0161
:10C1E00001960F94BD1F811129C08AE00E94284347
:10C1F0000E94F359B5018AE798E10E946160CE017F
:10C2000001960E94DE3B8AE00E942843CE014C96B4
:10C210000E94DE3BE6960FB6F894DEBF0FBECDBFA0
:10C22000DF91CF911F910F91FF90EF90DF90CF9012
:10C23000BF90AF90089581EE92E1C4CFCE014C96AD
:10C240000E947BE98BE1FE013196DE015C96019054
:10C250000D928A95E1F7CE0101960E94DE3B72CFE6
:10C260002F923F924F925F926F927F928F929F9206
:10C27000AF92BF92CF92DF92EF92FF920F931F93F4
:10C28000CF93DF9300D000D000D01F921F92CDB784
:10C29000DEB7B82E80915A11843008F0D1C10F94C6
:10C2A0005D4E6B017C0180915A11811108C0809113
:10C2B0006D1090916E10891B8F7709F4D9C681E6B5
:10C2C000A82E13C08A3019F08D3009F0F6C01092F4
:10C2D00055118091F3109091F410FC01E151FF4E43
:10C2E0001682892BF1F40F94670980915A118430DA
:10C2F00008F0ECC080916D1090916E10891B8F77C3
:10C3000009F4E4C00E941D5F97FFDCCF0E94EF5943
:10C3100089E997E00E94614380916D1080936E10CF
:10C32000E4CF1092F4101092F31005EF10E1F80131
:10C330008191803209F446C08E3409F0A9C064E9C5
:10C3400077E0C8010F94256A4C01892B41F06EE417
:10C3500070E0C80104960F94EF74009709F4C801C7
:10C360004AE050E070E060E001960F9495672B0181
:10C370003C018091EF109091F010A091F110B091DC
:10C38000F2100196A11DB11D481659066A067B06DA
:10C3900029F060E081E697E0892851F16AE270E0D7
:10C3A000C8010F941E759C01009729F1982F901BCE
:10C3B000912C992349F09150F801E90FF11D8081EA
:10C3C0009826F7CF8F01B3CF4AE050E070E060E0ED
:10C3D000C90101960F949567292D30E050E040E0A7
:10C3E000621773078407950751F060E082E497E0D5
:10C3F0000F9444357ACF60E088E197E0F9CF40921E
:10C40000EF105092F0106092F1107092F210809143
:10C410006F088130E1F067E470E0C8010F94EF74B9
:10C420000097A9F04AE050E070E060E001960F94B8
:10C430009567643071058105910548F487E796E0BA
:10C440000E94614360E08DE696E00E9457CBC09267
:10C45000C408D092C508E092C608F092C70880913F
:10C46000F5108B3309F441CF80915A11843008F0D4
:10C470003CCF80915C118A9DC001112465EF70E171
:10C48000835A9E4E0F94FA7480E00F94FE342DCFA1
:10C490008091A31680FFBBCF6AE874E4C8010F94B3
:10C4A000256A009731F0FC01838180538A3008F0BF
:10C4B000AECF60E08EEE96E09BCF23EF30E145EF0C
:10C4C00050E165E571E10E948C240FCF8091A316A5
:10C4D00082FFB6C01A82198271E6F72EE0E1EE2ED5
:10C4E000F9E6DF2E80915A11843008F0A9C00E942D
:10C4F000C4248111A5C041E050E0BE016B5F7F4FB5
:10C5000088E098E10E94B3E60D8110E0019711F0F8
:10C510000FEF1FEF8091101890911118A091121831
:10C52000B091131880939F169093A016A093A11614
:10C53000B093A2160E94C4240F3F100749F4811142
:10C5400007C00E94EF5987EB97E00E946143CACF72
:10C5500040915C11242F30E00A3061F00D3051F031
:10C56000882309F45FC089819A81009719F00196A8
:10C570009A8389831092AC0489819A81F29EF0019A
:10C58000F39EF00D1124E65AFE4EE80FF91F1382B8
:10C59000892B69F50F9467090E94C424882309F444
:10C5A000A1CF0E9430F488E098E10E947BE980915D
:10C5B0009A16882391F1815080939A168D9DC0011F
:10C5C000112462E08456984F0F94325BE0919A16E2
:10C5D00024E0E29FF0011124E856F84F6081718158
:10C5E000828193810E94742A0E94EEE17BCF1A829D
:10C5F000198281E00F94FE3480919F169091A016CD
:10C60000A091A116B091A216809356119093571144
:10C61000A0935811B0935911BFCF0E9484E9E092C2
:10C620006F0860CF4F9DA0011124435A5E4E9E01BA
:10C630002F5F3F4F6CEA74E0802F0E948C2452CF12
:10C640000F945D4E6B017C01B11004C08091A9066E
:10C65000882351F0C092B608D092B708E092B8088B
:10C66000F092B908BB24B39480912A0590912B05D0
:10C67000A0912C05B0912D050097A105B10551F1B0
:10C680004091B6085091B7086091B8087091B90808
:10C69000840F951FA61FB71FA7019601281B390BF2
:10C6A0004A0B5B0BDA01C901B7FD14C00E94EF59B8
:10C6B0006091C2087091C30882E198E00E946160B5
:10C6C0008AE00E94284340E070E060E090E080E073
:10C6D0000E941C5E80911B0290911C02A0911D0281
:10C6E000B0911E02892B8A2B8B2B79F090913116F9
:10C6F00080913216981709F4ACC1C092B608D09256
:10C70000B708E092B808F092B9088091BD04909102
:10C71000BE049099E0C101969093BE048093BD043D
:10C720008091BD049091BE048E3E92406CF00E94B8
:10C73000EF598FEE97E00E94614340E070E060E0C7
:10C7400090E080E00E941C5E0F945D4E4B015C0106
:10C750008091BF08811108C0209131169091321646
:10C7600081E0291301C080E0209193153091941548
:10C7700091E089272A3A31050CF480E091E040915C
:10C78000B1045091B2046091B3047091B404452B8C
:10C79000462B472B09F490E0981789F0882309F479
:10C7A000A0C1D501C40180569444A24FBF4F8093CD
:10C7B000B1049093B204A093B304B093B404409036
:10C7C000DC095090DD096090DE097090DF0920914E
:10C7D000AD043091AE044091AF045091B004C30158
:10C7E000B2010F94A86A882319F18091B104909145
:10C7F000B204A091B304B091B4044092AD0450923D
:10C80000AE046092AF047092B004892B8A2B8B2BFC
:10C8100009F449C0D501C40180569444A24FBF4FCA
:10C820008093B1049093B204A093B304B093B40482
:10C830008091B1049091B204A091B304B091B4047A
:10C840000097A105B10579F1881A990AAA0ABB0ACD
:10C85000B7FC29C01092B1041092B2041092B30434
:10C860001092B4048AED97E00E94614360E086EC88
:10C8700097E00E9457CB80919515909196151816C8
:10C88000190624F490E080E00E94B2F38091E6085B
:10C890009091E7081816190634F41092E7081092E0
:10C8A000E6080E94B6DD8091B9049091BA04A09187
:10C8B000BB04B091BC0446015701881A990AAA0A20
:10C8C000BB0AD501C401B7FD9CC1209131169091DE
:10C8D00032164091640280916302291306C190913F
:10C8E0000E0A899FC0011124880F892F881F990B78
:10C8F00091958D8380910F0A489FC0011124880F64
:10C90000892F881F990B91958E830F945D4E6983B3
:10C910007A838B839C8340E0BE016F5F7F4FCE01A3
:10C9200005960E9489F46D8170E089E00F94544D62
:10C9300041E0BE016F5F7F4FCE0105960E9489F4F2
:10C940006E8170E087E00F94544D8091A806882393
:10C9500009F44AC100913B0210913C02C8010297C0
:10C960002091951530919615281739070CF43CC184
:10C97000809032168F82188619861A861B868091BF
:10C9800031169F80891509F4CAC0892D90E030E6E0
:10C99000A32EA89EF001A99EF00D1124ED5DF54F88
:10C9A000458956896789708D452B462B472B81F425
:10C9B000418D528D638D748D452B462B472B41F451
:10C9C000458D568D678D70A1452B462B472BE1F188
:10C9D00020E6B22EB89E9001B99E300D1124A90117
:10C9E0004D5D554F1A01FA016181728183819481F5
:10C9F0000F9448744B015C01F10161A172A183A104
:10CA000094A10F94AD6A2B013C01F10165A176A1BF
:10CA100087A190A50F94AD6A9B01AC01C301B2013F
:10CA20000F949472A50194010F940E6B4B015C015D
:10CA3000288539854A855B850F94FA73181624F486
:10CA400088869986AA86BB868F818F5F8F708F8339
:10CA500096CFBB2019F01092BF0457CE0F945D4EB5
:10CA60000091B6081091B7082091B8083091B90824
:10CA700080901B0290901C02A0901D02B0901E029C
:10CA8000080D191D2A1D3B1D601B710B820B930B9A
:10CA900097FDE1CF8091BF04811137CE81E0809373
:10CAA000BF045F9A8091B4088E7F8093B4088A9AFD
:10CAB0008091B4088D7F8093B4088091080180959F
:10CAC0008170809306018091B4088B7F8093B408B5
:10CAD0000E94E1261ACE181619060CF021CE0197F5
:10CAE0001BCE80E090E0DC0162CE2091321650E651
:10CAF000259F900111242D5D354FF901EA5AFF4F12
:10CB00009081899FC0011124880F892F881F990B5C
:10CB100091958D83295A3F4FF9018081EDCE209167
:10CB200035023091360240913702509138026885C3
:10CB300079858A859B850F940E6B4B015C01B8014A
:10CB4000012E000C880B990B0F94AF6A9B01AC016E
:10CB5000C501B4010F949A7169837A838B839C8396
:10CB60004091390250913A02B801CE0101960E94DB
:10CB700061ED89809A80AB80BC804090B504509074
:10CB8000B6046090B7047090B804A3019201C50187
:10CB9000B4010F94A86A87FF16C028E431EE4AE773
:10CBA0005FE3C301B2010F940E6B20E037ED43EA5F
:10CBB0005CE30F949A71A50194010F940E6B698345
:10CBC0007A838B839C8369817A818B819C8160933A
:10CBD000B5047093B6048093B7049093B8040F948F
:10CBE0000673CB010E94B2F3F4E6CF0ED11CE11C18
:10CBF000F11CC092B904D092BA04E092BB04F09246
:10CC0000BC040F94670980916F08882309F4F0C170
:10CC100080915D02882309F471C08091BD08811163
:10CC20006DC00E948240811105C08091A9068823B1
:10CC300009F464C0F894649B10C0809159029091EB
:10CC40005A02A0915B02B0915C028093930690938C
:10CC50009406A0939506B093960660919306709102
:10CC600094068091950690919606789420E030E0A5
:10CC7000A9010F94A86A87FF41C001E00093BD0895
:10CC80008091A906811138C00E9455450093BC08C7
:10CC900040E36EE778E085ED95E40E945A4561E057
:10CCA00089EC95E40E943C4510912E0560E0102728
:10CCB00088E39BE069F48CE698E00E94244580E3D9
:10CCC0000E9428438AE00E94284360E08FE498E0B5
:10CCD0000E9424458AE598E00E94614380E30E9417
:10CCE00028438AE00E942843112331F085E598E02B
:10CCF00090932D0880932C080E9430F490910901A4
:10CD0000892F8095817010910802181709F45AC074
:10CD10002091A31620622093A3168093080290FD11
:10CD200010C064EF71E080E090E00E945E400E94DD
:10CD3000A6E98091A31683FDBEC1112309F442C068
:10CD400002C00E9495E9123008F46BC100E00E9415
:10CD5000312E83E0809384020F945D4E6C597F4F97
:10CD60008F4F9F4F609356057093570580935805DA
:10CD700090935905002331F1123021F58091A316CB
:10CD800083FF20C00F941559882379F081E00F9418
:10CD9000315842EB50E062E179E089EA96E10E9485
:10CDA000B3E689EA96E10E947BE90E94CC3B8111BF
:10CDB00044C10E94B63B0F94205A81E0809399169B
:10CDC0000F94625A0F945D4E6B017C0110911F020B
:10CDD0001123F1F08091C0088823D1F04091C00464
:10CDE0005091C1046091C2047091C304460157017F
:10CDF000841A950AA60AB70AB501A40177FD1AC0DC
:10CE0000833009F430C10CF01FC181300CF024C113
:10CE1000212F30E0A8EEB3E00F944071C60ED71E6C
:10CE2000E81EF91EC092C004D092C104E092C20470
:10CE3000F092C3048091D908813009F073C00F9437
:10CE40005D4E6B017C018091C8049091C904A09152
:10CE5000CA04B091CB04A7019601281B390B4A0BD9
:10CE60005B0BDA01C901B7FD3AC0D701C601805F8B
:10CE7000984DAF4FBF4F8093C8049093C904A093BF
:10CE8000CA04B093CB0480900D0690900E06A0903B
:10CE90000F06B09010060F942717AB01BC0140930A
:10CEA0000D0650930E0660930F0670931006809146
:10CEB0001C0890911D08A0911E08B0911F088819A8
:10CEC0009909AA09BB09840F951FA61FB71F809354
:10CED0001C0890931D08A0931E08B0931F08809112
:10CEE000C4049091C504A091C604B091C704460142
:10CEF0005701881A990AAA0ABB0AD501C401B7FDCD
:10CF000011C020E8C20E2EEED21E26E3E21EF11C56
:10CF1000C092C404D092C504E092C604F092C70443
:10CF20000E942FF30F94251C0E9494CF8091290515
:10CF3000882379F10F945D4E6B017C01809125056A
:10CF400090912605A0912705B0912805460157012B
:10CF5000881A990AAA0ABB0AD501C401B7FD19C0EB
:10CF60002091290530E0A8EEB3E00F944071C60E81
:10CF7000D71EE81EF91EC0922505D0922605E09224
:10CF80002705F092280580E00F9440228AE00E9455
:10CF9000284380912405882359F10F945D4E6B013D
:10CFA0007C018091200590912105A0912205B091EE
:10CFB0002305A7019601281B390B4A0B5B0BDA01ED
:10CFC000C901B7FD15C02091240530E0A8EEB3E0FB
:10CFD0000F944071C60ED71EE81EF91EC0922005A0
:10CFE000D0922105E0922205F09223050F94385942
:10CFF0002B960FB6F894DEBF0FBECDBFDF91CF9159
:10D000001F910F91FF90EF90DF90CF90BF90AF9066
:10D010009F908F907F906F905F904F903F902F9058
:10D02000089560E08FE898E00E9457CB80916305F7
:10D0300081118CCE0E946F9B89CE8CEA98E09093F0
:10D040002D0880932C08BECE843009F0E1CE0E94DA
:10D05000F35983EB98E004C00E94F35982EE98E004
:10D060000E946143D5CE0E94F3598BEC98E0F8CF33
:10D070008091C4089091C508A091C608B091C708D6
:10D08000A7019601281B390B4A0B5B0BDA01C9017A
:10D09000885E9340A109B109B7FD11C981EB97E002
:10D0A0000E946143C092C408D092C508E092C608AD
:10D0B000F092C70804C9123028F460E08DE998E0C6
:10D0C0000E9457CB01E043CE2F923F924F925F9246
:10D0D0006F927F928F929F92AF92BF92CF92DF9288
:10D0E000EF92FF920F931F93CF93DF93CDB7DEB7ED
:10D0F000EE970FB6F894DEBF0FBECDBF8091DF086C
:10D10000888B87E50E947339882309F41FC120E0CA
:10D1100030E0A901609186067091870680918806AB
:10D12000909189060F94A86A811108C00E94EF5956
:10D1300081E99EE00E94614310E01BC18AE50E94E4
:10D14000C139882339F10E9449392091CC093091A5
:10D15000CD094091CE095091CF090F9499716B017F
:10D160007C0120E030E040E251ECC701B6010F94B1
:10D17000FA7387FD0AC020E030E040E251E4C701C5
:10D18000B6010F94A86A181674F40E94EF5984E847
:10D190009EE0D0CFC090D809D090D909E090DA09AC
:10D1A000F090DB09DECF40E050E060EC7FE788E5FF
:10D1B0000E94473A2091C4093091C5094091C6099F
:10D1C0005091C7090F9499712B013C0140E050E048
:10D1D00060EC7FE789E50E94473A2091C8093091C9
:10D1E000C9094091CA095091CB090F9499714B011B
:10D1F0005C016FEF89E40E943B3A182F6FEF8AE4DD
:10D200000E943B3A082FA3019201C301B2010F947F
:10D210008C7481116EC0A5019401C501B4010F94F5
:10D220008C74811166C08BA19CA1ADA1BEA18BABFA
:10D230009CABADABBEAB20917E0630917F0640919A
:10D24000800650918106C301B2010F9499712B01A0
:10D250003C0120E030E040E05FE36BA97CA98DA9B0
:10D260009EA90F940E6B9B01AC01C301B2010F94F8
:10D270009A712BA93CA94DA95EA90F9494720F94A1
:10D280000673162F4FA058A469A47AA42091820691
:10D29000309183064091840650918506C501B40102
:10D2A0000F9499714B015C0120E030E040E05FE3B6
:10D2B000C301B2010F940E6B9B01AC01C501B40117
:10D2C0000F949A71A30192010F9494720F940673B4
:10D2D000062F812F012E000C990B97FD2FC005976B
:10D2E0007CF5802F002E000C990B97FD2BC0059725
:10D2F0005CF5153008F020CF053008F01DCF80E038
:10D300000E94723E95E01902F0011124E00FF11D18
:10D3100007FDFA95EE0FFF1FEE0FFF1FE65EF94FB8
:10D32000C082D182E282F38288890E94723E88891B
:10D33000882309F401CF0F94E610FECE10E0D1CF80
:10D3400014E0CFCF00E0D5CF04E0D3CF8AE40E9431
:10D350007339182F811127C070E060E086E50E94C4
:10D36000923B9A838983059708F18FE59EE00E949E
:10D370006143812FEE960FB6F894DEBF0FBECDBF8E
:10D38000DF91CF911F910F91FF90EF90DF90CF90A1
:10D39000BF90AF909F908F907F906F905F904F90D5
:10D3A0003F902F9008950E94C03EC6CE60E084E476
:10D3B0000E94A13B8F8740E050E0BA018AE50E94BD
:10D3C000473A6BA77CA78DA79EA740E050E86BE388
:10D3D00076E483E50E94473A20E030E040E752E4FB
:10D3E0000F949472609378027093790280937A021A
:10D3F00090937B02E0902C16F0902D16D7018D9023
:10D400009D90AD90BC9020E030E0A901C501B40131
:10D410000F949A716BAF7CAF8DAF9EAF20E030E080
:10D4200040E450E40F94A86A87FF06C01BAE1CAE10
:10D43000B0E4BDAFE0E4EEAF20E030E84DE953E406
:10D44000C501B4010F949A71662E7BAB8FAB98AF78
:10D4500020E030E844E953E40F94FA7318163CF4E2
:10D46000612CF0E8FBAB24E92FAB83E488AFD70154
:10D4700014968D909D90AD90BC90179720E030E071
:10D48000A901C501B4010F949A71D62EE72EF82E8A
:10D49000092F20E030E040E951E40F94A86A87FFAB
:10D4A00005C0D12CE12CF0E9FF2E01E420E030E0B2
:10D4B0004BE953E4C501B4010F949A71B62EC72EFF
:10D4C00089AF9AAF20E030E04DE853E40F94FA734F
:10D4D000181634F4B12CC12CBDE8B9AFE3E4EAAFBF
:10D4E00088E40E947339882309F415C20E944939DF
:10D4F0000F9406731B0177FF02C06F5F7F4F759516
:10D5000067957195619571096A567F4F072E000CDA
:10D51000880B990B0F94AF6A762E872E982EA92E22
:10D520002D2D3E2D4F2D502F0F94FA7318161CF4ED
:10D53000D72C74010A2D2BAD3CAD4DAD5EAD672DE2
:10D54000782D892D9A2D0F94FA73181624F07BAC40
:10D550008CAC9DACAEAC872D982DA92DBA2D8B8BA4
:10D560009C8BAD8BBE8B8D2D9E2DAF2DB02F8F8BB9
:10D57000988FA98FBA8FB101330C880B990B0F9438
:10D58000AF6A1B012C01AC019B016D2D7E2D8F2DEF
:10D59000902F0F949A71D62EE72EF82E092F2B2D4F
:10D5A0003C2D49AD5AAD0F94A86A87FF04C0BD2C2D
:10D5B000CE2CF9AE0AAFA2019101672D782D892DED
:10D5C0009A2D0F949A71D62EE72EF82E092F262D1C
:10D5D0003BA94FA958AD0F94A86A87FF04C06D2CD2
:10D5E000EBAAFFAA08AF862D9BA9AFA9B8AD8B8F78
:10D5F0009C8FAD8FBE8F8B2D9C2DA9ADBAAD8F8F1B
:10D6000098A3A9A3BAA3BE01695E7F4FCE0143963A
:10D610000E942534882309F4AFC1BE01615E7F4FAB
:10D62000CE014B960E942534E82E882309F4A4C12C
:10D630002F89388D498D5A8D6F8D78A189A19AA136
:10D640000F94997120E030E040E85EE30F940E6B98
:10D650004B015C012B893C894D895E896B8D7C8DEA
:10D660008D8D9E8D0F94997120E030E040E85EE34F
:10D670000F940E6B6BA37CA38DA39EA38FA298A681
:10D68000A9A6BAA689819A811816190674F48DE2A2
:10D690009EE00E9461438F85882321F083E29EE013
:10D6A0000E9461438AE00E9428430E9430F40F9454
:10D6B000220780E00E94723E80E090E0A0E2B1E4A8
:10D6C0008FA798ABA9ABBAAB60E0CE018F960F9451
:10D6D000590820918606309187064091880650911E
:10D6E00089066BA17CA18DA19EA10F94A86A8111CE
:10D6F00030C020918A0630918B0640918C06509163
:10D700008D066FA178A589A59AA50F94A86A8111A5
:10D7100020C020917E0630917F0640918006509176
:10D7200081066B897C898D899E890F94A86A8111F5
:10D7300010C020918206309183064091840650915A
:10D7400085066F89788D898D9A8D0F94A86A8823B4
:10D75000A9F00E94C03E88E0FE01B396A6E8B6E0BC
:10D7600001900D928A95E1F788E0FE017396AEE78D
:10D77000B6E001900D928A95E1F7188A60E085E4A1
:10D780000E94A13B88248394811102C062E0862E0E
:10D790001B861C861D861E861A8A9E2C43EFC42E6D
:10D7A0004DE0D42E51E0A52E5EE0B52E1A8915303D
:10D7B0000CF0ECC06B857C858D859E859B01AC0152
:10D7C0000F948C748111E2C03324339435E0232EFE
:10D7D000911005C033243A9422242A9484E091E0E5
:10D7E0009926F12EFF0CFF0CF10EF394898B198909
:10D7F0006A89121509F4C6C0062E000C770B880B37
:10D80000990B0F94AF6A2FA138A549A55AA50F947B
:10D810000E6B2F89388D498D5A8D0F949A712B017B
:10D820003C01612F110F770B880B990B0F94AF6A96
:10D830002BA13CA14DA15EA10F940E6B2B893C89BD
:10D840004D895E890F949A716B837C838D839E834F
:10D850004F82588669867A8689819A81892B79F0E8
:10D860006F2D8FE09EE00E94434669E170E08DE0FD
:10D870009EE00E94D54B8AE09EE00E9461431F9289
:10D88000F9E1FF931F92FF92DF92CF92BF92AF9286
:10D890001F920E943CCB2981482DBE01695F7F4FBA
:10D8A000CE0103960F941B452B013C014B865C86F1
:10D8B0006D867E860FB6F894DEBF0FBECDBFAC017D
:10D8C0009B010F948C7481115AC009898A8925E0C3
:10D8D000020380011124080F111D87FD1A95000F06
:10D8E000111F000F111F065E194FA30192016BA5B6
:10D8F0007CA58DA59EA50F949A71D8016D937D93FB
:10D900008D939C931397188A81E00E943061F39461
:10D910008989830D6BCF4D2D5E2D6F2D702F86E481
:10D920000E94473A1B012C014BAD5CAD6DAD7EAD45
:10D930008CE40E94473A6B8B7C8B8D8B9E8B2F8A5D
:10D94000388E498E5A8E4B2D5C2D69AD7AAD82E4AE
:10D950000E94473A6B017C01462D5BA96FA978AD07
:10D9600082E50E94473A6B8F7C8F8D8F9E8FCF8E82
:10D97000D8A2E9A2FAA247CE83E49EE0F8CC888937
:10D980000E94723E8A898F5F8A8B10CF0F94A043CA
:10D990000E941C34882359F088890E94723E80E0DE
:10D9A00090E0A0ECBFE78B879C87AD87BE876B8537
:10D9B0007C858D859E859B01AC010F948C748111B3
:10D9C00059C08F85811126C082E0F82E02E094E0D4
:10D9D000C92E12E0DC2CD11A21E041E0612F802F0A
:10D9E0000E943E2521E04FEF612F8F2D0E943E25A2
:10D9F0002FEF41E06D2D802F0E943E252FEF4FEF3E
:10DA00006D2D8F2D0E943E25115020F70150F3946B
:10DA10000F3FF9F60E94B4450E94E43F8F858111C3
:10DA200024C088ED99E00E9457354B015C0180EDE0
:10DA300099E00E94853C9B01AC01C501B4010F94A3
:10DA40000E6B9B01AC016091D8097091D90980914E
:10DA5000DA099091DB090F9499716093D80970935A
:10DA6000D9098093DA099093DB098F858111E888C1
:10DA7000E092DF080F9409078091DF0881110F946D
:10DA800065090E94202C0F94E6106B857C858D859E
:10DA90009E8511E09B01AC010F948C74811169CCBF
:10DAA0004BCBCF93DF93C82FD62F8091241083FDCB
:10DAB00014C08091200A811110C080918902909138
:10DAC0008A02AC014150510920919515309196156B
:10DAD0002417350714F40E94B2F340E06D2F8BE059
:10DAE0000E94589CCC2339F040E061E080E0DF9157
:10DAF000CF910D9438248091200A91E0892780935A
:10DB0000740280917402882389F08091931590911A
:10DB100094152091951530919615821B930B97FFC4
:10DB200003C0919581959109029744F41092740273
:10DB30008091241083FF06C0C1E01AC080E00E94DB
:10DB40003061DFCFC091200AC11112C080918902DB
:10DB500090918A020197209195153091961528177A
:10DB6000390754F70E94F3598CE99AE00E94614307
:10DB70008C2FDF91CF910895AF92BF92CF92DF9219
:10DB8000EF92FF920F931F93CF93DF93CDB7DEB742
:10DB900064970FB6F894DEBF0FBECDBF0E94925AB5
:10DBA000D82E87FDB5C08AE50E94C139882309F4C3
:10DBB000C0C040E050E0BA018AE50E94473A7B01CC
:10DBC0008C014D2D63E085E00E94589C2091D8097E
:10DBD0003091D9094091DA095091DB0960E070E099
:10DBE00088EC93E40F9499715B016C019701A80193
:10DBF0000F94FA73181614F07501860120E030E0D6
:10DC0000A901B701C8010F94FA73181624F4E12C86
:10DC1000F12C00E010E0B701C8010F940673072E45
:10DC2000000C880B990B0F94AF6A6D837E838F83F2
:10DC3000988720E030E0A9010F94A86A882321F09A
:10DC4000CE0105960E94C22A80E090E0A0EAB1E4ED
:10DC500089879A87AB87BC871D861E861F86188A90
:10DC60008CE40E947339882309F468C00E94493902
:10DC70006B017C0120E030E0A901C701B6010F94DF
:10DC8000FA7387FF04C0F7FAF094F7F8F094C98AA2
:10DC9000DA8AEB8AFC8A209195153091961524300A
:10DCA000310574F08091931590919415821B930B1C
:10DCB00097FF03C091958195910901E004970CF4B9
:10DCC00000E063E080E00E94516D811140C083E07C
:10DCD00080933002109262050E946F9B6D817E815D
:10DCE0008F8198858B019C01305809831A832B837F
:10DCF0003C8320E030E0A9010F94A86A882321F03A
:10DD0000CE0101960E94C22A109262050E946F9B6A
:10DD100064960FB6F894DEBF0FBECDBFDF91CF91F2
:10DD20001F910F91FF90EF90DF90CF90BF90AF9039
:10DD30000895E12CF12C00E211E443CFC0901506C8
:10DD4000D0901606E0901706F090180693CF83E067
:10DD5000E82E22E0AE01475F5F4FBE016F5E7F4F4E
:10DD6000CE010D960F940844B9CF6F927F928F9297
:10DD70009F92AF92BF92CF92DF92EF92FF920F935A
:10DD80001F93CF93DF9300D000D01F921F92CDB787
:10DD9000DEB75C014B013A01F22E68010091A10649
:10DDA00010929D0610929E0610929F061092A00659
:10DDB0001092A1060F94694E809195159091961539
:10DDC0008C159D051CF4C6010E94B2F360E080E052
:10DDD0000E94516D811124C1109262050E946F9BB7
:10DDE0001C141D0444F4C6010E94B2F340E060E03C
:10DDF00080E00F94382440E060E088E00E94589C66
:10DE000060E081E00E94516D80E090E0A0E7B2E424
:10DE100089839A83AB83BC8380E090E0A0E8B0EC78
:10DE20008D839E83AF83B887BE016F5F7F4FCE0126
:10DE300005960F94A90887E00F943B06811158C0FE
:10DE40008091D8099091D909A091DA09B091DB09A4
:10DE50004091010550910205609103057091040500
:10DE6000C090FD04D090FE04E090FF04F090000507
:10DE7000C092A408D092A508E092A608F092A70844
:10DE80004093A8085093A9086093AA087093AB0820
:10DE90008093AC089093AD08A093AE08B093AF0800
:10DEA00080E090E0A8E4B2E489839A83AB83BC83EA
:10DEB000CE0101960F9456108091050590910605AC
:10DEC000A0910705B09108058093AC089093AD0828
:10DED000A093AE08B093AF0880E090E0A0EAB0E471
:10DEE00089839A83AB83BC83CE0101960F9456102D
:10DEF000C12CD12C80E7E82E82E4F82EC982DA8288
:10DF0000EB82FC8280E090E0A0E8B0E48D839E8309
:10DF1000AF83B887BE016F5F7F4FCE0105960F9428
:10DF2000A90820E030E0A9016091090570910A0577
:10DF300080910B0590910C050F94A86A87FF0BC088
:10DF4000C982DA82EB82FC82BE016F5F7F4F89E07B
:10DF500095E00F94A9088091090590910A05A09178
:10DF60000B05B0910C058093DC099093DD09A0931B
:10DF7000DE09B093DF098093B0089093B108A093B5
:10DF8000B208B093B30880EB98E00F9473048091CB
:10DF9000190681110F945B58109262050E946F9BC5
:10DFA00061E085E49BE00E9424458091A9068150B0
:10DFB0008093A90645E651E26DE47BE085E00F948D
:10DFC00012458091A906882339F00E94EEE18091E4
:10DFD000A90681508093A90680E00F94C2430E9455
:10DFE000CE268091D908823011F40F94E9170F944E
:10DFF000A0430E946F9B28960FB6F894DEBF0FBE19
:10E00000CDBFDF91CF911F910F91FF90EF90DF90E7
:10E01000CF90BF90AF909F908F907F906F9008951A
:10E02000E12C2F2DA301B401C5010F940844D8CED3
:10E030004F925F926F927F92AF92BF92CF92DF9298
:10E04000EF92FF921F93CF93DF9300D000D01F92E7
:10E050001F92CDB7DEB75C01E62EF42E642F80E070
:10E060000E94516D182F81111BC0EE2021F01092DB
:10E0700062050E946F9B812F28960FB6F894DEBF31
:10E080000FBECDBFDF91CF911F91FF90EF90DF903A
:10E09000CF90BF90AF907F906F905F904F9008951A
:10E0A000EE2029F040E06F2D83E00E94589C80E034
:10E0B00090E0A0E7B2E48D839E83AF83B88780E0D1
:10E0C00090E0A0E8B0EC89839A83AB83BC83BE0167
:10E0D0006B5F7F4FCE0101960F94A90868E873E14A
:10E0E00080E090E00E945E40C12CD12C88ECE82EAC
:10E0F00081E4F82ECD82DE82EF82F88680E090E027
:10E10000A0E8B0E489839A83AB83BC83BE016B5FD4
:10E110007F4FCE0101960F94A90840905D1050905A
:10E120005E1060905F1070906010C0925D10D09291
:10E130005E10E0925F10F092601080E090E0A0E24C
:10E14000B2E48D839E83AF83B887F501808191818E
:10E15000A281B38189839A83AB83BC83BE016B5F49
:10E160007F4FCE0101960F94A90840925D10509206
:10E170005E1060925F1070926010129A64E670E018
:10E1800080E090E00E945E4076CF8F929F92AF92A7
:10E19000BF92CF92DF92EF92FF921F93CF93DF93C4
:10E1A00000D000D01F921F92CDB7DEB70E94925AC6
:10E1B000182F87FDADC08AE50E94C139812C912CB2
:10E1C00090E2A92E91E4B92E882341F040E050E07E
:10E1D000BA018AE50E94473A4B015C01412F64E095
:10E1E00083E00E94589C20E030E0A901C501B40101
:10E1F0000F94FA7318167CF580E090E0A0EAB0E482
:10E200008D839E83AF83B8872091D8093091D90937
:10E210004091DA095091DB09C501B4010F949A715C
:10E220006B017C0120E030E048EC53E40F94A86AD5
:10E2300087FD06C0C12CD12C88ECE82E83E4F82E93
:10E24000C982DA82EB82FC82BE016B5F7F4FCE0116
:10E2500001960F943A0885E50E947339882309F4E2
:10E2600069C00E9449396B017C0120E030E0A901BE
:10E27000C701B6010F94FA7387FF04C0F7FAF09450
:10E28000F7F8F094F7FAF094F7F8F094C982DA828C
:10E29000EB82FC8244E061E0CE0101960E9418709E
:10E2A00020E030E0A901C501B4010F94FA731816FB
:10E2B0005CF580E090E0A0EAB0E48D839E83AF83BC
:10E2C000B887A50194016091D8097091D90980910E
:10E2D000DA099091DB090F9499716B017C0120E0C0
:10E2E00030E0A9010F94FA7318161CF0C12CD12C40
:10E2F0007601C982DA82EB82FC82BE016B5F7F4FBE
:10E30000CE0101960F943A08109262050E946F9B0D
:10E3100028960FB6F894DEBF0FBECDBFDF91CF9128
:10E320001F91FF90EF90DF90CF90BF90AF909F90A4
:10E330008F90089588E01802F0011124EF5EF94FE4
:10E34000C080D180E280F38090CFBF92CF92DF92E5
:10E35000EF92FF920F931F93CF93DF9300D01F9202
:10E36000CDB7DEB77C016B018A01B22E61E088E394
:10E370009BE00E94244545E651E26FE37BE085E0A7
:10E380000F9412459091A90681E0890F8093A90608
:10E390008091A31682FF06C08B7F8093A3169E5F99
:10E3A0009093A9060F94211880E1E0EDF9E0ADEF1C
:10E3B000B4E001900D928A95E1F70E9430F481E07B
:10E3C0000F94C24320E030E0A901F7016081718120
:10E3D000828193810F94A86A8823F1F08091200AAA
:10E3E00081110CC08091890290918A02019720913D
:10E3F0009315309194152817390774F080E090E058
:10E40000A0E7B2E489839A83AB83BC83BE016F5FCC
:10E410007F4FC7010F94A90887E00F943B06811135
:10E4200003C0B6010F94791B20E030E0A901F80188
:10E4300060817181828193810F94A86A882329F079
:10E4400042E06B2DC8010E941870129A64E670E0D9
:10E4500080E090E00E945E4081E00F900F900F906E
:10E460000F90DF91CF911F910F91FF90EF90DF9070
:10E47000CF90BF900895CF92DF92EF92FF92CF930B
:10E48000DF936B017C01D42FC091C00883E080939F
:10E49000C00881E08093BF08C114D104E104F104F5
:10E4A00031F00F945D4EC60ED71EE81EF91E809106
:10E4B000BF08882389F0C114D104E104F10421F4D8
:10E4C0008D2F0E943061F3CF0F945D4E6C197D0942
:10E4D0008E099F0997FDF4CF1092BF08C093C00822
:10E4E000DF91CF91FF90EF90DF90CF9008951F9331
:10E4F000CF93DF93D82FC62F0E945C5D61E08C2FF5
:10E500000E94E43B0F945D4E685370458F4F9F4FC0
:10E5100060939D0670939E0680939F069093A0063D
:10E520001092A1061091C00883E08093C00830E0EB
:10E5300020E04AEF55E46AE27BE082E00E947D45FC
:10E5400081E08093BF088091BF08882309F463C0ED
:10E5500060E08C2F0E94E43B8091A106882309F49F
:10E5600056C040E060E08AE00E94589C0E94F35947
:10E5700080E19BE00E94614330E020E04AEF5AE0F6
:10E5800061E07BE082E00E947D4541E060E070E078
:10E59000CB010E943B7230E020E050E040E06DEEA5
:10E5A0007AE085E00E947D4510929D0610929E06BD
:10E5B00010929F061092A0061092A1060F94694E29
:10E5C00060E080E00E94516D8D2F0E945C5D0F9491
:10E5D0005D4E685370458F4F9F4F60939D067093BB
:10E5E0009E0680939F069093A0061092A10630E0AD
:10E5F00020E04AEF55E461EE7AE082E00E947D453A
:10E6000081E08093BF0861E08C2F0E94E43B81E0B1
:10E610000E94306198CF1093C008DF91CF911F9175
:10E620000895CF92DF92EF92FF920F931F93CF93B3
:10E63000DF93CDB7DEB7A0970FB6F894DEBF0FBE5D
:10E64000CDBF0E94925A87FDD1C0482F61E081E082
:10E650000E94589C85E40E947339882309F4D5C030
:10E660000E9449396B017C0120E030E0A9010F9440
:10E67000FA7387FF04C0F7FAF094F7F8F094F7FA0A
:10E68000F094F7F8F094C98ADA8AEB8AFC8A8CE075
:10E69000EBE9F2E0DE01119601900D928A95E1F727
:10E6A0008AE50E94C139882351F040E050E0BA0168
:10E6B0008AE50E94473A69877A878B879C8788E535
:10E6C0000E94C139882351F040E050E0BA0188E54A
:10E6D0000E94473A69837A838B839C8389E50E94F1
:10E6E000C139882351F040E050E0BA0189E50E9429
:10E6F000473A6D837E838F83988785E50E947339BF
:10E70000882309F489C00E9449396B017C0120E00B
:10E7100030E0A901C701B6010F94FA7387FF04C066
:10E72000F7FAF094F7F8F094F7FAF094F7F8F09419
:10E73000CD8ADE8AEF8AF88E198E1A8E1B8E1C8E79
:10E740008CE40E947339882309F46FC00E94493910
:10E750006B017C0120E030E0A901C701B6010F94F4
:10E76000FA7387FF04C0F7FAF094F7F8F094CD8EAF
:10E77000DE8EEF8EF8A262E070E082E40E94923BAF
:10E78000F82E8091A906811131C021E0AE014B5EC7
:10E790005F4FBE016F5F7F4FCE0141960E94A57112
:10E7A000882321F16F2D81E00E94777282E50E941B
:10E7B000C139882309F442C00E94453940E050E045
:10E7C00060EA71E44D875E876F87788B2091A90698
:10E7D000222361F08C012F2DAE01435F5F4FBE01FC
:10E7E000635E7F4FCE0149960E94B56EA0960FB62C
:10E7F000F894DEBF0FBECDBFDF91CF911F910F9177
:10E80000FF90EF90DF90CF900895C12CD12C80E83D
:10E81000E82E80E4F82E33CFC0901106D090120677
:10E82000E0901306F090140672CFC0901506D090B9
:10E830001606E0901706F09018068CCF90E080E066
:10E84000BDCFCF92DF92EF92FF920F931F93CF93A2
:10E85000DF93CDB7DEB76C970FB6F894DEBF0FBE6F
:10E86000CDBF8CE40E947339882309F4C3C00E9491
:10E8700049396B017C0120E030E0A9010F94FA7363
:10E8800087FF04C0F7FAF094F7F8F094F7FAF094E1
:10E89000F7F8F094C98EDA8EEB8EFC8E8CE0EBE903
:10E8A000F2E0DE01119601900D928A95E1F788E57C
:10E8B0000E94C1398823A1F040E050E0BA0188E508
:10E8C0000E94473A2091C4093091C5094091C60978
:10E8D0005091C7090F94997169837A838B839C83C4
:10E8E00089E50E94C1398823A1F040E050E0BA01D7
:10E8F00089E50E94473A2091C4093091C5094091A9
:10E90000C6095091C7090F9499716D837E838F83D7
:10E9100098878AE50E94C139882351F040E050E091
:10E92000BA018AE50E94473A69877A878B879C8774
:10E93000F090A316F2FAFF24F0F840E061E080E0E6
:10E940000E94589C60E080E50E94A13BE82E1D8655
:10E950001E861F86188A8091A90681113CC02E2D23
:10E96000AE01435F5F4FBE016F5F7F4FCE0149969F
:10E970000E94A571882379F18091190681110F9465
:10E980005B58FF2011F0EE2031F160E080E00E9442
:10E990007772898D9A8DAB8DBC8DB0588D8B9E8B87
:10E9A000AF8BB88F198A1A8A1B8A1C8A1D861E860D
:10E9B0001F86188A8091A906882369F010E000E07C
:10E9C00020E0AE014B5E5F4FBE016F5E7F4FCE0118
:10E9D0000D960E94B56E6C960FB6F894DEBF0FBE12
:10E9E000CDBFDF91CF911F910F91FF90EF90DF90FE
:10E9F000CF900895C12CD12C80E8E82E80E4F82E29
:10EA000045CF2F923F924F925F926F927F928F925B
:10EA10009F92AF92BF92CF92DF92EF92FF920F93AD
:10EA20001F93CF93DF93CDB7DEB7E5970FB6F8947A
:10EA3000DEBF0FBECDBF8DAB2091C0082CAB21E057
:10EA40002093C00880914C058D3409F409C68435A3
:10EA500011F40C942F8A873409F091C180914A05F2
:10EA600090914B058B31910509F4DDC108F079C116
:10EA70008430910508F030C120916F0882309105F3
:10EA800008F48EC1213009F091C111E0029709F01C
:10EA900010E00E945E3A19821A821B821C821D823B
:10EAA0001E821F82188682E50E94C139882309F4DC
:10EAB00090C10E9449396B017C0120E030E0A9013E
:10EAC0000F94A86A882309F4EAC04090D0095090B6
:10EAD000D1096090D2097090D3098091D4099091A6
:10EAE000D509A091D609B091D7098CA79DA7AEA74B
:10EAF000BFA78090A4089090A508A090A608B09009
:10EB0000A7088091A8089091A908A091AA08B0919F
:10EB1000AB0888AB99ABAAABBBABA5019401C30111
:10EB2000B2010F94A86A81110DC028A939A94AA978
:10EB30005BA96CA57DA58EA59FA50F94A86A8823C7
:10EB400009F4ADC0A3019201C501B4010F949971FC
:10EB500020E030E040E05FE30F940E6B68A779A7F8
:10EB60008AA79BA72CA53DA54EA55FA568A979A955
:10EB70008AA99BA90F94997120E030E040E05FE3FF
:10EB80000F940E6B2B013C0120E030E0A901C7017E
:10EB9000B6010F94A86A881F8827881F181709F4E0
:10EBA0000FC180E090E0A0E8BFEB8CA79DA7AEA7C7
:10EBB000BFA728A539A54AA55BA5CA01B9010F942D
:10EBC0000E6B4B015C01A3019201C301B2010F94D2
:10EBD0000E6B9B01AC01C501B4010F949A710F94A7
:10EBE00048744B015C01AC019B01C701B6010F9455
:10EBF000997168AB79AB8AAB9BABA5019401C70156
:10EC0000B6010F949A719B01AC0168A979A98AA9F0
:10EC10009BA90F940E6B6B017C0120E030E0A901F1
:10EC20000F94FA7387FDD1C0C701B6010F944874E1
:10EC30006B017C01C301B2019058A50194010F94AE
:10EC400094722CA53DA54EA55FA50F940E6BA70150
:10EC500096010F940E6B28A539A54AA55BA50F94C4
:10EC60009A7169837A838B839C83A501940168A53B
:10EC700079A58AA59BA50F9494722CA53DA54EA5B8
:10EC80005FA50F940E6BA70196010F940E6BA30165
:10EC900092010F949A716D837E838F83988720E011
:10ECA00030E0A90169817A818B819C810F94A86AE7
:10ECB0008111A3C020E030E0A9016D817E818F81A8
:10ECC00098850F94A86A811198C00E94EF598CE32F
:10ECD00091E10E9461436AC08531910509F466C0E3
:10ECE0008A31910509F49CC0049709F048C080E579
:10ECF0000E94C139C12CD12C7601882321F00E94B9
:10ED00003A2C6B017C0183E50E94C139882361F0B4
:10ED10000E94493920E030E04AE754E40F940E6B3A
:10ED20000F940D736B017C010E9430F480912413C9
:10ED3000811105C060E082E591E10E9457CB0F94FC
:10ED40005D4EC60ED71EE81EF91E0F945D4E6C195F
:10ED50007D098E099F0997FF29C080E00E943061DC
:10ED6000F4CF8A32910509F4F0C260F48D31910537
:10ED700009F418C208F470C04E9709F46CC20F94DD
:10ED8000FA4314C08B35910509F4C2C38C35910543
:10ED900009F4C2C38A35910591F71092DA0806C0CA
:10EDA000213021F40E945E3A0F94A30DFDA9F111C8
:10EDB00002C00F94BE4E2CA92093C0080C94C482AC
:10EDC00080E090E0A0E8BFE3F0CEC12CD12C76012A
:10EDD00031CF89E40E94C139882331F00E9449393A
:10EDE00069837A838B839C838AE40E94C139882358
:10EDF00009F455CF0E9449394ECF412FBE016F5FB4
:10EE00007F4F84EA98E00F94574F0F945D4E6093C4
:10EE1000B6087093B7088093B8089093B908C6CF26
:10EE20000E94F750C3CF87E00F94252D8111BECFEC
:10EE30008CE0E7EAF2E0DE01119601900D928A95EE
:10EE4000E1F770E060E080E50E94CE39BE016F5FBF
:10EE50007F4F0F94791BAACF87E00F943B06811157
:10EE600006C060E08FE40E94A13B81119FCF0E9409
:10EE700030F4109240026091DF088CE40E94A13BC4
:10EE8000E82E80E00E94723E0F945D4E6093B608BB
:10EE90007093B7088093B8089093B9080F9422072D
:10EEA00081E0809329080F9415128AE50E94733936
:10EEB000F82E882369F081E00F943B06182F82E03A
:10EEC0000F943B0611110C94948A11E0811101C03A
:10EED00010E088E50E947339082F81110C94448A50
:10EEE00011110CC089E50E947339811342C1012FB1
:10EEF000F11204C001E011E0FF24F39482E50E94C6
:10EF0000C139882309F438C10E9449396CA37DA313
:10EF10008EA39FA320E030E0A9010F94A86A882364
:10EF200081F0011105C0111103C0FF2009F410C1C7
:10EF300060E0CE0184960F9459080E94B1420E946D
:10EF40006042002309F47FC0112309F479C01092B4
:10EF5000D0091092D1091092D2091092D3091092BF
:10EF6000D4091092D5091092D6091092D7090F949E
:10EF7000650980E39DE20E9416344B015C0184E345
:10EF80009DE20E9416342B013C01AC019B01C5019E
:10EF9000B4010F94FA7318160CF0F3C0A501940194
:10EFA000C301B2010F9494729B01AC010F940E6BDC
:10EFB00020E030E040E85FE30F949A710F944874CA
:10EFC00020E030E048E452E40F940E6B68A379A38C
:10EFD0008AA39BA320E030E040EC5FE3C301B201D1
:10EFE0000F940E6B905869837A838B839C8320E007
:10EFF00030E040EC5FE3C501B4010F940E6B905814
:10F000006C8F7D8F8E8F9F8FAE01405E5F4FBE01F4
:10F010006F5F7F4FCE014C960F9418080F945114D8
:10F020001092D0091092D1091092D2091092D309EE
:10F030001092D4091092D5091092D6091092D709CE
:10F0400080E00F944615112319F081E00F944615C6
:10F05000FF2009F47DC083E00F94252D811178C035
:10F060000F9465092091060930910709409108091C
:10F070005091090960E070E086E193E40F94997182
:10F080002B013C0120910A0930910B0940910C0998
:10F0900050910D0960E070E086E193E40F9499715E
:10F0A0004B015C018091D8099091D909A091DA09AE
:10F0B000B091DB098093AC089093AD08A093AE08A3
:10F0C000B093AF0800912C1610912D16D8012D91F8
:10F0D0003D914D915C91C301B2010F949971609380
:10F0E000A4087093A5088093A6089093A708F80138
:10F0F0002481358146815781C501B4010F949971EE
:10F100006093A8087093A9088093AA089093AB080D
:10F1100084EA98E00E94FD248823C1F11C8E1D8E94
:10F120001E8E1F8E88E0E4EAF8E0DE011196019061
:10F130000D928A95E1F7AE01445E5F4FBE016B5FB1
:10F140007F4FCE0101960F94180882E00F94461568
:10F150000F94650980912808809329088E2D0E94BC
:10F16000723E0F94090783E0809384020F94E610A7
:10F170001DCE012F182FC2CE60E070E080E890E431
:10F18000C5CEA3019201C501B4010CCF60E08DE6AC
:10F1900091E10E9457CB0E94F3598BE591E10E94C7
:10F1A0006143D6CF14E00F945D4E6093B608709320
:10F1B000B7088093B8089093B9088091DF0881114F
:10F1C00027C08EE40E947339882321F08EE791E1F5
:10F1D0000E94C78A87E00F94252D81111FC00E94CD
:10F1E00064688823D9F0115001F130E020E045E651
:10F1F00051E269EA71E185E00E947D4561E08CE9B8
:10F2000091E10E94244584E891E10E94C78ACBCF16
:10F2100060E08FE40E94A13B882399F20E9455454B
:10F2200087E492E10E94C78AC1CD61E08AE392E15E
:10F230000E94244585EC91E10E94C78A61E080E547
:10F2400091E20E94244540E070E060E086EB91E1AD
:10F250000E941C5EABCD00912C1610912D16D8018A
:10F260002D913D914D915C916091D0097091D109A2
:10F270008091D2099091D3090F949A71AB01BC018E
:10F2800088E50E94473A69837A838B839C83F801DF
:10F2900024813581468157816091D4097091D509C7
:10F2A0008091D6099091D7090F949A71AB01BC0156
:10F2B00089E50E94473A6D837E838F839887BE01DC
:10F2C0006B5F7F4FCE0101960E942534882309F49D
:10F2D0006DCD80E00E94723E0F94220761E085E4CC
:10F2E0000E94A13B182F21E0482FBE016B5F7F4F8A
:10F2F000CE0101960F941B456B017C01AC019B0173
:10F300000F948C74811119C049815A816B817C8161
:10F3100089E692E10E944B464D815E816F8178853E
:10F3200084E692E10E944B46B701A6018FE592E187
:10F330000E944B468AE00E9428430F94090711114E
:10F340000E94202C0F94E61031CD80916F088130FF
:10F3500009F02CCD89E40E94C139082FF12C8823B3
:10F3600019F00E944539F82E8AE40E94C139E82E2E
:10F37000882379F00E944539182F002309F4C0C072
:10F38000F4E0FF1508F0B9C081E792E10E94614303
:10F390000DCD10E00111F4CF80E1E0EDF9E0A4EA39
:10F3A000B8E001900D928A95E1F7002319F16F2DD5
:10F3B000FF0C770B880B990B0F94AF6A2091860690
:10F3C0003091870640918806509189060F940E6B04
:10F3D00020917E0630917F064091800650918106F3
:10F3E0000F949A716093A4087093A5088093A6085F
:10F3F0009093A708EE2019F1612F110F770B880B5E
:10F40000990B0F94AF6A20918A0630918B06409138
:10F410008C0650918D060F940E6B209182063091D0
:10F42000830640918406509185060F949A716093EB
:10F43000A8087093A9088093AA089093AB0860E08D
:10F4400080E50E94A13B8823C1F10023D1F0E09127
:10F450002C16F0912D1620813181428153816091CB
:10F46000A4087091A5088091A6089091A7080F9410
:10F4700099716093A4087093A5088093A60890934F
:10F48000A708EE20D1F0E0912C16F0912D162481E2
:10F490003581468157816091A8087091A9088091B3
:10F4A000AA089091AB080F9499716093A808709383
:10F4B000A9088093AA089093AB0840E050E0BA01F5
:10F4C00086E40E94473A6B017C0120E030E0A9010C
:10F4D0000F94FA731816C4F420E030E040E752E4C9
:10F4E000C701B6010F94947269837A838B839C83DE
:10F4F000CE0101960F94561059CCEE2009F44CCF52
:10F50000153008F449CF40CF60E070E0CB01ECCF7C
:10F510008FE08093DA084ACC80914905882381F1F5
:10F52000893009F043CC63EBA62E62E0B62E70ED75
:10F53000C72E79E0D72EE12C00E010E0D5018D91A7
:10F540005D010E94C139F82E882361F0133011F457
:10F55000082FFE2C0E944939F60160837183828353
:10F560009383EF2C1F5FF4E0CF0ED11C143031F7E2
:10F57000EE2009F457C00F9465090F94E61016CCDD
:10F5800053EBC52E52E0D52EF12CE12C00E010E01B
:10F59000D6018D916D010E94C139382E8823D9F191
:10F5A0000E9449394B015C01133059F0F701EC53CB
:10F5B000F64F20813181428153810F9499714B0123
:10F5C0005C01F701E053F64F208131814281538184
:10F5D000C501B4010F9499712B013C012DEB37E368
:10F5E00046E855EB0F94FA7387FD0AC02DEB37E31D
:10F5F00046E855E3C301B2010F94A86A18165CF4FB
:10F600001330C1F48092DC099092DD09A092DE09EA
:10F61000B092DF09032D1F5FB4E0EB0EF11C143034
:10F6200009F0B6CF002309F4A8CF8CED99E00F9430
:10F630007304A3CFF701E650F74F5F01A3019201D6
:10F6400060817181828193810F949A71D5016D934C
:10F650007D938D939C931397812F0F941B06DBCF83
:10F6600080914A0590914B058937910511F40C94CE
:10F67000C08408F0C4C18D34910509F47FC608F038
:10F68000D0C08A31910509F4B4C508F073C0843143
:10F69000910509F4FAC408F050C08131910509F4CC
:10F6A000BBC408F044C0029708F069CB80E50E9413
:10F6B000C139C12CD12C7601882321F00E943A2C2B
:10F6C0006B017C0183E50E94C139882361F00E94AF
:10F6D000493920E030E04AE754E40F940E6B0F9470
:10F6E0000D736B017C010E9430F480915105909163
:10F6F0005205009709F48AC40F941C3480914A057E
:10F7000090914B0562E972E1892B11F46AE872E18C
:10F7100030E020E04AEF55E482E00E947D4540E081
:10F72000C701B6010E943B720F94A0433FCB4297A2
:10F7300009F025CB0E94DC3939CB8731910509F4DA
:10F74000D9C470F48531910509F4D0C4469709F005
:10F7500016CB8091A31682FD29CB0E9495E926CB7A
:10F760008831910509F4DBC4499709F008CB0E9460
:10F7700021741CCB8032910509F4BFC5C0F58D31D1
:10F78000910509F4A3C570F48B31910509F444C5C2
:10F790004C9709F0F4CA80915105909152050F944D
:10F7A000E95A04CB8E31910509F497C54F9709F0BA
:10F7B000E6CA0F9427176C8F7D8F8E8F9F8FBE01A7
:10F7C0006F5F7F4FCE014C960E94CD31CE010196E6
:10F7D0000F941C340E94F359BE016F5F7F4F85E088
:10F7E00093E10E9461608AE00E942843DFCA893465
:10F7F000910509F4AFC550F48132910509F4A6C50D
:10F80000C09709F0BCCA0E94214DD0CA8B34910523
:10F8100009F4B0C58C34910509F0B1CA0F942118D0
:10F82000C5CA8C36910509F4C1CA08F083C0853574
:10F83000910509F492C790F58235910509F47DC7C9
:10F8400020F58E34910509F49DC58135910509F0A7
:10F8500096CA0E9496EC0E9441F40E94E4400E94E5
:10F86000E7401092CB081092CA081092C90868EEBF
:10F8700073E080E090E00E945E400E94E32660E03A
:10F8800080ED93E10E9457CB91CA8335910509F42D
:10F890005CC78435910509F44DCF71CA893691054D
:10F8A00009F460C690F58C35910509F47BC788365C
:10F8B000910509F064CA8091241083FD77CA0E94E3
:10F8C000925A87FD73CA89E40E94C139882311F4D2
:10F8D0000C944A8A0E946B2C90E01816190614F4B6
:10F8E00081E090E026E0289FF001299FF00D11248F
:10F8F000E059F74F808191810E94B2F361E080E08E
:10F900000F944A5E0F94635E51CA8A36910509F4DA
:10F9100054C68B36910509F032CA60E080E50E943A
:10F920003B3A823008F042CAE82FF0E0E25FF54F40
:10F9300010823CCA8237910509F4D5C7A0F58F36ED
:10F94000910509F474C6C8F48D36910509F4ACC567
:10F950008E36910509F013CA8EE40E94C1398823BE
:10F9600009F424CA0E945B2C6093EF107093F0108E
:10F970008093F1109093F21019CA8037910509F421
:10F9800015CA8137910509F0FAC983E50E94C1398A
:10F99000882309F493C60E946B2C8D3308F089C626
:10F9A00080931F0203CA8637910509F4ACC7B8F4E7
:10F9B0008337910509F49FC78537910509F0DFC9A1
:10F9C0008091510590915205009709F498C7DC0188
:10F9D0002C91222309F493C70F941C34E7C987376D
:10F9E000910509F4C9C78837910509F0C8C981E0B4
:10F9F00080932908809328080F941512D7C982395B
:10FA0000E1E09E0711F40C94E58708F095C1833D71
:10FA1000910511F40C94A48508F0F6C0883C91057A
:10FA200011F40C94418508F06CC08139910509F4FA
:10FA3000AFC760F58D37910509F499CE8C389105E3
:10FA400009F09DC98091241083FDB0C989E40E940A
:10FA5000C139882311F40C94708A0E946B2C90E0B9
:10FA60001816190614F481E090E026E0289FF001B2
:10FA7000299FF00D1124E059F74F828193810E9454
:10FA80003A3961E080E00F944A5E90C98B39910564
:10FA900009F42CC68E3B910509F071C980912410A0
:10FAA00083FD84C989E40E94C139882311F40C9430
:10FAB0007B8A0E946B2C90E01816190614F481E0E2
:10FAC00090E026E0289FF001299FF00D1124E059D5
:10FAD000F74F8281938110E00E943A3960E081E023
:10FAE0000F944A5E2091E6083091E7088091E4087F
:10FAF0009091E508821793070CF0EDC581EC93E136
:10FB0000ECC58C3C910511F40C949C8540F5893C26
:10FB1000910509F4E7C78B3C910509F030C90E94B3
:10FB2000925A87FD43C913EBE12E12E0F12E10E04B
:10FB300000E0D7018D917D010E947339882349F03F
:10FB40000E944939F801EB5DFF4E64A375A386A3BB
:10FB500097A30C5F1F4F0031110559F727C98D3C42
:10FB6000910511F40C94A085B6E0EB2EB9E0FB2EC4
:10FB700010E08E3C910509F002C988E5810F0E94D2
:10FB80007339882351F00E944939F70160837183EA
:10FB900082839383812F0F941B061F5FF4E0EF0E87
:10FBA000F11C133051F780914F0587FDE6CC809111
:10FBB0005005837009F0E1CC409106095091070986
:10FBC000609108097091090986E094E10E944B4612
:10FBD00040910A0950910B0960910C0970910D092F
:10FBE00083E896E40E944B4640910E0950910F091C
:10FBF000609110097091110980E896E40E944B46CB
:10FC00008AE00E942843D2C88D3221E0920711F485
:10FC10000C94A58608F06AC08831A1E09A0711F417
:10FC20000C94058608F043C08C3D910509F490C7FB
:10FC30008D3D910509F0A3C80E94925A082F87FDB7
:10FC4000B5C883E50E94C139002E000C110B780164
:10FC5000EE0CFF1C882309F4BEC70E944539F7014A
:10FC6000E35CFD4F91838083000F111F000F111F74
:10FC700098012B573D4F7901BC01990F880B990BC7
:10FC80000F94AF6A2AE037ED43E25CE30F940E6B0A
:10FC90000B5F194FD8012D913D914D915C910F94BF
:10FCA0000E6BF70160837183828393837FC88232F6
:10FCB000E1E09E0711F40C94A1868C32914009F08A
:10FCC0005EC864E071E083E50E94CE398C0168EE85
:10FCD00073E080E50E94CE39893823E1920710F065
:10FCE00088E893E1B8010E947A9660C8803321E0E9
:10FCF000920711F40C94278768F48E32A1E09A07DA
:10FD000011F40C949B878F32914009F038C80E94FF
:10FD1000E1464CC88039E1E09E0711F40C94E1877C
:10FD20008139914009F02BC88091B508811125CC0B
:10FD300081E00F94CB1321CC883F31E0930711F47D
:10FD40000C94578908F0E6C08C3AB1E09B0711F497
:10FD50000C942C8808F0B3C08D39F1E09F0711F4A2
:10FD60000C94128A88F58A3931E0930709F41EC889
:10FD70008C39914011F00C94BF7680914D058878B4
:10FD800011F00C94ED8780914F05867011F00C9462
:10FD9000ED870E94F35983EB94E10E9461438091C7
:10FDA0005D020E942D464091590250915A02609185
:10FDB0005B0270915C0283E994E10E944B468AE009
:10FDC0000E9428430C94D676843AB1E09B0711F444
:10FDD0000C941D88853A914011F00C94BF766FEF1A
:10FDE0007FEF89E40E94923B082F6FEF7FEF8AE458
:10FDF0000E94923B182F8AE50E94C139D12C8111B3
:10FE000008C081E50E94C139D82E882311F40C94D2
:10FE10008C8AC02E81E0800F863010F00C942488EC
:10FE2000912E81E0810F863010F00C9424880E947E
:10FE300049392B013C01F02E07FDF12C07FF02C0D0
:10FE400004E0C02E812E17FD812C17FF02C014E0A4
:10FE5000912EB5E03B2ECF1410F40C94D676E82CFE
:10FE60003F9C500111249E1410F40C9421880E2DF7
:10FE700010E020E030E0A901DD2069F0F501E00F9D
:10FE8000F11FEE0FFF1FEE0FFF1FE65EF94F2081FF
:10FE90003181428153810A0D1B1D000F111F000F7C
:10FEA000111F065E194FC301B2010F949A71D80158
:10FEB0006D937D938D939C931397E394D4CF853F5B
:10FEC000F1E09F0711F40C944F8978F4863E31E0FD
:10FED000930711F40C94DD88843F914011F00C9449
:10FEE000BF760E9415F00C94D676863FB1E09B0752
:10FEF00011F40C945389873F914011F00C94BF7614
:10FF000061E083E50E94A13B91E089270F94C6251B
:10FF10000C94D6768335F3E09F0711F40C94FE8998
:10FF200028F58B3532E0930711F40C947A8978F434
:10FF30008C30B2E09B0711F40C94698988359240AB
:10FF400011F00C94BF760E9411730C94D6768D3B01
:10FF5000F2E09F0711F40C94FA898E3B924011F065
:10FF60000C94BF760E94C5700C94D676873E33E021
:10FF7000930711F40C94028AC8F48C36B3E09B0703
:10FF800011F40C94D676803A934011F00C94BF761D
:10FF900020915105309152059091A3169260909353
:10FFA000A316C9010F94E95A0C94D676883EF3E063
:10FFB0009F0711F40C942B8A893E934011F00C9406
:10FFC000BF760F94625A81110C94D6760E94B63B8C
:10FFD0000F94205A0F9427176D33710581059105F1
:10FFE00020F085E795E10E94C78A81E795E10E94AC
:10FFF000C78A84EE80935B058DE595E10E9461439D
:020000021000EC
:1000000089E595E10E94C78A0C94D67660E08AE97A
:1000100092E10E9457CB72CB80914D0584FD17C0B1
:1000200080914F0587FD13C080915005837079F44E
:1000300060E08DEA92E10E9457CB5F988A988091A8
:10004000080181708093060112980C94D67688E599
:100050000E94733981115F9889E50E94733981117B
:100060008A988AE50E947339882329F080910801D3
:1000700081708093060185E40E947339882311F40E
:100080000C94D67612980C94D6768091A31683FFA2
:1000900025C085EC92E10E9461438091A31683FF05
:1000A00017C084EC96E10E9479EA8BE1E4ECF6E17A
:1000B000DE01119601900D928A95E1F770E060E003
:1000C000CE0101960F94B520CE0101960E94DE3B31
:1000D00086EB92E10E9461430C94D6760E94F3591C
:1000E00086ED92E10E9461430C94D6760E94A6E9C7
:1000F0000C94D6768091510590915205FC01219186
:10010000222331F02032D9F7DF0111971C92F7CF6B
:1001100060E00F94325B10925B050C94D67683E519
:100120000E94C139882321F00E945B2C0E94742A0E
:1001300084E50E94C1398823A9F00E945B2C6B01E1
:100140007C010F94CE17C0920906D0920A06E09265
:100150000B06F0920C06CD28CE28CF2819F081E0AE
:100160008093D9088091A9068823F9F080E090E077
:10017000A0EAB1E489839A83AB83BC831C8E1D8E75
:100180001E8E1F8E18A219A21AA21BA210E000E058
:1001900020E0AE014F5F5F4FBE01645E7F4FCE0136
:1001A00080960E94B56E0C94D6760E94AD4088234E
:1001B00081F00E94EEE10E94D14080E599E00F9429
:1001C00071591092561110925711109258111092A5
:1001D000591161E08DE991E20E94244545E651E222
:1001E00060EE72E185E00F9412450F94A0430C94E9
:1001F000D6768091A31683FD02C00C94D67683E553
:100200000E94C139882311F40C94D6760E945B2C8D
:100210000E94742A0C94D67683E40E947339882352
:1002200061F186EF92E10E94614380910B1888236F
:10023000F9F0BE016F5F7F4F88E098E10E940CEA01
:10024000CE0101960E9413E6CE0101960F94BB5A8F
:100250008091E112882339F080E20E94284381EEE8
:1002600092E10E9413E68AE00E9428430C94D6761D
:100270008CEE92E10E946143F6CF83E50E94C13982
:10028000882301F10E946B2C182F8C3308F08CE32B
:10029000809324050F945D4E6B017C01212F30E08B
:1002A000A8EEB3E00F944071C60ED71EE81EF91EEB
:1002B000C0922005D0922105E0922205F0922305FC
:1002C0000C94D6760F9438590C94D6768091A31658
:1002D0008E7F8093A3160C94D6768091A31683FD0F
:1002E00002C00C94D6760F94E04380915105909112
:1002F00052050F94B8590C94D6768091A31682FDBE
:100300000E9430F48091A31683FD02C00C94D6762F
:1003100060E080E50E94A13B182F682F8091510575
:10032000909152050F94325B83E50E94C139882376
:1003300021F00E945B2C0E94742A0E94EEE11111B0
:100340000C94D6760E94D1400C94D6760E946B60B5
:100350000C94D67680E50E947339882311F40C94AE
:10036000D6760E946B2C853608F084E680935B0578
:100370000C94D6760E94D1400C94D6760E94E4402C
:100380000C94D67670E060E083E50E94923B8E3458
:10039000910531F40E9451F30F94A0430C94D6764A
:1003A00080E793E10E9461436091180870911908F9
:1003B00087E693E10E94394660911A0870911B0804
:1003C0008AE593E10E9439466091180870911908F6
:1003D00080911A0890911B08681B790B8091D908AD
:1003E000815021E030E0823010F030E020E0621BEC
:1003F000730B8FE493E10E9439468AE00E94284300
:1004000087E493E10E94614380911C0890911D084C
:10041000A0911E08B0911F088C8F9D8FAE8FBF8F4B
:10042000BE016F5F7F4FCE014C960E94CD31BE0161
:100430006F5F7F4F8AE393E10E94616080912008A3
:1004400090912108A0912208B09123088C8F9D8F54
:10045000AE8FBF8FBE016F5F7F4FCE014C960E9463
:10046000CD31BE016F5F7F4F8AE293E10E946160F0
:1004700020E030E04AE754E46091240870912508B8
:1004800080912608909127080F949472AB01BC01CB
:1004900082E193E10E944B468DE60E9428438AE068
:1004A0000E9428430C94D6768091241083FF02C0CA
:1004B0000C94D6760E94925AF82E87FF02C00C94B4
:1004C000D67689E40E94C139882311F40C94558AA8
:1004D0000E946B2C90E01816190614F481E090E04D
:1004E00026E0289FF001299FF00D1124E059F74FD5
:1004F0008081918110E00E94B2F361E081E00F946D
:100500004A5E2091951530919615809193159091A2
:10051000941582179307F4F483E893E19F938F93E4
:100520008EE893E19F938F931F920E943CCB0F9094
:100530000F900F900F900F9001E00F94635E0023D7
:1005400011F40C94D67640E0612F8F2D0F9438244F
:100550000C94D67688E793E1112301F3012FEDCFB8
:10056000182FEBCF0E94925A182F87FD0AC083E9FB
:1005700093E10E946143812F0F9440228AE00E9400
:1005800028433CA93093C008E5960FB6F894DEBF27
:100590000FBECDBFDF91CF911F910F91FF90EF90D4
:1005A000DF90CF90BF90AF909F908F907F906F9093
:1005B0005F904F903F902F90089560E080E50E94FB
:1005C0003B3AF82E81E08F1510F40C94D67681E436
:1005D0000E94733960910E0A062F10E0811102C04B
:1005E0000FEF10E089E40E94C139882309F46EC737
:1005F0000E946B2C90E01816190614F481E090E02C
:1006000026E0289FF001299FF00D1124E059F74FB3
:1006100004811581EF2DF0E0E25FF54F0F3F1105EA
:1006200019F010F00FEF10E000830C94D67683E5FC
:100630000E947339882331F060E083E50E943B3AE1
:10064000809324100E94F35984EA93E10E9461434D
:1006500080912410882351F110E000E020E0809187
:10066000241090E0B0E0A0E0002E04C0B695A7955D
:10067000979587950A94D2F780FF12C0FF24F394D0
:10068000F20E222319F08CE20E942843F801EE0FAB
:10069000FF1FE656FC4E859194910E9461432F2DD9
:1006A0000F5F1F4F05301105D1F6DDCD86E993E1CF
:1006B000E1CD8CE380931F020C94D6760E94F3590F
:1006C00060911F028BEA93E10E9443468AE00E94F8
:1006D00028430C94D67682EB93E160E00E9457CBDE
:1006E00060E0812F0F94B3220C94D67683E50E94AC
:1006F000C139882311F40C94D6760E946B2C182FE4
:100700008C3308F08CE3809329050F945D4E6B01C8
:100710007C01212F30E0A8EEB3E00F944071C60EAB
:10072000D71EE81EF91EC0922505D0922605E0923C
:100730002705F09228050C94D6768091DA088F7DF3
:1007400080618093DA080C94D6768091DA088F7EE7
:1007500080628093DA080C94D67683E50E94733920
:10076000882311F40C94D6760F945D4E6093B608EE
:100770007093B7088093B8089093B9080E944939DC
:1007800020E030E04AE754E40F940E6B0F940D73B1
:1007900060932A0570932B0580932C0590932D056B
:1007A0000C94D6760E94925A87FF02C00C94D6769B
:1007B00080914D0584FD09C080914F0587FD05C0DE
:1007C00080915005837009F489C023EBC22E22E08A
:1007D000D22E35E2E32E30E1F32E10E0D6018D91DA
:1007E0006D010E94C139882309F465C0133009F0F6
:1007F0006DC00E9449394B015C0120E030E040EAC5
:1008000051E40F94A86A87FF4EC0A501940160913E
:1008100045107091461080914710909148100F94A8
:1008200094722B013C01AC019B016091F209709123
:10083000F3098091F4099091F5090F940E6B609380
:10084000F2097093F3098093F4099093F509A301D9
:1008500092016091551070915610809157109091AF
:1008600058100F940E6B6093551070935610809330
:100870005710909358106091020A7091030A80916A
:10088000040A9091050A0F94AD6AA30192010F9496
:100890000E6B0F940D736093020A7093030A80939A
:1008A000040A9093050A8092451090924610A092F7
:1008B0004710B09248101F5FF4E0EF0EF11C1430A7
:1008C00009F08CCF0E940CF40C94D6760E94493922
:1008D000F701648B758B868B978BEDCF81E00F943E
:1008E00065430C94D6760F94004383E396E10E940F
:1008F00063EF0C94D6760E9488430C94D6760F94BE
:10090000A0430C94D676009151051091520594E0C5
:10091000F12C40E09150F9F0F8018081282F2B7FD5
:10092000213499F421812133B1F4813411F18534DA
:1009300009F441E098012E5F3F4F89012F5F3F4F3F
:10094000F80180818032C9F3E5CF803521F48181BF
:1009500080538A3078F341110E94F359FF2021F02F
:1009600081EE93E10E946143C8010E942F430C94E1
:10097000D676FF24F394DECF0F94CA110C94D6766A
:1009800010922908109228080F9415120C94D6760C
:1009900070E060E083E50E94923B823040F00E946C
:1009A000EF5984EE93E10E9461430C94D6768C015A
:1009B000112788E40E94C1398823C1F00E9445397B
:1009C0008A3A91050CF44BC00E9445398D32914012
:1009D0000CF048C00E94453926E0209FF001219F7D
:1009E000F00D1124E059F74F9183808382E40E9437
:1009F000C1398823A9F00E9445390597B4F10E94B6
:100A000045398D389105A4F50E94453926E0209F8F
:100A1000F001219FF00D1124E059F74F9383828359
:100A200086E40E94C139882311F40C94D6760E9482
:100A3000453997FD20C00E9445398F3F910509F047
:100A4000ECF40E94453926E0209FF001219FF00D33
:100A50001124E059F74F958384830C94D6768AEA63
:100A600090E0BACF8CE291E0B7CF85E090E0CECFB6
:100A70008CE890E0CBCF90E080E0E5CF8FEF90E086
:100A8000E2CF0E94925A182F87FF02C00C94D676AC
:100A90000091F90884E40E94C139F82E8823B1F04E
:100AA0000E9449394B015C0120E030E0A9010F941C
:100AB000A86A8823A9F024E01202F0011124EB5067
:100AC000F74F80829182A282B3820F2D602F83E53F
:100AD0000E94A13B8093F9080E941EDD0C94D676FB
:100AE00080E0F8CF0E94925A87FF02C00C94D6761D
:100AF00003EB12E085E2E82E80E1F82E97EBC92E99
:100B000092E0D92ED8018D918D010E9473398823EE
:100B100059F00E9449390F940D73F7016083718376
:100B2000828393830E94BEF3F4E0EF0EF11CC016A3
:100B3000D10641F70C94D6760E945C460C94D6768A
:100B40000E9423440C94D6760E94B75A0C94D67611
:100B500082E40E947339882341F08091760290915B
:100B60007702909321028093200282E50E947339DC
:100B7000882341F080912002909121029093770286
:100B80008093760283E50E94C139882331F00E9468
:100B90004539909377028093760280914D0590912C
:100BA0004E05A0914F05B0915005892B8A2B8B2BB8
:100BB00011F00C94D67660917602709177028DE0F8
:100BC00094E10E94D54B85E20E9428438AE00E946E
:100BD00028430C94D6760E94F35985E40E9428435A
:100BE00080E3800F0E942843F701E35CFD4F6081A2
:100BF000718181E194E10E94D54B85E20E942843F6
:100C00008AE00E9428430C94D67680E50E947339CE
:100C1000882311F40C94D6760E9445398C01892BD7
:100C200009F082C083E50E947339882391F00E9405
:100C300045398F3F980731F48DE196E10E94EE40EF
:100C40000C94D676BC018DE196E10E945C410C9437
:100C5000D6760E94F35970E060E08CE194E10E9446
:100C6000D54B80911F1658E5C52E52E0D52EC81AD7
:100C7000D10887FDD394CC0CDD1CCC0CDD1C0D2CD5
:100C8000000CEE08FF0880911E1678E8872E912C44
:100C9000881A910887FD9394880C991C880C991CDC
:100CA000092C000CAA08BB0880911D1690E08F3F0C
:100CB000C9F1FC01EE0FFF1FE80FF91FEC52FA4ECD
:100CC0008181928133E0880F991F3A95E1F7B0E076
:100CD000A0E044E0B595A795979587954A95D1F7FB
:100CE00002969C012F5F3F4F032E000C440B550BC7
:100CF000281939094A095B09A4EBB0E00F942D715A
:100D0000A7019601281939094A095B090F940E7148
:100D1000B90189E194E10E94D54B8AE00E94284301
:100D20000C94D67680E0DDCF0E94EF59B80183E3C2
:100D300094E10E94D54B84E294E10E9461430C94BB
:100D4000D6760E94F7590C94D67660E085E40E942E
:100D50003B3A811174C080E50E947339882351F0B9
:100D60000E944939609398157093991580939A154C
:100D700090939B1589E40E947339882381F00E9427
:100D800049392CEA35EC47E25EE30F940E6B609331
:100D90009C1570939D1580939E1590939F1584E4E8
:100DA0000E947339882381F00E9449392CEA35EC7E
:100DB00047E25EE30F9494726093A0157093A115BF
:100DC0008093A2159093A3150E94F3594091981512
:100DD0005091991560919A1570919B1582E494E158
:100DE0000E944B462CEA35EC47E25EE360919C158D
:100DF00070919D1580919E1590919F150F949472FE
:100E0000AB01BC018EE394E10E944B462CEA35EC29
:100E100047E25EE36091A0157091A1158091A21543
:100E20009091A3150F940E6BAB01BC018AE394E182
:100E30000E944B468AE00E9428430C94D6760E947A
:100E4000EF5986E494E10E9461430C94D67680E5E4
:100E50000E947339882351F00E9449396093E90850
:100E60007093EA088093EB089093EC0889E40E9461
:100E70007339882381F00E9449392CEA35EC47E226
:100E80005EE30F940E6B6093ED087093EE08809311
:100E9000EF089093F00884E40E947339882381F06E
:100EA0000E9449392CEA35EC47E25EE30F949472D4
:100EB0006093F1087093F2088093F3089093F4081C
:100EC0000E94F3594091E9085091EA086091EB08BB
:100ED0007091EC0880E694E10E944B462CEA35ECD8
:100EE00047E25EE36091ED087091EE088091EF08B3
:100EF0009091F0080F949472AB01BC018CE594E1E1
:100F00000E944B462CEA35EC47E25EE36091F10823
:100F10007091F2088091F3089091F4080F940E6B91
:100F2000AB01BC0188E594E10E944B468AE00E9437
:100F300028430C94D67683E50E947339182F8823B2
:100F400069F00E9445399C0190938A02809389023E
:100F500091E0232B09F090E09093200A80E50E9415
:100F60007339882361F02091890230918A02232B02
:100F700011F00E947F2C8093200A0C94D6761111D8
:100F80000C94D6760E94F35980E894E10E94614364
:100F90008091200A882391F088E694E10E946143C1
:100FA0006091890270918A028FE694E10E94D54B8C
:100FB0008BE694E10E9461430C94D67684E694E13A
:100FC000EDCF0E9430F40C94D6760E941C340E941F
:100FD000202C0F94E6100C94D67688E40E94733986
:100FE000882321F00E947F2C80932E0582E50E94A9
:100FF0007339082F83E50E947339182F011102C03D
:10100000882341F00E94CE26112321F00E947F2CDC
:1010100080935D0284E40E947339882311F40C9458
:10102000D6760E9449396093590270935A02809390
:101030005B0290935C020C94D6760E94A65B0C94A3
:10104000D676F3940C942B7F0E94EF5984EE94E1B2
:101050000E9461430C94D67687E00F94252D811170
:101060000C94D67664E2C62E6DE2D62EE0EDF9E061
:10107000F9A7E8A79E012F5F3F4F1901790110E002
:1010800000E0C6010E941634A8A5B9A58D909D90D8
:10109000AD90BD90B9A7A8A7A50194010F9499712F
:1010A0002B013C01F701408251826282738220E071
:1010B00030E040EA51EC0F94FA7387FD0AC020E05B
:1010C00030E040EA51E4C301B2010F94A86A181657
:1010D00084F4F801E85BF24DE4911E1654F4B7FA7B
:1010E000B094B7F8B094D7018D929D92AD92BC9216
:1010F0001397F70181909190A190B1907F0120E02A
:1011000030E040EA51ECC501B4010F94FA7387FD59
:101110003FC020E030E040EA51E4C501B4010F9443
:10112000A86A1816ACF10F5F1F4FF4E0CF0ED11C68
:101130000330110509F0A5CF56E0E52E59E0F52E54
:1011400010E0F10181919191A191B1911F01F701FD
:1011500081939193A193B1937F01812F0F941B06EB
:101160001F5F133071F70F94E61060E08DEF94E18C
:101170000E9457CB63E972E084E690E00E947A9681
:101180006AEB72E084E690E00E947A960C94D67640
:101190000E94EF598BE195E10E94614361E08DE08F
:1011A00095E10E9457CB0E946F9B68E270E088EC4B
:1011B00090E00E947A960C94D67684E50E9473396A
:1011C0008823A1F010925C0510925D0510925E05D7
:1011D00010925F05109260058FEF0E94822A61E0F5
:1011E00070E084E50E94923B8093600583E50E9455
:1011F0007339882321F00E9445390E94822A83E4B2
:101200000E947339882331F080912F02803210F4CC
:101210000E94593C80E50E947339882331F00E9476
:101220004539803210F40E94593C85E50E9473399B
:10123000882311F40C94D6760E944539803210F040
:101240000C94D67641E050E060E070E0082E04C0D7
:10125000440F551F661F771F0A94D2F7409550958B
:101260006095709500915C0510915D0520915E057B
:1012700030915F05402351236223732340935C0523
:1012800050935D0560935E0570935F0590912F020A
:1012900089130C94D676109223100C94D6760F9462
:1012A0000F2D0C94D6760F9424120C94D67620939E
:1012B0008E060F94032D10928E06882311F40C9441
:1012C000D6760E94F35989E395E10E9461430C941C
:1012D000D6768091A31682FF05C080648093A31602
:1012E0000C94D67683FD02C00C94D6760F94E0431E
:1012F0000C94D6760E94925A082F87FF02C00C9455
:10130000D67685E50E947339882359F10E944939C0
:101310004B015C01E02E002E000CFF0820E030E0C5
:10132000A9010F94FA7387FF04C0B7FAB094B7F815
:10133000B09420E030E84BE354E4C501B4010F94CD
:10134000FA73970143E0220F331F4A95E1F72F5EAE
:10135000394F1816D4F1D9018D929D92AD92BC925D
:1013600013978CE40E947339882311F40C94D67679
:101370000E9449396B017C01002E000C110B20E00A
:1013800030E0A9010F94FA7387FF04C0F7FAF094D4
:10139000F7F8F09420E030E84BE354E4C701B601DD
:1013A0000F94FA73980193E0220F331F9A95E1F797
:1013B0002F5E394F18169CF0D9011496CD92DD920C
:1013C000ED92FC9217970C94D67680E090E8ABE310
:1013D000B4E4F90180839183A283B383C2CF80E018
:1013E00090E8ABE3B4E4F90184839583A683B783E3
:1013F0000C94D6760E94BC6D0C94D6760E94DF4B7E
:101400000C94D67681E080936F081092791360E097
:1014100083E50E94A13B81110C94D6760F94273569
:101420000C94D67683E50E947339882341F00E949C
:101430007F2C809319060E94BE3B0C94D6760E94A6
:10144000F35984E495E10E946143809119060E945A
:101450002D460C94D6760E94398B0C94D67610913A
:101460004A050F945D4E6093B6087093B708809359
:10147000B8089093B908112311F40C94D676812FF3
:101480000E944CEC0C94D67611110C94777711E0F5
:101490000C94727783E50E94C139882311F40C946F
:1014A000827C0E9445390C947C7C83E50E94C13982
:1014B000182F811107C082E50E94C139082F8823A7
:1014C00009F44EC80E9445390C947B8283E50E9442
:1014D000C139882309F49EC80E945B2C8B019AC8ED
:1014E00083E50E94C139882311F40C94D6760E94BA
:1014F00045390C943F7D83E50E94C139182F811135
:1015000007C082E50E94C139882311F40C94D67675
:101510000E9445390C946C7D0E94EF5984EC94E153
:101520000E9461430C94D676882309F4B0CF0C94C2
:101530007A77DF92EF92FF920F931F93CF93DF930F
:10154000EC01E090C208F090C3088AE0D82E6AE06F
:1015500070E0CE010F94EF748C01009711F0FC0144
:101560001082CE010E94AC3281E00E94017501150B
:10157000110519F0E801D992EACFC701DF91CF91A7
:101580001F910F91FF90EF90DF900C94AC324F922F
:101590005F926F927F928F929F92AF92BF92CF9203
:1015A000DF92EF92FF920F931F93CF93DF93CDB70C
:1015B000DEB77C014DB65EB66090C2087090C3087D
:1015C0008DB69EB66AE070E0C7010F94E3696C01C6
:1015D0008C010E191F09892B21F4C7010F94F5699D
:1015E0008C01C80101962DB73EB7281B390B0FB6E9
:1015F000F8943EBF0FBE2DBF8DB79EB701965C011C
:10160000A801B7010F94166AF501E00FF11F1082CF
:10161000C5010E94AC3281E00E940175C114D10461
:1016200051F076019FEFE91AF90A0FB6F8949EBEC1
:101630000FBE8DBEC5CF0FB6F8949EBE0FBE8DBE39
:10164000C3010E94AC320FB6F8945EBE0FBE4DBE11
:10165000DF91CF911F910F91FF90EF90DF90CF908E
:10166000BF90AF909F908F907F906F905F904F90C2
:1016700008954F925F926F927F928F929F92AF9256
:10168000BF92CF92DF92EF92FF920F931F93CF936F
:10169000DF93CDB7DEB7C059D1090FB6F894DEBFDE
:1016A0000FBECDBF0E94CC3B882369F083E50E942A
:1016B0007339882301F120E040E070E060E089E9BF
:1016C0009BE90E948099C057DF4F0FB6F894DEBFA8
:1016D0000FBECDBFDF91CF911F910F91FF90EF9083
:1016E000DF90CF90BF90AF909F908F907F906F9042
:1016F0005F904F90089583E40E947339882319F016
:101700000E948E9BE0CF8090B9099090BA09A0907A
:10171000BB09B090BC098091C20980FF05C09091BF
:101720002410986090932410869581708093200AED
:101730008EE191E10E94C78A809148099091490900
:101740009E012F5F3F4F7901009799F09F938F93F0
:1017500085E191E19F938F933F932F930F943F6A7D
:10176000C7010E94998A0F900F900F900F900F90D1
:101770000F908091460990914709009799F09F93A7
:101780008F938CE091E19F938F93FF92EF920F9450
:101790003F6AC7010E94998A0F900F900F900F9097
:1017A0000F900F906E0131E8C30ED11C6091250996
:1017B000709126098091270990912809860123E0DC
:1017C00041E00F9475659F938F938AEF90E19F930B
:1017D0008F93FF92EF920F943F6AC7010E94998AFC
:1017E00082EF90E10E94C78A87E08093B4088093DB
:1017F00004060F900F900F900F900F900F90809114
:1018000041098823F9F06091420970914309809160
:1018100044099091450923E041E00F9475659F9339
:101820008F9389EE90E19F938F93FF92EF920F94A5
:101830003F6AC7010E94998A0F900F900F900F90F6
:101840000F900F9080914A098823A1F01F928F93E7
:101850001F921F928CED90E19F938F93FF92EF92D6
:101860000F943F6AC7010E94998A0FB6F894DEBFB1
:101870000FBECDBF80914B098823A9F01F928F9393
:101880001F9281E08F938CED90E19F938F93FF9255
:10189000EF920F943F6AC7010E94998A0FB6F8949D
:1018A000DEBF0FBECDBF40904C0950904D096090F7
:1018B0004E0970904F0920E030E0A901C301B20148
:1018C0000F94A86A811104C08091C20982FF20C0D0
:1018D000860121E041E0C301B2010F9475659F9339
:1018E0008F938091C20982FB882780F91F928F9382
:1018F0008FEC90E19F938F93FF92EF920F943F6A4A
:10190000C7010E94998A0FB6F894DEBF0FBECDBF03
:1019100060911709709118098091190990911A091D
:101920008E010F581F4F23E041E00F947565782E0C
:10193000692E609113097091140980911509909195
:101940001609860123E041E00F9475656F927F923E
:101950009F938F938EEB90E19F938F93FF92EF92E3
:101960000F943F6AC7010E94998A60911B09709188
:101970001C0980911D0990911E0923E041E00F94FC
:10198000756583EB90E10E94C78ADF92CF9289EA66
:1019900090E19F938F93FF92EF920F943F6AC7015C
:1019A0000E94998A809124098F93809123098F93B3
:1019B00082EA90E19F938F93FF92EF920F943F6A98
:1019C000C7010E94998A60911F0970912009809136
:1019D00021099091220923E041E00F9475659F93BE
:1019E0008F9388E990E19F938F93FF92EF920F94EA
:1019F0003F6AC7010E94998A8CE0E9E2F9E0A6E01B
:101A0000B9E001900D928A95E1F78CE0E5E3F9E009
:101A1000AAEFB8E001900D928A95E1F780E00F946B
:101A20001B0681E00F941B0682E00F941B06809139
:101A3000C1098093DA0881E0809319060E94BE3BB9
:101A400080E599E09F938F9385E39DE39F938F9328
:101A5000FF92EF920F943F6A0FB6F894DEBF0FBE6D
:101A6000CDBFC7010E94998A8091C0098F93809150
:101A7000BF098F938091BE098F938091BD098F9389
:101A8000BF92AF929F928F928AE890E19F938F933B
:101A9000FF92EF920F943F6AC7010E94998A0FB696
:101AA000F894DEBF0FBECDBF0ECECF93DF93C091B3
:101AB0005B11C093E50981E6C89FE0011124C35A78
:101AC000DE4E8091241080FF05C00E94F359CE01A4
:101AD0000E942F43CE010E94AC3280E0DF91CF9173
:101AE0000C94017560913D0270913E02072E000C2E
:101AF000880B990B0F94AF6A2AE037ED43E25CE361
:101B00000F940E6B20910506309106064091070652
:101B1000509108060F940E6B6093850270938602B5
:101B200080938702909388020895E0919F08E230A5
:101B300030F4F0E0E25FF54F80918D0880830895E6
:101B4000809198168823C1F0815080939816E4EC18
:101B5000F6E1882351F08150990B2BE1289FF00189
:101B6000299FF00D1124E650F94E8BE1AFEDB6E15F
:101B700001900D928A95E1F720919816211105C0E8
:101B80008091A31680628093A31681E090E0A0E08C
:101B9000B0E0211103C080E090E0DC018093850873
:101BA00090938608A0938708B093880810928A08BB
:101BB00081E08093840883E0809384020895CF932A
:101BC000DF93EC01CB01BA010F94AF6A29EC38EC3A
:101BD00048EC5EE30F94947220E030E040E05FE375
:101BE0000F949A710F940D736883DF91CF910895CC
:101BF000E0919F0886E0E802F0011124E059F74FD8
:101C000080918D0890E09583848308958F929F92B0
